:10000000005600201D6300006D6200007D6200004C
:1000100095620000AD620000C562000000000000B3
:10002000000000000000000000000000DD62000091
:10003000ED62000000000000FD6200000D630000A2
:1000400055620000000000000000000025FD0000D7
:1000500055FC0000D1FC0000000000000000000082
:10006000214200001DE10000FDE000006DFD0000E8
:100070000000000000000000000000008DFD0000F6
:100080002DE9F843054688464FF0A0441C4EDFF8A2
:1000900078901C4F237E002BFCD1A37E2BB94FF010
:1000A00001022274A37E002BFBD072B6735DF3B9FC
:1000B00000F02EF8C0B90122D9F8103043F0040343
:1000C000C9F8103087F83220BFF34F8F00BF30BF20
:1000D00087F83200D9F8103023F00403C9F8103043
:1000E000BFF34F8F62B6D5E700BF30BFFAE70023FA
:1000F0007355B8F1000F00D0C04762B6BDE8F88371
:10010000202700200000105000ED00E0000000005B
:100110005FF800F069410000FFFFFFFFFFFFFFFFF6
:10012000FFFFFFFFFFFFFFFFFFFFFFFFFFFFFFFFDF
:10013000FFFFFFFFFFFFFFFFFFFFFFFFFFFFFFFFCF
:10014000FFFFFFFFFFFFFFFFFFFFFFFFFFFFFFFFBF
:10015000FFFFFFFFFFFFFFFFFFFFFFFFFFFFFFFFAF
:10016000FFFFFFFFFFFFFFFFFFFFFFFFFFFFFFFF9F
:10017000FFFFFFFFFFFFFFFFFFFFFFFFFFFFFFFF8F
:10018000FFFFFFFFFFFFFFFFFFFFFFFFFFFFFFFF7F
:10019000FFFFFFFFFFFFFFFFFFFFFFFFFFFFFFFF6F
:1001A000FFFFFFFFFFFFFFFFFFFFFFFFFFFFFFFF5F
:1001B000FFFFFFFFFFFFFFFFFFFFFFFFFFFFFFFF4F
:1001C000FFFFFFFFFFFFFFFFFFFFFFFFFFFFFFFF3F
:1001D000FFFFFFFFFFFFFFFFFFFFFFFFFFFFFFFF2F
:1001E000FFFFFFFFFFFFFFFFFFFFFFFFFFFFFFFF1F
:1001F000FFFFFFFFFFFFFFFFFFFFFFFFFFFFFFFF0F
:10020000FFFFFFFFFFFFFFFFFFFFFFFFFFFFFFFFFE
:10021000FFFFFFFFFFFFFFFFFFFFFFFFFFFFFFFFEE
:10022000FFFFFFFFFFFFFFFFFFFFFFFFFFFFFFFFDE
:10023000FFFFFFFFFFFFFFFFFFFFFFFFFFFFFFFFCE
:10024000FFFFFFFFFFFFFFFFFFFFFFFFFFFFFFFFBE
:10025000FFFFFFFFFFFFFFFFFFFFFFFFFFFFFFFFAE
:10026000FFFFFFFFFFFFFFFFFFFFFFFFFFFFFFFF9E
:10027000FFFFFFFFFFFFFFFFFFFFFFFFFFFFFFFF8E
:10028000704700BF034613F8012B002AFBD1181A50
:100290000138704700487047A8C701002420704704
:1002A0000520704708B505F053FF08BD08B505F0F7
:1002B000CDFF43690148984708BD00BFA8C70100AA
:1002C00010B50C4611461A46012807D010B1022875
:1002D0000BD010BDE0B200F041F8FAE7BDF80830ED
:1002E000C9B2E0B200F07CF8F3E7E0B200F02AF91E
:1002F000EFE700BF044B00229A80DA805A819A818E
:10030000B4221A81704700BF24280020014B1878BE
:10031000704700BF2428002010B40446034B0FCBC5
:1003200084E80F00204610BC704700BF282800203A
:1003300082B0094B5B690020DAB262F30700C3F3B5
:10034000072262F30F20C3F3074262F317401B0E2C
:1003500063F31F6002B070472428002010B50446E4
:100360001D4B1B7813F0030F02D010F00C0F15D1AA
:1003700014F0030F1CD113F0080F02D014F0040F77
:1003800022D113F0040F15D014F0080F12D0124B25
:1003900000229A80DA80B4221A810BE005F0D8FEA0
:1003A00002690D4B1A61FFF7A5FF00F001F901E0AA
:1003B000FFF7A0FF084B1C70084C204600F032FEEF
:1003C000204600F025FB10BD034B00229A80DA8006
:1003D000B4221A81EEE700BF24280020B0C7010034
:1003E00010B5044600F046FF042C00D010BDFFF706
:1003F0008DFF10F00C0F05D000F045FF0368984703
:1004000000F0E0F84B4C204600F05AFE204600F089
:10041000A5FB494B1A78042A37D0082A4AD0464B04
:100420005B89B3F5616F05D3434B002159819989ED
:1004300001319981404B99894EF66023994251D000
:100440003D4BD9884EF6602399424FD03A4B99885C
:100450004EF6602399424DD012F0080FC6D000F03E
:1004600012FF0368984703689847002846D1324B2B
:100470001B7813F0080FB9D02E4800F05BFE00285F
:1004800048D02D4BB4221A81B0E72B49CB880133D9
:100490009BB2CB802949A1FB0301490901EB8101F2
:1004A000A3EBC1039BB2002BB9D123494B89013384
:1004B0004B81B4E720490B89013B0B818B880133C9
:1004C0009BB28B801E49A1FB03014909C1EB0111BD
:1004D000A3EB81039BB2002BA1D117494B890133B8
:1004E0004B819CE7144B00219981A9E7124B002115
:1004F000D980ABE7104B00219980ADE700F0C3FE37
:100500000368984700F067FD0128B0D10A4BB42278
:100510001A81ACE7084B1B7813F0080F3FF466AF65
:10052000054B1B89002B7FF461AF05F08FFE03683C
:1005300098475BE7B0C7010024280020CDCCCCCC85
:100540008988888810B5062819D8DFE800F01904D2
:100550001D201823260005F0FBFD044605F076FE5D
:10056000C3684FF48062002120469847FFF7C2FE1F
:100570000D4800F057FD04F1F00000F036FA10BD10
:10058000094800F073FDFAE7084B1975F7E7074BC8
:100590005975F4E7054B9975F1E7044BD975024895
:1005A00000F040FDEBE700BFB0C7010024280020A9
:1005B00008B580220021024818F04BFA08BD00BFA0
:1005C0003C2800202DE9F04F85B082460022924958
:1005D00011F832306FF3C71301F8323001EBC20368
:1005E00058786FF3C710587098786FF3C7109870E9
:1005F000D8786FF3C710D87018796FF3C7101871D7
:1006000058796FF3C710587198796FF3C7109871C4
:10061000D8796FF3C710D8710132102AD8D1DAF81F
:100620000030984703900023029345E04FF0010803
:100630004FF0140CB5423AD801974FF04C093346AD
:10064000464698462BE04FF001084FF0140CF1E7B6
:10065000425C42F08002425402F07F0202EB0C0B3B
:10066000BBF14C0F0FDD425C69F3060242540133CB
:100670009BB29C420FD319461EF80320D209E7D043
:10068000002EF4D0E4E7624410F801B062F3060BE8
:1006900000F801B0EBE70135ADB2A84507D3A7429A
:1006A000F9D8019B5C4A02EBC50E7046E3E7029B5A
:1006B000013302930A2B66D09DF80880DAF81C30CB
:1006C00040469847012805D0DAF81C304046984744
:1006D0000228ECD1DAF80C30404698478146DAF827
:1006E000103040469847834603014C4A82FB03265C
:1006F000F218DE17C6EBE2264FEAC903484A82FB2E
:1007000003271F44DB17C3EBA727DAF81430404652
:100710009847DAF8083040469847002814BF10245C
:100720000224B6B2351B25EAE575ADB226440F2E7C
:10073000A8BF0F26B6B2BBB21F1B27EAE777BFB22E
:100740001C44072CA8BF0724A4B2DAF8083040469E
:100750009847A9F143091FFA89F940F2B233994544
:100760003FF664AFBBF16E0F7FF66DAF002814BF8C
:100770004FF0140C4FF0010C002814BF4FF001088B
:100780004FF0000856E70026234F1FE0043AE55CCF
:1007900062F30605E55404E0013AE55C62F3060500
:1007A000E5540133082B0ED0C25CD209F9D1C25CEA
:1007B00002F07F02122AEFD8032AE7D8E25C6FF337
:1007C0000602E254EDE70136102E04D0002307EBB9
:1007D000C6000446E8E7039B1BB1002421460E4DEA
:1007E00005E0FFF7E5FEF8E70134102C0DD00023FB
:1007F00005EBC400C25C02F07F02092A84BF01310C
:1008000089B20133082BF5D1EEE7034BA3F8801032
:1008100005B0BDE8F08F00BF3C280020E1000EE0ED
:1008200049D6B9F22DE9F04F83B00646019114463E
:100830000368984770B13E4A92F88230013382F8DB
:100840008230A146002C5ED00027B8469346DFF8E0
:10085000E8A037E0FFF7ACFE4FF00008019B83F8FB
:10086000008055E0F3682046984740B3336920463E
:10087000984720B3F36820469847054633692046D9
:10088000984700018AFB00230344C017C0EBE32014
:1008900080B2ED00274B83FB05232B44ED17C5EBFE
:1008A000A325ADB20BEBC000435D03F07F03122B19
:1008B00005D808F101085FFA88F8019B1C70013720
:1008C0004F4510D0FCB2F369204698470128C9D0A3
:1008D000F369204698470228C4D0F3692046984718
:1008E0000328ECD1BEE7B8F1000F0CD0104BB3F8E1
:1008F0008030402B10D8B8F1010F09D012D9002355
:10090000019A137004E04FF00008019B83F8008007
:10091000404603B0BDE8F08F4FF00008019B83F81C
:100920000080F5E74FF00008019B83F80080EFE7B7
:100930003C28002049D6B9F2E1000EE0431E9BB2EC
:100940004FF6FD7293421CD84B1E9BB293421AD8AD
:1009500009010E4B83FB01231944C1F3CF21C000D1
:100960000B4B83FB00231844C0F38F20094B03EB90
:10097000C101085C00F07F0013288CBF002001201B
:100980007047012070470120704700BFE1000EE072
:1009900049D6B9F23C280020F8B506460F4C256828
:1009A000238903EB83035B00F4336B8005F04EFC7B
:1009B0000435238903EB830307690A22314605EBDB
:1009C0004300B847238901339BB2238122685278C0
:1009D0009A4201D800222281F8BD00BFC028002021
:1009E000704708B5FFF7D8FF08BD10B5044605F0FD
:1009F0002DFCC3684FF44472002120469847034BF6
:100A00001C60462363700A23237010BDC028002099
:100A100030B5A5B00446436898474F4B1B7913F097
:100A2000030F09D0A368984710F0080F21D1A368DD
:100A3000984710F0040F1CD1474B1B7913F00C0F93
:100A400009D0A368984710F0020F41D1A3689847D6
:100A500010F0010F3CD1A36898473F4D2871E3681F
:100A600004A89847BDF81830EB8000236B8125B0AF
:100A700030BD002501950295ADF80C5005F0E6FB60
:100A8000C3680A22294601A898479DF8043002222B
:100A900062F302038DF80430E36810A89847BDF8AC
:100AA0000430BDF8462062F30F13ADF80430E3685C
:100AB0000CA89847BDF83E30ADF80630E36808A8AA
:100AC00098470B9BADF8083001A8FFF765FFB3E727
:100AD000002501950295ADF80C5005F0B7FBC368F1
:100AE0000A22294601A898479DF80430032262F3A0
:100AF00002038DF8043063689847BDF8043002881B
:100B000062F30B13ADF80430134A52891209C3F390
:100B1000072362F307138DF80530E36820A8984790
:100B2000BDF88230ADF80630E3681CA89847BDF8E0
:100B30007030ADF80830E36818A89847BDF86E30FB
:100B4000ADF80A30E36814A89847179BADF80C304D
:100B500001A8FFF721FF7EE7C02800202DE9F04F14
:100B6000A7B0044643689847A368984710F0080F59
:100B700004D1A368984710F0040F3BD0236898472E
:100B800003689847054600F026FA90B12368984715
:100B9000036898478046002603960496ADF81460D3
:100BA00002460A2103A800F002FA37464FF00A096C
:100BB000A4E0284600F013FA0028E7D163689847BC
:100BC000B0F86030002B40F02B81944BDD8801356C
:100BD000E36816A89847BDF860309D4200F08F8109
:100BE000E3680DA898478D4BBDF83C20DA805A8900
:100BF00001325A8127B0BDE8F08FDAF80C30284670
:100C00009847DAF8103028469847236898470368D1
:100C10009847824600F0EBF9051EC0F2FA8063683F
:100C20009847C388ADF80430636898470389ADF8E6
:100C30000630636898474388BDF804201344ADF834
:100C40000830636898478388BDF806201344ADF8E0
:100C50000A30EDB2DAF80C30284698478346DAF8C5
:100C600010302846984701AA0146584600F078F906
:100C7000002840F0D0804FF4C973ADF8043040F63E
:100C80005C03ADF8063040F2A623ADF8083040F61C
:100C90001613ADF80A30DAF80C3028469847834628
:100CA000DAF810302846984701AA0146584600F065
:100CB00057F9003018BF01209DF81E3060F345132E
:100CC0008DF81E306368984790F86330C3F30203D1
:100CD0009DF8202063F302028DF820206368984776
:100CE00090F86230C3F30203BDF8202063F388124A
:100CF000ADF8202006A8FFF74FFE0136D8F80030E7
:100D00009847F3B28342BFF459AFF3B226AA134413
:100D100013F88C5C06970797ADF82070D8F81C3054
:100D200028469847012805D0D8F81C30284698470F
:100D30000328E2D123689847036898478246E3680E
:100D400009A89847BDF828B005F080FAC3684A465C
:100D5000394606A898479DF818306FF302038DF8BE
:100D60001830DAF81C3028469847012814BF0020B4
:100D700001209DF8183060F3C3038DF81830BDF8DA
:100D80001830BDF82A2062F30F13ADF818304FEA7F
:100D90001B129DF81A3062F303038DF81A309DF888
:100DA0001C306BF303038DF81C30DAF80C30284646
:100DB0009847BDF81A3060F30F13ADF81A30DAF81F
:100DC000103028469847BDF81C3060F30F13ADF87B
:100DD0001C302369984711909DF81E30C0B260F313
:100DE00001038DF81E30DAF81830284698479DF830
:100DF0001E3060F383038DF81E3003F00C030C2BC0
:100E00007FF4FBAE9DF81E3043F00C038DF81E30CE
:100E1000F3E6384650E701204EE700BFC028002027
:100E2000002309930A93ADF82C3023689847036890
:100E30009847064600F0DBF8051E4FDB05F006FA82
:100E4000C3680A22002109A898479DF8243001228E
:100E500062F302038DF82430E36812A89847BDF8C6
:100E60002430BDF84E2062F30F13ADF824306368D0
:100E7000984790F8603013F0020F3AD163689847B2
:100E800090F8603013F0040F35D16368984790F8FC
:100E9000603013F0080F30D16368984790F86030E5
:100EA00013F0100F14BF062200229DF8263062F3C3
:100EB00003038DF82630EDB2F36828469847BDF855
:100EC000263060F30F13ADF8263033692846984773
:100ED000BDF8283060F30F13ADF8283009A8FFF7EC
:100EE0005BFD636898470023A0F860301B4A53817C
:100EF0006BE60122D9E70422D7E70522D5E70025D2
:100F000009950A95ADF82C5005F0A0F9C3680A229E
:100F1000294609A898479DF82430042262F3020369
:100F20008DF82430E36822A89847BDF82430BDF836
:100F30008E2062F30F13ADF82430E3681EA89847A3
:100F4000BDF88630ADF82630E3681AA898471D9B97
:100F5000ADF8283009A8FFF71FFD41E6C0280020A2
:100F6000134672B1128882420DD89A8882420CD3FD
:100F7000DA888A420BD3588888428CBF002001202F
:100F80007047002070470020704700207047002005
:100F9000704710B50446084611460023224600F06B
:100FA000B3F90021204600F0DCF9C0B210BD08B54D
:100FB000002300F0A9F908BD08B500F0A5F908BDA7
:100FC00008B5002100F0CDF9C0B208BD08B500F0A9
:100FD000C8F9C0B208BD08B500F06EF908BD08B583
:100FE00000F07EF908BD08B500F052F908BD08B55B
:100FF00000F0DEF908BD000010B54368984704888A
:10100000003418BF012405F021F98368224603212A
:101010000220984705F01AF983682246032104202C
:10102000984710BDF8B507460F4B1B68BBB10024AD
:1010300025460D4E56F8253053B156F825309847C1
:1010400003682BB156F8253098470368384698470F
:101050000134E4B2254656F82430002BEAD1384654
:10106000FFF7CAFFF8BD00BF1C120020F8B5074605
:10107000124B1B68F3B100242546104E56F825305C
:101080008BB156F82530984743683846984750B199
:1010900056F825309847C3682BB156F82530984745
:1010A000C368384698470134E4B2254656F82430E0
:1010B000002BE3D13846FFF79FFFF8BD1C1200203C
:1010C0002DE9F04107461A4B1B68002B2DD0002458
:1010D0002646174D05E00134E4B2264655F8243083
:1010E0001BB355F82630002BF5D055F8263098471D
:1010F0004368384698470028EDD055F82630984781
:1011000090F81480BB68984718EA000FE3D055F8B0
:10111000263098478368002BDDD055F82630984755
:101120008368384698470028D5D0BDE8F08100BFD5
:101130001C1200202DE9F04107461C4B1B68002BB8
:1011400032D000242646194D05E00134E4B226468B
:1011500055F824302BB355F82630002BF5D055F830
:10116000263098474368384698470028EDD055F810
:101170002630984790F81480BB68984718EA000F0B
:10118000E3D055F8263098470369002BDDD055F899
:10119000263098470369384698470028D5D0012063
:1011A00000E00020BDE8F0810020FBE71C120020D9
:1011B00008B5436898470078C0F3400008BD704701
:1011C00030B587B0044603689847036898470246DD
:1011D0001F4903A800F0B9FC9DF8153013F0020F69
:1011E0002ED0BDF80C30CD3B9BB240F29D229342F5
:1011F00029D8BDF80E2040F67B039A4225D99DF8E8
:101200001430043BDBB2382B01D9002019E0002355
:10121000019302934FF00203012565F387138DF8C4
:10122000043005F013F8436801A8984763689847AD
:1012300090F8603043F0020380F86030284600E008
:10124000002007B030BD0020FBE70020F9E700BF19
:10125000CC28002008B54FF49F7354224021024847
:1012600000F05EFC08BD00BFCC280020004870479D
:10127000C4C7010008B5022800D008BD19461046B1
:1012800000F00AFDF9E70148704700BFDCC7010024
:1012900038B505460368984748B10024AB68E0B20A
:1012A0009847034630B901340A2CF7D100E00023F7
:1012B000184638BD0123FBE738B505460368984753
:1012C00050B10024EB69E0B29847012806D0013400
:1012D0000A2CF7D1002000E0002038BD0120FCE7F7
:1012E00038B505460368984750B10024EB69E0B271
:1012F0009847032806D001340A2CF7D1002000E0DB
:10130000002038BD0120FCE72DE9F84F82468946D0
:101310001646984600252F4609E07B1CDBB20AF8EA
:1013200007404B451BD01F4601350A2D17D0ECB2A4
:10133000F369204698470028F6D0F368204698477E
:101340008346336920469847B8F1000FE5D04246FE
:1013500001465846FFF704FE0028DED1E4E7BDE869
:10136000F88F2DE9F843074688460024264604E016
:101370000136F6B201340A2C17D0E5B2FB692846D3
:1013800098470028F6D0FB682846984781463B6975
:1013900028469847B8F1000FEAD042460146484631
:1013A000FFF7DEFD0028E3D1E4E770B2BDE8F88383
:1013B00038B505460368984760B10024EB69E0B290
:1013C000984728B901340A2CF8D14FF0FF3038BDC6
:1013D00060B2FCE74FF0FF30F9E7000008B5436862
:1013E00098470078C0F3C00008BD064B43221A801E
:1013F0006F225A8040F2F5329A8040F6F502DA8088
:10140000704700BFE8280020F0B585B005460368A6
:101410009847036898470246204902A800F05BFA03
:101420009DF80830022B03D00024204605B0F0BD03
:10143000BDF80A70BDF80C60194A31463846FFF70E
:101440008FFD04460028F0D00023009301934FF055
:101450000203042262F38503012464F387138DF8E9
:10146000003047FA02F38DF8023046FA02F38DF8A5
:10147000033006F00F0646EA07168DF8046004F004
:10148000E5FE4368684698476B68984790F8603077
:1014900043F0080380F86030C7E700BFF028002061
:1014A000E828002010B584B00D4C46230393642334
:1014B00002931E230193032200921223012104F1BF
:1014C000080000F0E1F9432323806F23638040F29A
:1014D000F533A38040F6F503E38004B010BD00BFF0
:1014E000E828002000487047E0C7010008B54368BD
:1014F0009847037813F0240F14BF0120002008BD83
:1015000038B543689847C58804894188294482884A
:101510002244034B5D809C80D9801A8138BD00BF76
:101520001C2900202DE9F04784B080464368984785
:101530000378C3F38009C3F34017D8F80030984705
:10154000036898473C4E024606F1140102A800F0D9
:10155000C2F99DF808A0BDF80A50BDF80C40B21CB5
:1015600021462846FFF7FCFC30BB06F10A02214663
:101570002846FFF7F5FC034600285AD1184604B068
:10158000BDE8F0872C4B1A700023F7E71FB32A4BF6
:101590001B78012B1FD00023F0E7D8F804309847C0
:1015A00090F8603043F0040380F860300123E5E7F1
:1015B0000023E3E70023E1E70022BAF1010FE1D0C5
:1015C000BAF1020FF4D1B9F1000FDFD01FB91A4BF5
:1015D0001B78002BEED1002301934FF00203012270
:1015E00062F3850362F387138DF80030124E33786F
:1015F0008DF801302B118DF8023023118DF8033056
:1016000004F00F0444EA05158DF8045004F01EFEA2
:101610004368684698473378002BBED0D8F804302A
:10162000984790F8603043F0200380F86030012341
:10163000A4E70122C1E700BF1C29002070B586B0D5
:101640000646036998470590040E0CBF6423832364
:10165000002C0CBF46220A22194D03920293242328
:1016600001930723009312230322022105F11400A2
:1016700000F00AF973689847C688018942883244A5
:1016800083880B446E80A980EA802B81002C14BFD4
:101690006521432140F21A3208BF6F2240F2D33055
:1016A00040F2F533002C14BF04461C466981AA8120
:1016B000EC8140F6F5022A8200222A7006B070BD45
:1016C0001C29002000487047F8C7010010B50446E7
:1016D000C28A038A9A4202D901234375837494F81B
:1016E0002530012B0FD0227D0A4B53F822302046A3
:1016F000984701280CD0022814BF00200220638DD7
:101700000133638510BD042363750123A374EAE7E5
:101710000120F4E72C120020C289B0F91830B0F98A
:1017200020105B1A002BB8BF5B42934218DCB0F963
:101730001A30B0F922105B1A002BB8BF5B429A42F4
:1017400010DBB0F9262043889A4207DCB0F92A3032
:1017500040898342CCBF00200120704700207047A1
:10176000002070470020704770B5044690F8245060
:10177000012D05D9AB1EDBB2012B08D9002070BDAD
:10178000012383740020207503236375F7E7C68C5B
:10179000013636B2C684FFF7BFFF08B90123A37430
:1017A000032D01D00020EAE723889E42BCBF01231D
:1017B000A37463889E42C4BF0123A37400232375CE
:1017C000E27C237B9A4201D00020D8E7B4F928308C
:1017D000A2889342BCBF0122A274E2889342C4BF94
:1017E0000123A374B4F92A3022899342BCBF012299
:1017F000A27462899342C4BF0123A374002323858A
:10180000A37C4BB10020A0746685A38B2383E38B5C
:1018100063830123E374B2E70023E3740220AEE79D
:1018200010B5044690F8243023B9038D01330385A5
:10183000002010BD012B25D1FFF76EFF18B9022340
:1018400063750123A3740122E284E37C1344DBB2B9
:10185000E3742275B4F92010A183B4F92220E28345
:101860003BB1A37C2BB9E07C012814BF00200120F0
:10187000DFE70020A0740123638520852183628334
:10188000E374F0E70020D4E730B4BDF80850BDF8A9
:101890000C400280438001FB02F292B2AB1A8380BB
:1018A000A21AC280058144810173BDF81030C38142
:1018B000BDF81430038200238374C3740385438509
:1018C000C38443754FF6FF72028342838283C283CF
:1018D000037530BC7047F0B585B005460C4616461A
:1018E000002301930293ADF80C30498B208BFFF756
:1018F00025F8D0B10A2201A93046FEF793FF01284E
:1019000022D90023A374E37423856385E38463757C
:101910004FF6FF7222836283A283E28323752B70CA
:101920006B80AB80284605B0F0BD0023A374E37440
:1019300023856385E38463754FF6FF722283628398
:10194000A283E2832375D5E79DF80470E0B1F368C4
:101950003846984720843369384698476084F3694D
:101960003846984784F824003046FFF73CFB98B986
:10197000002384F825302046FFF7A8FE228B638BD6
:1019800028706A80AB80CDE74FF6FF7323846384B1
:10199000002384F82430E7E7012384F82530EAE7C0
:1019A00070B504460E461578CB692846984701283D
:1019B00001D0012070BD002323806380A380E380D9
:1019C00023816381A381E38123746374227E02F007
:1019D000F80263F3C3022276F36828469847A08191
:1019E000336928469847E081237C01332374E0E77C
:1019F0002DE9F04104460F461678CB6830469847EB
:101A000080463B69304698470546FB693046984713
:101A1000032841D0A389A8EB03031BB22380B4F9A8
:101A200002209A42B8BF1A4616466280B4F9047082
:101A30009F42A8BF1F46A780E089281A00B2E08015
:101A4000B4F908208242B8BF02462281B4F90A10D4
:101A50008142A8BF01466181B4F9125001EB050C27
:101A6000604553DA491B884250DD521B904203DC2B
:101A7000227E42F002022276EA1993424BDA7F1B61
:101A8000BB4248DD721B9342DEBF237E43F0080356
:101A900023760120BDE8F08100232374B4F90020EF
:101AA000E38A9A4222DB217E01F00801002914BF5B
:101AB0000020102059428A4206DC227E12F0040FD8
:101AC00004BF40F00800C0B2B4F9062093420FDC16
:101AD000237E13F0020F0BD140F00400C0B29142FC
:101AE000D8DB237E13F0010F08D0D3E70020E1E715
:101AF000914207DB237E13F0010F03D140F0020077
:101B0000C0B2C7E7002808BF0120C3E7217E41F02B
:101B100001012176A9E7227E42F004022276B1E794
:101B200041828282C3820023038043808380C380FA
:101B3000038143818381C38103744374027E02F075
:101B4000F80263F3C302027670472DE9F04186B0D4
:101B500004460D46164600238DF81730314903AA76
:101B600003C982E8030000930193ADF808300A220C
:101B700069463046FFF70DFA80469DF800708DF8F3
:101B80001770F36938469847002831D0B8F1010F33
:101B90002ED1736938469847AB8A834228D3B368FD
:101BA0003846984720BBF3689DF817009847804651
:101BB00033699DF81700984707462B7C06AA02EB6D
:101BC000830353F80C3C0DF1170231462846984721
:101BD000A989EA896B7C5E1C6E7421806280A4F8FE
:101BE0000480E78023726072204606B0BDE8F08171
:101BF00000232B806B80AB80EB802B816B81AB81D2
:101C0000EB812B746B742A7E02F0F80263F3C3023B
:101C10002A7623806380A380E3802372012363728A
:101C2000E2E700BF10C80100014B1888704700BFF1
:101C30005C2900200A207047024B5B6803EB001010
:101C4000807B70475C290020024B5B680001185CB8
:101C5000704700BF5C290020024B5B6803EB00105B
:101C6000408870475C290020024B5B6803EB001042
:101C7000808870475C290020024B5B6803EB0010F2
:101C8000008970475C290020024B5B6803EB001061
:101C9000407870475C290020014B198058607047DC
:101CA0005C2900200048704718C8010000487047B0
:101CB0001800002000487047E404002010B5064CCE
:101CC00004F110000CF098F9207504F118000CF0E4
:101CD00099F92077204610BD4C050020024A4FF4A8
:101CE000F071024809F048B81C9701002C0500204B
:101CF0000149024809F0CCB81C9701002C050020CE
:101D0000024A4021024809F037B800BF309701006D
:101D1000700500200149024809F0BAB83097010067
:101D2000700500200048704788050020704700BFFC
:101D3000704700BF10B5054C04F10C000CF05CF9C5
:101D4000E36820752361204610BD00BFD805002040
:101D5000004870473000002070B546780C4CB50044
:101D6000294604F114000B4A09F006F831462046D2
:101D7000094A09F001F82946201D084A08F0FCFF2D
:101D8000294604F10800064ABDE8704008F0F4BF97
:101D9000140600202098010034980100509801009A
:101DA0006C98010010B50A4C0A4904F1140009F0BE
:101DB0006FF82046084909F06BF8201D074909F023
:101DC00067F804F108000649BDE8104009F060B862
:101DD0001406002020980100CC970100E497010030
:101DE000FC97010010B5054C04F10C000CF004F94F
:101DF000E36820752361204610BD00BF3406002033
:101E0000004870474800002010B5074C074A04F10D
:101E100008000C2108F0B0FF2046BDE81040044A3D
:101E2000062108F0A9BF00BF7006002098980100A5
:101E3000B098010010B5064C064904F1080009F0FD
:101E400027F82046BDE81040034909F021B800BF3B
:101E50007006002098980100B09801000048704773
:101E6000A0050020704700BF704700BF10B5064CAA
:101E700004F10C000CF0C6F8207504F110000CF011
:101E8000C7F8204610BD00BFA806002000487047D4
:101E90006000002070B506780C4CB500294604F1AE
:101EA00014000B4A08F068FF31462046094A08F042
:101EB00063FF2946201D084A08F05EFF294604F109
:101EC0000800064ABDE8704008F056BFE40600204E
:101ED0002C99010040990100589901007099010066
:101EE00010B50A4C0A4904F1140008F0D1FF20464D
:101EF000084908F0CDFF201D074908F0C9FF04F18B
:101F000008000649BDE8104008F0C2BFE406002002
:101F10002C99010040990100589901007099010025
:101F200010B5064C04F10C000CF06CF8207504F1AF
:101F300010000CF06DF8204610BD00BF0407002013
:101F40002DE9F0410CF054F80446FFF7B7FE0546C2
:101F5000FFF748FF0746FFF7E3FF224606462946FC
:101F6000012001F04BFE22462946022001F046FEE8
:101F7000FFF7E0FE8046FFF779FF0546224641461F
:101F8000092001F03BFE224629460A2001F036FED8
:101F900022463946052001F031FE22463146062010
:101FA00001F02CFEFFF79AFEBDE8F041FFF7A8BE56
:101FB00010B5FFF7C5FF094B1B689847084B1B6816
:101FC0009847084B1B689847BDE81040064A074BE6
:101FD000127853F822305B68184700BF9011002038
:101FE000F4100020BC1000205D160020209A010093
:101FF00070B5FFF763FE0446FFF7F4FE0646FFF7F1
:102000008FFF0546FFF774FEFFF784FE214601208F
:1020100001F042FE2146022001F03EFE314605203D
:1020200001F03AFE2946062001F036FEFFF782FE57
:102030000546FFF71BFF04462946092001F02CFE48
:102040002146BDE870400A2001F026BE70B500248C
:102050009CB011AE214630462C220BADCDE90B448D
:10206000CDE90D440F94ADF8404016F0F2FC08ABFA
:10207000CDE90233CDE90544CDE900560648049385
:1020800009940894CDF827402B4604682A4629462F
:102090000B20A0471CB070BDEC2900200B4A0C4B54
:1020A000127810B553F82230DB689847FFF7CEFF5F
:1020B000FFF79EFF074B1B699847074B1B69984723
:1020C000BDE81040054B1B69184700BF5D16002096
:1020D000209A010090110020F4100020BC10002074
:1020E00070B5064607F00AFA194D012804462B7808
:1020F0001CD09EB99C421BD0012B1AD0154E56F80D
:102100002330DB68984720462C7007F0FDF92B78C8
:1021100056F82330BDE870405B681847012E12D096
:10212000032EE7D1022B03D00224E5E7012B00D1D7
:1021300070BDFFF7B3FF20462C7007F0E5F9BDE84E
:102140007040FFF735BF002BF2D00024D4E700BF6A
:102150005D160020209A0100614A2DE9F04F1278A7
:10216000604B8BB053F822305F4C9B689847C0F3AC
:10217000074307930990C0F3072A07F0CBF90646F7
:1021800007F0CCF9B379227883469A4204D0B0792B
:1021900005F03AFCB3792370544B0124986804F09D
:1021A000B9FF0025ED23DFF868815148DFF854912D
:1021B000504F0593224621464346CDE90309CDE918
:1021C00001550094642000F09BF93B6898F80020CA
:1021D0009978914213D0F321CDE901552546464A1D
:1021E000023305910392CDF81090009422462146C7
:1021F000642000F085F93B689B7888F800300CF08B
:10220000F3F93B688DF82300DB7883422CD1BBF1D6
:10221000000F3ED1002D3CD1079B002B43D0737E95
:10222000002B49D1337E002B55D1079B012B01D1C7
:102230000DF056FF7222314B00921A683049314B33
:10224000632000F0A5F9FFF729FFFFF7B1FE772221
:102250002D4B00921A682A492A4B632000F098F906
:1022600001200BB0BDE8F08F01224FF481710023F3
:102270002648CDE90491CDE9013303900DF1230304
:1022800064200092114600F03BF93B68D8780CF0CE
:1022900097F9002007F048F9337E002BCAD00020C0
:1022A00007F032F9C6E7337E7BB95046FFF718FFD7
:1022B00001200BB0BDE8F08F337E002BF5D028460F
:1022C00007F022F94FF0010AEFE7079807F01CF931
:1022D0004FF0010AE9E7284607F016F9A5E700BF25
:1022E0005D160020209A01005C160020080A0020DC
:1022F000EC990100340A0020F89901004C070020F5
:1023000094990100DC99010050070020149A010003
:10231000840700202DE9F04792B00446884607F074
:10232000F9F800233F4FC27DC7E900333B81002A03
:1023300056D094F82B0094F82AA094F82990504590
:1023400094F8281038D8A0F1160EC21FA0F10F067D
:102350005FFA8EFED2B2F6B2894521D84B4612E022
:10236000A3F10A04022C4ED800EB431438F91450A0
:10237000012437F914C0AC45B8BF27F81450013315
:10238000DBB299420CD3022AEAD9022E2BD89C1F29
:10239000022C28D800EB4315022438F91550E8E741
:1023A0000130C0B20EF1010E0132013682455FFAF2
:1023B0008EFED2B2F6B2CFD23E2200210DF10A003B
:1023C00016F047FB002340F20155822400971A467D
:1023D00002A91E20ADF808508DF80D4007F038FA1C
:1023E00012B0BDE8F087BEF1020FC8D8A3F10A040D
:1023F000022C11D99C1E022CC1D800EB431438F9D1
:1024000014500324B5E79C1E022CB8D800EB4314EB
:1024100038F914500024ACE700EB431438F9145099
:102420000424A6E760160020F0B5204E83B00546D0
:1024300001F1200014461F467160FDF723FF1C4B7D
:102440001C4A99682130376048609460607822782F
:10245000E37802FB00F203F07F0303FB02F3164C68
:1024600022790B60D3B2012B01D003B0F0BD7721EC
:10247000FF221E46114F397022712379FF2B10D194
:1024800020222946684616F0B5FA009B032B04EB80
:10249000830206DC019BD2F8052006FA03F31342FF
:1024A000EBD105233B7003B0F0BD00BF1C20002022
:1024B000580A00203C0C0020DC200020080B0020E3
:1024C00070B504460E461546049A194620F8022BAC
:1024D00020341E2216F07CFB20463146DF2216F007
:1024E00077FB45B13046FDF7CDFE2946C0F1DF024E
:1024F000204416F06DFB2046BDE87040FDF7C2BEDB
:10250000F0B5C5B004460E4615460146202204A883
:102510001F4616F06FFA049B032B0EDC01221B48AA
:10252000059900EB8303D3F805C002FA01F313EA1F
:102530000C0F02D00379934201D045B0F0BD4F9B00
:102540004D99009300224E9B04A8FFF7B9FF4FF06E
:10255000000E9DF80BC04A9B4B9A63F3060C8DF856
:102560000F0020464C9C62F3C71C3B4604A902AAFC
:102570008DF808608DF809508DF80E408DF80BC06D
:102580008DF80CE0FFF750FFD7E700BFDC200020FC
:10259000F0B5C5B004460D4616460146202204A8F3
:1025A0001F4616F027FA049B032B0EDC0122154868
:1025B000059900EB8303D3F805C002FA01F313EA8F
:1025C0000C0F02D00379934201D045B0F0BD4A9B75
:1025D0003246009329463B4604A8FFF771FF0025C9
:1025E0008DF80F0004A902AA20462B46ADF808502A
:1025F0008DF80B508DF80C508DF80E50FFF714FF2E
:10260000E3E700BFDC200020F0B5644687B001F0AE
:1026100069FD002601F0B8FD0125042040F22F37A6
:102620002369A268DB68E168CDE901560090064D98
:1026300006480597CDE903057220FFF761FF23697E
:10264000D86807B0F0BD00BFB09B0100189B010027
:102650002DE9F04F91F81CE090F802C00F460EFBF8
:102660000CF5097D85B00191DDF838804DB3444605
:10267000002605EB450C08EB0C1C226294F8245054
:1026800084F8246094F8255084F8256094F8265046
:1026900084F8266094F8275084F8276094F828502E
:1026A00084F8286094F8295084F8296094F82A5016
:1026B00084F82A6094F82B5084F82B603034A445B9
:1026C000DBD1BEF1000F32D03D460026074603F1B4
:1026D000FF3921B3CB4600242B69062213F804A04E
:1026E00002A84FEA6A01013116F084F9BA780AF0BB
:1026F000010306FB0233029A03EB4303920002EB51
:102700000313039943441BF8012F186A01EB81015D
:102710008A4002431A622B7D0134A342DCDC2B7F0A
:102720000136019AB342914401DD297DD1E705B01C
:10273000BDE8F08F2DE9F041002482B0089D2A62A7
:102740002A6595F8242085F8244095F8252085F8F9
:10275000254095F8262085F8264095F8272085F80D
:10276000274095F8542085F8544095F8552085F871
:10277000554095F8562085F8564095F8572085F82D
:10278000574095F8282085F8284095F8292085F8A5
:10279000294095F82A2085F82A4095F82B2085F8BD
:1027A0002B4095F8582085F8584095F8592085F821
:1027B000594095F85A2085F85A4095F85B2085F8DD
:1027C0005B400A7D12B30F465E1E3B69062213F87A
:1027D000048068464FEA6801013116F00BF908F0F1
:1027E0000108009A4FEA48039844930003EB08134A
:1027F00001992B4416F8012F186A01EB81018A40D8
:1028000002431A623B7D0134A342DEDC02B0BDE824
:10281000F08100BF2DE9F04F97B06846D1F8013044
:1028200006AF1E7D1D7F796006FB05F3D1F80920F8
:102830005C00FA62DA1DD208A0EBC200854604F102
:102840000803DB08DB0006A8ADEB030DF86006A863
:10285000ADEB030D06AAADEB030DFB6ABC60DB68B4
:10286000BA623B620A2322467400A046FF217B61C4
:10287000386116F0EEF806AB7B62B3007B637A69D1
:102880007B681F2AD3F8053040F31981104644466F
:10289000954901FB02F102EB421200EB421202EBFE
:1028A000C23201F1404102F140422031013241F097
:1028B0001F0103F5B46019625A629A623033834291
:1028C000F9D18A480122049089488D21039004237C
:1028D0000020A04602900192059100937C6907F1C7
:1028E0003C0311466420FC63FFF70AFEBC6800212C
:1028F0002246B86A16F0ADF82246FF21786A16F033
:10290000A8F8142344463B6301F0ECFB01F03CFCC7
:102910000421FB6A4FF0000CDB68009196210591C1
:102920007249202204917349722003910121CDE95B
:10293000011C0F21FFF7E4FD45B34FF000093B6A8E
:10294000D7F824A0A3F1040BBB6AA3F10208002E60
:1029500000F0AB80D446DE464346A0445EF8042F28
:1029600033F8020FBCF800108242C8BF90B28A420E
:10297000B8BF91B2434518802CF8021BEED109F183
:1029800001097B6B4D459B44A244E0D13B6B013B6D
:102990003B63B9D1A046002D35D09B46BB6AD7F822
:1029A0000C90023BFB617B6AD7F81480023B3B63CF
:1029B0003B69BD61A3F1020AB6B150460021D7F8C8
:1029C00030C0FD6935F8023F3CF802EF30F8022FC5
:1029D000A3EB0E039A42C8BF09F8018001F101017F
:1029E000C8BF03808E42EDD1FB690BF1010B23447C
:1029F000FB613B6BA24423443B63BB69B1445B4531
:102A0000DAD1A046BD69A9217869FB6A01307861F5
:102A1000DB68059135490422049136490446039147
:102A2000002001210092CDE9011020220F21642015
:102A3000FFF766FD3E2C7FF422AFAC222B4B0092B9
:102A40002D4900226420FFF7A3FD0020CDE90100FD
:102A50000120AD21254B294A00900493FB68642096
:102A60000591039229463246FFF74AFDAF221F4BDC
:102A70000092234900226420FFF78AFD1B4B4FF090
:102A8000B00C049300230224CDE901331D483B69B7
:102A9000324603902946CDF814C000946420FFF715
:102AA0002FFD4437BD46BDE8F08F09F101097B6B6E
:102AB0004D45A0449B44A2447FF449AF66E77A6940
:102AC00044461146084800FB02F002EB421201EBBB
:102AD000421202EBC23203F5B46118625A629A6282
:102AE00030338B42F9D1ECE620841002B09B010018
:102AF000689B0100189B0100749B0100889B0100EA
:102B0000949B0100A49B01002DE9F04FD2F80180B5
:102B1000D2F805C098F81C9098F814A0B9F1000FED
:102B200022D04FF0000E0139BAF1000F17D00C4639
:102B30008678D8F810200EFB06F60AEB020712F88A
:102B400001BB14F8015F0BF00103334403EB4303B3
:102B50000CEB031303EB5B039742DD73EFD10EF134
:102B6000010ECE455144DFD1BDE8F08FF0B5DCE970
:102B7000002087B064460F46FFF7C6FFD4E9022164
:102B8000002040F239360125CDE90100054C064808
:102B90003B46CDE90304059600956420FFF7B0FCA1
:102BA00007B0F0BDB09B0100E09A01002DE9F04FA5
:102BB0008DB082788A4602EB4202120100AFADEB83
:102BC000020D6E46F8610021684615F042FF4FF491
:102BD000B4620021C84815F03CFF9AF81450BE6159
:102BE00035B3DAF810000124054406E05368854245
:102BF00043EA0E0EC2F804E01AD010F8013B03F0CD
:102C0000010C4FEA4C0262441F2B04FA03FE06EB50
:102C10000212EBDD117A203B8C4604FA03F3C1F378
:102C200001010B4363F3010C854282F808C0E4D133
:102C30009AF81C30BB62002B00F08381DAF8182070
:102C4000002411460120FA62194412F8013B00FAEF
:102C500003F3914244EA0304F7D1FB693C6293F821
:102C600002C0BCF1000F00F07D810021BA69C7F8F5
:102C70002CA010460D464FF0010B4FF0190992465B
:102C80003B6AC3F313065FFA86F8C6F3072E360CC9
:102C900001EB41030AEB03135C781A7A6FF3C30468
:102CA0005C709C7A02F0030224F03F049C7293F85B
:102CB0002E401A7224F01F045D7283F82C5083F8A2
:102CC0002D5083F82E4003F1080280F80BB080F8F5
:102CD0002F909379013123F00F0333438C4582F811
:102CE000048082F805E000F130009371D0D14FF0FC
:102CF00040533A6AD7F82CA09A64BB6A002B00F0C4
:102D00002A81DAF81830FB6200234FF0010B7B6256
:102D10009946794BBB624FF0000CFB6A29F0030225
:102D200013F80930BC6A0BFA03F8C8F31308C8F3A8
:102D30000D039B00BB604FEA98337B60131D3A6123
:102D4000FB60C7F81480A6464FEA4C05BB69654492
:102D500003EB051505F13008764628686968AA680E
:102D6000EB68103545450EF1100E0FC6F4D12388DF
:102D7000796A9AF80B2061F309032380002A40F056
:102D8000BD8023687A6962F31F332360FB699AF878
:102D90000C00DB783A6A0BFA03F3013842EA0301CC
:102DA0009AF81C20032800F2C880DFE800F0825B5C
:102DB0003602206894F82E5043EA103025F01F05A3
:102DC000C0F31403013A45EA13454A45A08584F847
:102DD0002E500FDDFA6A4A445078EAB20BFA00F03E
:102DE0000343C3F3140322F01F0242EA1342A385F4
:102DF00084F82E20B9F1000F08D0FA6A4A4412F87C
:102E0000012C0BFA02F21343C3F3140383F4FF13F0
:102E100083F4FF5383F01F032AE0E36A013A4A4533
:102E2000C3F3140311DDFA6A4A44507894F82E2053
:102E30000BFA00F00343C3F3044022F01F020243E5
:102E4000A38584F82E20C3F31403B9F1000F0FD02B
:102E5000FA6A4A4412F8012C0BFA02F21343C3F344
:102E6000140305E0226843EA1233DB43C3F314037F
:102E7000E2681940A07B94F82E30C2F3130222EAD4
:102E80000102A18520F00F0023F01F03C1F30441CC
:102E900040EA12401943A281A07384F82E10303406
:102EA000BCF1000F15D1DAF818304FF0010CFB62BD
:102EB00049E794F82E20C3F31403194022F01F02AF
:102EC00042EA1142A18584F82E203034BCF1000F73
:102ED000E9D07A6A9AF81C302032C2F309027A6289
:102EE000BA6A09F1010960324B45BA6233DDDAF89A
:102EF0001830FB620FE700BF98000460FB6A3A6974
:102F00009918FA689D1811F8013B20680BFA03F331
:102F1000226843EA103363F31F328D422260F2D1FC
:102F20002389BA6803F0030313432381A37A7A68E1
:102F300023F03F031343A37228E7E36AC3F31403A8
:102F400096E7FB6993F802C0BCF1000F07D14FF080
:102F50004053C3F848C03437BD46BDE8F08FBB6A64
:102F60003B6282E64FF040533A6A9A64CCE600BF77
:102F70002DE9F041827800AF02EB42021201ADEB85
:102F8000020D884605460021684615F062FD302294
:102F90000021614815F05DFD6FF01F019DF80130C3
:102FA00098F80C2003F0F40343F00903013A8DF87C
:102FB00000108DF801306C46032A03D8DFE802F0D8
:102FC000948002024FF0FF324FF04051002094F8FD
:102FD0002E3084F82C2043F01F0384F82E3084F820
:102FE0002D20C1F830014FF00132192604F13005CF
:102FF00028462346C4F80F20C4F81320C4F817202D
:10300000C4F81B20E277E27284F82F60D3F800C086
:103010005E689968DA681033AB42C0F800C0466059
:103020008160C26000F11000F0D198F814303BB319
:10303000D8F81000012603EB000C06E05368844525
:1030400043EA0808C2F804801AD010F8013B03F0E4
:10305000010E4FEA4E0272441F2B06FA03F804EBEE
:103060000212EBDD117A203B8E4606FA03F3C1F320
:1030700001010B4363F3010E844582F808E0E4D1BB
:103080002646DFF894E0F44630687168B268F36869
:103090001036AE420EF1100EACE80F00F3D1DFF89F
:1030A00080C06034654630687168B268F368103675
:1030B000A6420CF1100C0FC5F4D1BD46BDE8F0815D
:1030C0004FF0FF324FF04051002094F82E3084F83A
:1030D0002C2023F01F0343F00F0384F82E3084F8D4
:1030E0002D20C1F830017EE701224FF04051E878F1
:1030F00094F82E308240C2F3044523F01F030748A2
:103100002B43C2F3072584F82C2084F82D5084F833
:103110002E30C1F8300166E738060460FFFF0F006B
:1031200068060460F0B50D46A9B04C2200210446A3
:1031300002A815F08EFC00204FF040522978ADF81F
:10314000040082F8A8106978BDF80420A87861F31B
:103150008A12C2F3072160F3C601ADF804208DF88E
:103160000510BDF8041002AB0DF12A025985023397
:103170009342FBD14FF04056002286F8A7202F7DC6
:10318000C7B14FF0010C2969013911F8013F28A896
:1031900018441C2B00F8982C02F1010208DD96F867
:1031A000A7001D3B0CFA03F30343DBB286F8A730FC
:1031B0009742EAD102A915A84C2215F03FFC15A9A7
:1031C0004C22094815F03AFC4C2215A9074815F085
:1031D00035FC29462046FFF7E9FC20462946FFF743
:1031E000C7FE024829B0F0BD4C0004600000046036
:1031F0002DE9F04FD0F80D40D0F80160D4F800C0B0
:10320000D6F820E09CF800309CF8012096F8009059
:10321000D5185FFA85F808F1010B03F1010A0F4692
:10322000591ED0F8090089B08EF829B08EF8228096
:103230008EF824A08EF82510B9F1000F4CD0013281
:103240008EF8272000238EF828301A46636893F8FA
:10325000008008F03F0802F114030EEB4303997855
:10326000013268F30501112A9970F4D119211C4B20
:103270001C4A83F82F1030339342FAD133796BB163
:1032800043685BB1164D9CF80D20314600953846D9
:10329000FFF7DEF923685A781B78D51849F64043C2
:1032A00001356D0093FBF5F540F2E9100122002194
:1032B000042608AB43F8045D0B4C05900B48CDE9A0
:1032C0000121CDE90304114600966420FFF718F9A7
:1032D000034809B0BDE8F08F0A3B8EF82730B1E70C
:1032E0009800046038060460B09B0100289B010030
:1032F0002DE9F047D0F80D80D0F80150D8F8003013
:103300002C6A93F801C01B7895F800E00CEB0302DF
:10331000D2B202F1010A03F101090F46591ED0F899
:10332000096082B084F875A084F86E2084F87090EB
:1033300084F87110BEF1000F3BD00CF1010C84F841
:1033400073C000231A4684F87430D8F804C09CF87F
:10335000020000F03F0002F1140304EB430393F872
:103360004E10013260F30501112A83F84E10F2D19C
:103370009CF80010114AC901301D07F0FDFCD8F877
:1033800004300F4A197806F10800C90107F0F4FC6F
:103390002B7953B1736943B1D8F80020094C527BA3
:1033A000294638460094FFF7C5F9064802B0BDE843
:1033B000F0870A3B84F87330C3E700BFFC9A010032
:1033C000149B010038060460F0B500264FF040530E
:1033D00001250424D0F80D20D0F80110506812689F
:1033E000467090784FF00F0E83F82C01D0784FF490
:1033F000B47C83F82D01107A83F82A01907A83F83F
:103400002B01107983F82E01507983F82F010F7862
:10341000C87883F825714F7983F88E7083F884001B
:1034200083F8815083F8806083F8AE4083F8AF4022
:103430000E7993F8890086EA050767F305100227DD
:1034400083F8890093F8A10066F3041083F8A100C3
:1034500083F88D4083F8B05083F8C5E0A3F8C8C066
:1034600083F8CC70947B087A83F800418C7983F8D8
:103470000541CC7983F80A4183F80D01497A83F834
:103480001011117B83F8DA10D27A83F8A020BDE8FE
:10349000F04000F095BB00BF4FF0405310B5D0F89E
:1034A0000D10D0F809204C68526893F841116078EB
:1034B000054B02EBC01003EB0141802215F0BEFA70
:1034C00063780133637010BD8007016070B5194BDC
:1034D00084B01B78044613B106F01CF8C37ED4F800
:1034E0000130DB7A23B3D4F80930DE6806F18005B9
:1034F00006F50866A5F1800000231946DA01825816
:103500004DF823200133042B1144F7D100225DF83C
:103510002230D401A1EB430301325B10042A035192
:10352000F5D10430A842E7D105F50075B542E1D1E7
:1035300004B070BD971700204FF040532DE9F041C3
:10354000012604240025D0F80D20D0F801101268BF
:103550004FF00F0890784FF0030E83F8E000D0781A
:1035600083F8E100107983F8E200507983F8E300F2
:10357000107A83F8E600907A83F8E7004F79C878EC
:1035800083F88E7083F8840083F8816083F880501C
:1035900083F8AE4083F8AF400F7993F8890087EA4B
:1035A000060C6CF305104FF01E0C83F8890093F89D
:1035B000A10067F3041083F8A10083F88D4083F81D
:1035C000B06083F8C58083F887E0A3F8C85083F81B
:1035D000CCC0907B83F80001887983F80501C87915
:1035E00083F80A01497A83F81011117B83F8DA1005
:1035F000D27A83F8A020BDE8F04100F0E1BA00BF24
:103600004FF040532DE9F04101260025D0F80D1070
:10361000D0F80100D1E900219478497883F8E0409E
:10362000D4784FF0040883F8E14014794FF00F0E7E
:1036300083F8E2405479B14083F8E340147A31448E
:1036400083F8E640947AC9B283F8E7404779C478B2
:1036500083F88E7083F8844083F8816083F880500B
:10366000077993F8894087EA060C6CF305144FF04C
:10367000030C83F8894093F8A14067F3041483F89E
:10368000A14083F88D8083F8B06083F8C5E083F8AB
:1036900087C0A3F8C85083F8CC10917B83F8001141
:1036A000817983F80511C17983F80A11417A83F889
:1036B0001011117B83F8DA10D27A83F8A020BDE8CC
:1036C000F08100BF2DE9F04F99B0734C06AF07F1C0
:1036D000240A7861714D0E4694E80F008AE80F00C5
:1036E00007F1700307F134087B6407F110035046BB
:1036F0004146CAF80830CAF80C50FCF7C1FD94E8FE
:103700000F00674C88E80F0007F11003404607F1EF
:103710004401C8E90234FCF7B3FD012000F06CFC61
:103720003861002800F0B3800023E9461A46D0F83B
:1037300001505C48297D2C7FB961FC6101FB04FBD1
:103740006978B96029792B71F96002F1140300EBF3
:1037500043035988013241F4F861112A5980F4D1A8
:1037600069460BF10703DB08A1EBC3039D46D6F8BE
:103770000D20D6F809C0136806AC5B78DCF8081099
:1037800020465A467B60C7F820C015F057F97B6881
:10379000BBF1000F09D0224604EB0B0012F8011B0D
:1037A0000431824202F8011CF8D148F001024AF0CB
:1037B0000101CDE90021012019465A46234602F0B5
:1037C000E1FE3B6A5A461868214615F037F940F287
:1037D00041304FF0000B4FF0010C3B6ABA691B6897
:1037E000F969DFF8CC8005902F48CDE901BBCDE920
:1037F0000308CDF800C06420FEF782FED7F81CA0B5
:10380000DA4518DD5846D7F818C0D7F820E0BCF1E3
:10381000000F0DDD00222B7DDEF81C1000FB0323C2
:10382000895C14F803B0013259446245E154F2D185
:1038300001305045EBD1324621467869FFF764F9F3
:10384000D7E9062140F24B3000250126CDE904805E
:10385000164823460390CDE9015564200096FEF7F3
:103860004FFE2A46BB680F4C03F01F0002F1140301
:1038700004EB43035988013260F38A11112A5980FD
:10388000F4D13B693A7BD3F801301A71CD464C37FD
:10389000BD46BDE8F08F00BF288C0100092600005E
:1038A0006D2B000000000460EC9A0100E09A01001A
:1038B000B09B01002DE9F04FADF50D7D06AF7860AE
:1038C0008A4600F065FA061E40F3C580002403E036
:1038D0000134A64200F0BF802146012000F066FAC4
:1038E0000028F5D007F1140E0546F446D0F8014043
:1038F00004F12008664620686168A268E368103415
:1039000044450CF1100C0FC6F4D1002620684FF48A
:10391000F072CCF800008EF80460C5F801E0DAF827
:103920000D3001211B6807F138005B781C46FB60F5
:1039300015F08FF8ADF5F16D06AB184631464FF432
:10394000F06215F086F8012C40F389800124A1462D
:10395000031FDFF82081BB60DAF8055005F10F0B7B
:1039600005F2AF555846112221460BF1300B15F0E8
:1039700070F8AB45F6D1012240F27A33042539497B
:103980006420CDE902610593114607F11003CDF8DB
:103990001080CDF8049000953C61FEF7B1FD00F079
:1039A000A1FB00F0F1FB40F27E332F4A0593CDE9F5
:1039B00002624FF0C04320220F210095CDF8108005
:1039C000CDF804907220FEF79BFD4FF0C043B9681C
:1039D000DFF8A4C007F13802186851F8045F043317
:1039E0008542BCBF14700860634502F10102F3D147
:1039F0004FF463731D4A0593CDE9026207F1380362
:103A0000CDF81080CDE9009620220F216420FEF72A
:103A100077FDFB680134A3429ED15246786807F1D6
:103A20003801FFF771F84FF4647400220120104947
:103A300007F13803CDE9012200900391CDF8108001
:103A4000059420220F216420FEF75AFD07F5077721
:103A5000BD46BDE8F08F0023D3F80130FFDEDFF86C
:103A60001480DAE7389B0100489B0100E09A0100CE
:103A7000509B0100B09B01008007006008B500F07A
:103A800083FB022000F0B8FAD0F80930986808BD2E
:103A900008B500F079FB012000F0AEFAD0F809304B
:103AA000D86808BD30B4D0F80D20D0F8093052687D
:103AB00015789DB19C685B68803C03F17C00E41A3A
:103AC00000EBC515A0F18003221853F8041F8342B0
:103AD00042F8041FF9D18030A842F3D130BC7047BE
:103AE000704700BF002070474FF0405393F84121CA
:103AF000002082F0010283F8412193F8432182F0F3
:103B0000010283F8432170472DE9F047482286B02F
:103B1000FF212A4814F09DFF01A80AF06DFA8046A3
:103B200002A80AF06FFA074603A80AF071FA18F023
:103B3000FF081DD04FF0000A4FF001091F4E04ADE1
:103B4000019B082213F80A402846610004F0030490
:103B500014F050FF04EBC404049A3444059BA15CA8
:103B600009FA03F30AF1010A0B43C245A354E7D152
:103B700017F0FF071FD04FF000094FF001080F4E5C
:103B800004AD039B082213F809402846610004F0A5
:103B90000304043404EBC404344414F02BFFDDE9C3
:103BA0000423A15C013308FA03F309F101090B4373
:103BB000B945A354E5D106B0BDE8F087642E0020D6
:103BC00008B50AF0F7FC054B1B78984204D018465C
:103BD000BDE808400AF0D0BC08BD00BF8407002043
:103BE00010B50AF0E7FC04460AF0D8FC844203D082
:103BF000BDE810400AF0C0BC10BD00BF30B50138B0
:103C000085B00C460A2810D8DFE800F03B3E0F3B99
:103C100026110F0F2611060003A80AF0EDF922461F
:103C2000C1B2039801F07AFDA06305B030BD03A8CE
:103C30000AF0E8F90223C5B203992A460093204608
:103C400004F1150300F092FC22462946039801F086
:103C500079FBA06305B030BD03A80AF0CDF90223BB
:103C6000C5B203992A460093204604F1150300F0DB
:103C70007DFC22462946039801F022F8A06305B096
:103C800030BDCB7A002BD0D010462146FFF74AFA40
:103C9000206205B030BD00BF0138092808D8DFE830
:103CA00000F00808080705050505050500238B63D6
:103CB000704700230B627047037810B5022B04464F
:103CC0000BD0042B03D10022D0F801301A6200235C
:103CD0006374A374E374237510BDD0F80900084918
:103CE000043007F0D5F8D4F809000649083007F089
:103CF000CFF800236374A374E374237510BD00BF71
:103D0000C89B0100E89B0100002230B504460D4627
:103D100083B002AB43F8042D18460E4A152107F074
:103D20002BF822780C4B294653F82230204698472E
:103D3000C4F80500A06822686568E168019B986086
:103D40001A605D60D960226901981A61227D1A7536
:103D500003B030BDC09B0100249C01000B4B1A68CE
:103D60000AB90CE01A46D2F81130002BFAD1002320
:103D7000C2F8110043748374C374037570471860EC
:103D8000002343748374C374037570476C1600205A
:103D9000054B1B6833B10020D3F811300130002BE4
:103DA000FAD17047184670476C16002070B5164B54
:103DB00088B01B687BB1002402E0D3F8113053B106
:103DC0001A788242F9D101340029F6D0A142F4D107
:103DD000184608B070BD4FF4E1700122002404269B
:103DE00008AB43F8041D094D05900948CDE90124AD
:103DF000CDE90305114600966420FEF781FB2346BA
:103E0000184608B070BD00BF6C1600200C9C010065
:103E1000149C010070B5094E82B034684CB1084D55
:103E20000194D4F81140294601A807F031F8002C7C
:103E3000F6D10023C6E9003302B070BD6C16002035
:103E4000049C0100F8B5446805460AF0D1F8ACB10D
:103E500023780B2B12D80B4E0146074656F8333009
:103E600020469847D4F8110040B10378394606EB54
:103E7000C3066860736898470120F8BD0020686039
:103E8000F8BD00BF8807002010B504460AF0B0F85E
:103E9000636843B11C78054A014652F8342018463D
:103EA0009047012010BD184610BD00BF88070020B4
:103EB00038B5446805460AF09BF84CB12278054BAA
:103EC000014653F832302046984700236B6038BDD6
:103ED0006C6038BD8807002070B582B005460C467E
:103EE0000AF086F84FF0405393F84121014682F0E2
:103EF000010283F8412193F8432182F0010283F803
:103F00004321286818B90CE0D0F8110058B10278A4
:103F1000A242F9D10A4A686002EBC402536898478A
:103F2000012002B070BD4FF40B76064D064C009692
:103F30002B46002221466420FEF72AFBF7E700BF4C
:103F4000880700200C9C0100549C010038B50468CF
:103F500005460AF04DF86CB16B685BB92178064BE9
:103F60002A6803EBC1035B6801466A6020469847F4
:103F7000012038BD002038BD8807002008B54FF06B
:103F8000405393F8243093B172B60A48FFF7DEFF2E
:103F900058B10123084A1375BFF34F8F4FF04052B9
:103FA0000020064908721370937062B608BD0AF0CB
:103FB000D1FBE9E76C1600200000105020270020FC
:103FC00008B572B60948FFF7C1FF60B10422084B7B
:103FD0001A75BFF34F8F4FF040530122002005495F
:103FE00008721A709A7062B608BD00BF6C16002085
:103FF0000000105020270020054B1B6833B11A78B1
:10400000824203D0D3F81130002BF8D11846704704
:104010006C160020044B11B143F820107047034A7E
:1040200043F82020704700BF54070020E13A000009
:104030000B4B70B51C6809F0DBFF7CB10546094EDF
:1040400023782046294656F823309847D4F8114063
:10405000002CF5D1BDE87040FFF7C2BD70BD00BFB8
:104060006C1600205407002008B50E4B5A6802B1A8
:1040700008BD01461846FFF72FFF0028F8D00A4B6D
:104080001B680BB10AF066FB0123084A1375BFF3E6
:104090004F8F4FF040520020054908721370937003
:1040A00008BD00BF6C1600204427002000001050FF
:1040B0002027002038B50023064D074C074A084941
:1040C0002B72236011600AF0B7FDBDE83840FFF79E
:1040D00055BF00BF202700209C1700209817002004
:1040E0007D3F0000002330B401240649064D0748F7
:1040F000074A0B7207492B60047030BC1160FFF750
:104100003DBF00BF202700209C17002097170020EC
:10411000981700207D3F0000002330B40124064999
:10412000064D0748074A0B7207492B60047030BCE4
:104130001160FFF745BF00BF202700209C1700201B
:104140009717002098170020C13F000008B50AF01B
:1041500087FD00230249034A0B60136008BD00BFBE
:10416000981700209C170020024B5868003018BF99
:10417000012070476C160020024B1868B0FA80F0DE
:10418000400970476C16002008B5074908200AF05E
:1041900041F9FFF74DFF0AF063FD00230349044A8C
:1041A0000B60136008BD00BFE93A000098170020BB
:1041B0009C17002008B572B60AF052FD002308498A
:1041C000084A0B60136062B6074A516831B1536008
:1041D00006490820BDE808400AF01CB908BD00BF28
:1041E000981700209C1700206C160020E93A000068
:1041F00008B5044908200AF00DF9BDE80840FFF7AA
:1042000017BF00BFE93A000008B50449082014F0C0
:1042100007FDBDE80840FFF70BBF00BFE93A00000B
:1042200008222F4838B52F4C436822602E4ACBB164
:10423000002519781570022937D0D3F8113093B1C1
:104240002748FFF7FFFD002846D00123274A1375B2
:10425000BFF34F8F4FF04052002025490872137072
:1042600093700DE0137001250021224B20481F4A56
:104270001B680572117503B198471948FFF718FEBE
:1042800010221D4B2260D3F80021120708D500220E
:1042900008241A481A49C3F880410270C1F8402125
:1042A0004FF0405300225A7038BDD3F80D205168AA
:1042B0000A784978013A9142BFDAFFF7E5FD58B133
:1042C00001230A4A1375BFF34F8F4FF0405208493C
:1042D0000D7213709370D3E70122054B1A72CFE76A
:1042E0006C160020A40C002096170020000010502F
:1042F000202700204027002000E100E0A00C002043
:1043000000000250B8B4850005F10A0323F007034A
:10431000002800AFADEB030D11DD6B46043A1544E8
:104320000239181F31F8024F52F8043F03FB04F31F
:10433000AA424FEA132440F8043F1460F2D1BD466C
:10434000B8BC70472DE9F043089D1DB34FF04C0CED
:1043500001264FF00009079CD2B20CFB054CC9B2F4
:104360009719C0B20F44A1F10A08A1F1030EFFB2E0
:1043700080448644002B14BF45467546A0702671C4
:10438000E7706171A27184F81990A676E5714C34DA
:104390006445EFD1BDE8F083F0B5012A83B016463D
:1043A00005460C461F462DDC0146684614F022FBEC
:1043B00036B3009B3F2B1D46A8BF3F25019A002B1B
:1043C000134405F03F05B8BF00253F2B1A46A8BF90
:1043D0003F22002B4FF0000102F03F03B8BF002343
:1043E00004F1100207EB420C09B30A19103207EB73
:1043F0004202907965F3050090710131B142F3DB1F
:1044000003B0F0BD104606F081FC044106FB04F445
:104410000F2C294606DD0122684614F0EBFA01262E
:10442000009BC7E73246684614F0E4FAC1E79CF8FF
:10443000062063F305028CF80620DEE7F0B5012ABA
:1044400083B0154604460E461F462DDC01466846DD
:1044500014F0D0FA009B2DB33F2B1C46A8BF3F247D
:10446000019A002B134404F03F04B8BF00243F2BF3
:104470001A46A8BF3F22002B4FF0000102F03F0375
:10448000B8BF002306F1100207EB420CF1B18A1904
:10449000103207EB4202907964F30500907101310C
:1044A0008D42F3D103B0F0BD104606F02FFCF307A8
:1044B00044BF06416E4321462A46684654BF06F172
:1044C000FF36013614F096FA009BC5E79CF80620EB
:1044D00063F305028CF80620E1E700BF70B5DCF855
:1044E0000C3086B0644600259847FFF74DFED4E9AE
:1044F00001230121042040F253261B690295CDE9D6
:104500000001064D06480596CDE903057220FDF72A
:10451000F7FFA368186906B070BD00BFA09C01003A
:10452000AC9C010070B5644686B0DCF80830984752
:10453000FFF72AFE002201214FF4757604256368F7
:1045400008481B690292084A0596CDE90320CDE987
:10455000005114227220FDF7D3FF6368186906B07A
:1045600070BD00BFA09C0100AC9C01002DE9F04F84
:1045700087B006AF4578D7F82890D01D20F0070007
:1045800009FB05F5ADEB000D0DF1180A0E4650467E
:10459000002190461C4614F05CFAA94541DB4FF01F
:1045A000000B08F1FF3922224FF0FF31204614F0B2
:1045B00050FA33784FFA8BF0B8F1010FE0542DDD4B
:1045C0004FF0000E6FEA060C711C11F8012BA35678
:1045D000B3F1FF3F05D1431CAB42ACBF00235BB23C
:1045E000A35498421AD092FBF5F005FB1020012845
:1045F00014BF01204FF0FF30204482569A420DD064
:104600000CEB01029145A1EB060200F0958090456C
:1046100001DD1846D9E7BEF1000F4CD1BBF1000F08
:1046200046D09323DFF828B1009300225B4645492A
:104630006420FDF7ADFFB8F1000F6CDD013EB1461F
:1046400006EB080119F8013F93FBF5F205FB123266
:104650004945E254F6D10121992000223A4BCDE997
:1046600004B0CDE901120393009123464246642031
:10467000FDF746FF0AF1FF3316F8012FA256B145A8
:1046800003F8012FF8D1012100249D252F48CDF8F2
:1046900010B003905346642042460595CDE90114BD
:1046A0000091FDF72DFF20460437BD46BDE8F08F91
:1046B0004FF0010B77E7012189200022224BDFF820
:1046C00090B0CDE9011205900091CDE9033B42463F
:1046D00023466420013EFDF713FF06EB08010AF1B3
:1046E000FF3316F8012FA256B14203F8012FF8D17B
:1046F000012400218D251548CDE901410390CDF815
:1047000010B0642053464246059500942146FDF7BB
:10471000F7FE2046C8E70121992500200A4ACDE985
:1047200001100392CDF810B0234605950091424642
:104730006420FDF7E5FEA6E79045BCDD4FF0010ED5
:10474000184642E7CC9C0100F09C0100BC9C010093
:10475000A09C01002DE9F843D2F801600746727869
:104760000D46012A984618D9002814DD00244FF080
:104770004C094D1E00E07278510094FBF1F301FBEF
:10478000134315F8010F611009FB03830134FFF790
:1047900003FEA742EFD1BDE8F8830028FBDD00242B
:1047A0004FF04C09331993F915306110002B05DBDC
:1047B00009FB03837278285DFFF7EEFD0134A74201
:1047C000F0D1BDE8F88300BF70B5644686B0DCF870
:1047D00000200B4BFFF7BEFFD4E9012301214FF46A
:1047E00017760020074D084C1B68CDE9010005969F
:1047F0000091CDE903457220FDF782FE06B070BD41
:1048000014080460A09C01008C9C01002DE9F84371
:10481000D2F801501E466A78012A1ED900281ADDF6
:1048200001F1FF3821244FF04C0908EB000700E0AC
:104830006A78510094FBF1F301FB134318F8010F60
:1048400004EBD47109FB03634910FFF7F7FD4745FB
:1048500004F1FF34ECD1BDE8F8830028FBDD0C4601
:104860004FF04C0905F1140808EB000718F9013F57
:10487000C8F13601294401EBD171002B4FEA6101E7
:1048800005DB09FB03636A782078FFF7D7FDB8459D
:1048900004F10104EAD1BDE8F88300BF30B56446F5
:1048A00087B0DCF800200B4BFFF7B0FF40F2DD359E
:1048B0000121002263680848084C1B68CDE90122E9
:1048C000CDE903040595009114227220FDF718FE2E
:1048D00007B030BD980604608C9C0100A09C0100CC
:1048E000F0B4147980F8E8405579049C80F8E950D8
:1048F000957980F8EA50D57980F8EB50957A80F870
:10490000EE50157B80F8EF508D790E7880F88E5040
:1049100090F8895045F0300580F8895090F8A15002
:104920006FF3041580F8A150CD7880F8A950002EBF
:1049300051D180F8986090F88B5045F0010580F8CF
:104940008B500125072700264FF0060C80F88D704C
:1049500080F8B05080F8C56080F8815080F88050B1
:1049600080F8AEC080F8AF700D79002C80F88450CC
:10497000557CB8BF033480F89F50957CC4F38F04F6
:10498000DBB280F89E5080F89C60A0F8CA4080F8A6
:10499000CD30D37C80F80031CB7980F805310B7AAB
:1049A00080F80A314B7A80F81031137D80F8DA30C4
:1049B00090F8A330917D61F3061380F8A33090F84E
:1049C000A330D17D61F3020380F8A330537DF0BCA6
:1049D00080F8A0307047012580F8985090F88B50EF
:1049E0006FF3000580F88B50ABE700BF2DE9F0476F
:1049F000D0F80160D0F80930747882B06400D0F843
:104A00000D5033B10F46024619687878274BFFF7EF
:104A1000A1FEB76B95F80DC08CB34FF04C0938462A
:104A20004FF0000809FB04790CF01F0C0CF0030E8A
:104A30004FEA8E1E4FEA9C0C002101F1100300EB9F
:104A4000430393F806A0DA790AF03F0A22F007023E
:104A500001314AEA0E0A42EA0C02112983F806A043
:104A6000DA71EAD190F84A3080F8488023F01F03C9
:104A700080F8498080F84A304C308145DCD1337869
:104A80002A78A9786878CDE90074FFF75BFC40F6D6
:104A90001400234600902A4631464FF04050FFF75D
:104AA0001FFF02B0BDE8F047FFF79AB81408046092
:104AB00049F64043014411440331490093FBF1F1AD
:104AC00040F2A51070B501220026042588B008AB7D
:104AD00043F8041D064C05900648CDE90126CDE9B2
:104AE0000304114600956420FDF70AFD08B070BD6F
:104AF000A09C01007C9C01002DE9F04FD0F8013012
:104B0000D0F80D605C785A798BB0650096F8038018
:104B1000002A46D0D0F809209269002A41D0197D98
:104B200096F810B0DB68F1B14FF04C0E9446614A34
:104B30000CEB010A0EFB052E03F1FF3919F8013FBA
:104B40005B0865B110335B4A58001118CB799CF8AB
:104B500000704C3267F3C7037245CB71F5D10CF18D
:104B6000010CD445EAD1002D00F09E804C22514921
:104B70000B4602FB051283F825B04C339342FAD161
:104B800001AF38462422002113F063FFB8F1020F71
:104B900021D0B8F1040F45D0B8F1010F52D0002157
:104BA0002AE001AF38462422002113F052FFB8F169
:104BB000020F10D0B8F1040F34D0B8F1010F41D07A
:104BC000002DECD170783278B178FFF771FF394859
:104BD0000BB0BDE8F08F002DF4D03B46552105EB1E
:104BE000C500384403F1090203F8011B9A42FBD1C6
:104BF0009842F7D19DF804104FF0000C2D4C384628
:104C0000002301E010F8011FE2180133092B117293
:104C1000F8D10CF1010C654504F14C04D2DD17F814
:104C2000091FECE7002DCDD03B46AA2105EBC500BE
:104C3000384403F1090203F8011B9A42FBD1834275
:104C4000F7D1D7E7002DBDD0B9464FF0000EDFF801
:104C500068804946DFF864C0002311E0012C05D1CB
:104C6000032B03F0010201DC724506D003EBC30203
:104C700008781CF8022002430A700133082B06D082
:104C8000022CEBD19E45F1D10133082BF8D10CF168
:104C9000010CE04501F10101DED10EF1010E754577
:104CA00009F10909D5D1A5E72946242201A813F065
:104CB000D0FE87E7140804606D2E0020642E0020CB
:104CC0002DE9F04F83B04C230C4692F8018000AFE1
:104CD0004FEA480603FB06F3ADEB030D00219146B6
:104CE00005461A4668467B609A4613F0B2FE69464E
:104CF0005FFA84FC002E53D06B461A240DEB0A0099
:104D00005A781C7002F0EC0242F002025A704C33E6
:104D10009842F5D1BCF1000F28D000204FF04C0B89
:104D20004FF0010E013D05E053690130234360451A
:104D300053611ADA15F8013F09EB030292F91520C5
:104D40001F2B0EFA03F40BFB0212EDDD147E203B49
:104D5000A2460EFA03F3C4F301041C43013064F3CA
:104D6000010A604582F818A0E4DB86B100234C25D7
:104D70005524B8F1020F07D105FB0312D07C5474FF
:104D800020F001009474D07401339E42F1DC7A6803
:104D9000054813F053FE04480C37BD46BDE8F08FBC
:104DA000BCF1000FF3D0B8E714080460F0B5D0F8F8
:104DB0000130D0F809701E7D87B0FD69BB6806B36D
:104DC00000224FF4807C14E0786835F8124050F8E7
:104DD00022002402012838BF0120B4FBF0F0B0F516
:104DE000DC7F28BF4FF4DC7023F812000132B2429E
:104DF00007D028880028E7D123F812C00132B24238
:104E0000F7D140F20726002002254A78064C0749D0
:104E1000CDE90100CDE90314059600950121642038
:104E2000FDF76EFB07B0F0BDA09C0100609C010087
:104E30002DE9F04F97B0814606AFDFF8D8C16E4E2E
:104E400007F11C0807F12C0407F10C05F960BA61A1
:104E500096E80F0088E80F00C8E9025C404621464A
:104E600007F16803FB63FBF70BFA96E80F00634E4C
:104E700084E80F00C4E90256204607F13C01FBF725
:104E8000FFF9FB6899F80120D3F80160D3F80D50C1
:104E90007078D3F809A08001C7E9042A44F001041E
:104EA00005F034FFE98948F00105DAF800303A6985
:104EB000CDE9004501F022FCDAE900013D69EB464D
:104EC000EA1DAB0022F007020A33ADEB020D23F01E
:104ED00007037A690DF11808002DADEB030D796019
:104EE000F368146906AED7F80CA014DD002205F1B2
:104EF000FF3C9C44013B13F8011F18B110F801E07E
:104F000008F802E01CB154F8211046F8221063455D
:104F100002F10102EFD1F0B140F22122059200220C
:104F2000CDE901220122364B11460092354A642018
:104F3000CDE9033243462A46FDF7E2FADAF80130BA
:104F4000DAF80D10DA789AF800300132092B497B33
:104F50001ED0052B3ED094B10024042001214FF433
:104F6000107C0294CDE90001264C27483346CDE958
:104F700003042A46CDF814C06420FDF7C1FA49465F
:104F8000F868DD46FFF712FF4437BD46BDE8F08FF5
:104F90007B6840F64A30CDE903630091CDE90158C2
:104FA0004FF4F0734FF4487101F070FC4FF40C7C37
:104FB0000420164A1349002304910121CDE901136D
:104FC0007B6800900392CDF814C02A466420FDF758
:104FD00097FAC0E77B6840F64A30CDE90363009159
:104FE000CDE9015882234FF4487101F04FFC4FF492
:104FF0000F7C0420064ADDE7388C0100C947000019
:10500000049D0100A09C0100189D01000C9D010061
:1050100060A60100DD440000F8B59B0003F10A041E
:1050200024F0070400AF002AADEB040DEC460CDDC4
:10503000BC69ACF10405013C224414F8016F51F83D
:105040002660944245F8046FF7D11A46614613F082
:10505000F5FCBD46F8BD00BF10B5D0F80140D0F852
:1050600009204B781169227DE46882B008460094DB
:10507000FFF7D2FF02B010BD70B5D0F80150D0F8E4
:105080000940EE6882B04B782A7DD4E9031000967F
:10509000FFF7C2FF287D2269A16802B0BDE8704019
:1050A000FFF730B9D0F809304A7818699200D9680A
:1050B00013F0C4BC2DE9F047D0F80160D0F80930F6
:1050C000747882B06400D0F80D5033B10F460246B8
:1050D00019683878274BFFF799FBB76B95F80DC027
:1050E0008CB34FF04C0938464FF0000809FB0479A7
:1050F0000CF01F0C0CF0030E4FEA8E1E4FEA9C0CB6
:10510000002101F1100300EB430393F806A0DA79C4
:105110000AF03F0A22F0070201314AEA0E0A42EA87
:105120000C02112983F806A0DA71EAD190F84A300E
:1051300080F8488023F01F0380F8498080F84A30C7
:105140004C308145DCD133782A78A9786878CDE96C
:105150000074FFF7F7F84FF4D360234600902A4617
:1051600031464FF04050FFF7BBFB02B0BDE8F047BF
:10517000FEF736BD980604602DE9F04FD0F80130F7
:10518000D0F80D605C785A798BB0650096F8038092
:10519000002A44D0D0F80920906900283FD01A7D19
:1051A000D96896F810E0E2B14FF04C0ADFF8889128
:1051B00001EB020C013811F8013B10F8017FC3F13B
:1051C000210393FBF5F205FB12320AFB029223F056
:1051D000010320331344DA79614567F3C702DA71BA
:1051E000E9D1002D00F0A1804C2253490B4602FB6F
:1051F000051283F825E04C339342FAD101AF3846CB
:105200002422002113F025FCB8F1020F21D0B8F1BF
:10521000040F45D0B8F1010F52D000212AE001AFB0
:1052200038462422002113F014FCB8F1020F10D0EC
:10523000B8F1040F34D0B8F1010F41D0002DECD1FA
:1052400070783278B178FFF733FC3B480BB0BDE89B
:10525000F08F002DF4D03B46552105EBC5003844B6
:1052600003F1090203F8011B9A42FBD19842F7D1DE
:105270009DF804104FF0000C2F4C3846002301E03D
:1052800010F8011FE2180133092B1172F8D10CF14B
:10529000010C654504F14C04D2DD17F8091FECE759
:1052A000002DCDD03B46AA2105EBC500384403F1C3
:1052B000090203F8011B9342FBD18342F7D1D7E7E0
:1052C000002DBDD0B9464FF0040CDFF8748005F115
:1052D000040A49461948ACF1040E002312E0012CDF
:1052E00005D1032B03F0010201DD964507D003EB46
:1052F000C30291F800B0825C42EA0B020A700133EB
:10530000082B06D0022CEAD19C45F0D10133082BA2
:10531000F8D10130804501F10101DED10CF1010C21
:10532000E24509F10909D4D1A2E72946242201A8BE
:1053300013F08FFB84E700BF98060460642E002002
:105340006D2E00202DE9F04F83B04C23567800AF2E
:10535000750003FB05F3ADEB030D904683468946CC
:105360001A46684600217B609A466C4613F071FB32
:10537000002D5BD06B4600200DEB0A015A781870A7
:1053800002F0EC0242F012025A704C339942F5D10D
:10539000B9F1000F2EDD00214FF04C0A4FF0010E45
:1053A0000BF1FF3C07E05369013143EA0B0B8945E0
:1053B000C2F814B01DDD1CF8013F08EB0302C3F175
:1053C000210092F915201F280EFA00FB0AFB024269
:1053D000E9DD107EC3F1010383460EFA03F3C0F347
:1053E00001001843013160F3010B894582F818B0C0
:1053F000E1DC8DB100234FF04C0C6FF05500022E14
:1054000007D10CFB0342D17C507421F00101907450
:10541000D17401339D42F2DC7A682146054813F0CD
:105420000DFB04480C37BD46BDE8F08FB9F1000F05
:10543000F2DDB0E79806046070B5D0F8092086B0B8
:10544000D4699368218851B356689D1E301F383641
:1054500001E034F8021F50F8042F0902012A38BF76
:105460000122B1FBF2F2B2F5DC7F28BF4FF4DC720F
:10547000864225F8022FECD140F2C23500220224E8
:105480000C480D49CDE90122CDE9031005950094A2
:10549000142201216420FDF733F806B070BD4FF4EB
:1054A00080709A1E03F11C0122F8020F8A42FBD180
:1054B000E2E700BFA09C0100609C01002DE9F04FD5
:1054C00095B06F4E06AF07F11405DFF8D0C1B96093
:1054D0003A6196E80F0085E80F0007F1600307F1D5
:1054E00024047B6307F10803C5F80CC02846214655
:1054F000AB60FAF7C5FE96E80F00624E84E80F0035
:1055000007F10803C4E90236204607F13401FAF72F
:10551000B7FEBB6844F00104D3F80160D3F80990EA
:105520007078C7F80C90D3F80D8045F00105800124
:1055300005F0ECFBB8F80E10D9F800301422CDE9D4
:10554000004501F0DBF8357DEA46EA1DAB0002F4C8
:10555000FC720A33ADEB020D03F4FF63F9680DF141
:105560001808ADEB030DF268D9E9000306AE7B60C5
:105570000C69D7F8089085B10023013A12F8011F91
:1055800018B110F801C008F803C01CB154F821107C
:1055900046F8231001339D42F0D100B340F28E3221
:1055A000059200224FF0010B374BCDE90122374A1B
:1055B0005946CDE90332CDF800B043462A4664206F
:1055C000FCF79EFFD9F80130D9F80D10DA7899F878
:1055D00000305A440A2B497B1DD0062B3DD094B194
:1055E00040F2AE34002001214FF0040C05940290EB
:1055F000264C27483346CDE903042A46CDE900C1AD
:105600006420FCF77DFFD546B868FFF715FF3C37EF
:10561000BD46BDE8F08F7B6840F64A30CDE90363B4
:105620000091CDE901584FF4F0734FF4487101F047
:105630002DF940F29E3C0420164A144904910021A1
:10564000CDE901B159467B6800900392CDF814C0B2
:105650002A466420FCF754FFC1E77B6840F64A30D5
:10566000CDE903630091CDE9015882234FF44871DD
:1056700001F00CF940F2AA3C0420074ADDE700BF24
:10568000388C01009D480000249D0100A09C010071
:10569000389D01002C9D010090A6010025450000C9
:1056A00010B5D0F80140D0F809200B781169227D9F
:1056B000E46882B008460094FFF7AEFC02B010BD6B
:1056C00070B5D0F80150D0F80940EE6882B00B7880
:1056D0002A7DD4E903100096FFF79EFC287D2269FD
:1056E000A16802B0BDE87040FEF70CBE4FF0405319
:1056F00093F84111D0F80930090401F1C041D8688C
:1057000001F58431502213F099B900BFD0F8093067
:105710000A7818699200D96813F090B92DE9F0471A
:105720004C2692F8018000AF4FEA480406FB04F6CD
:10573000ADEB060D824689466846324600216D462D
:1057400013F087F9002C5ED06B461A200DEB060192
:105750005A78187002F0EC0242F002025A704C3390
:105760009942F5D119F0FF012AD00AF1FF304FF02C
:105770004C094FF0010E014405E05369814243EAB0
:105780000C0353611BD010F8013F93FBF4F204FBB0
:1057900012321F2B0EFA03FC09FB0252EDDD92F8C8
:1057A00018C0203BE2460EFA03F3CCF3010C43EAA7
:1057B0000C0363F3010A814282F818A0E3D1F4B12B
:1057C0002B4655212E44B8F1020F05D1DA7C5974CD
:1057D00022F001029974DA744C339E42F3D1002610
:1057E0004FF04C080A4B08FB065118464C2213F0A8
:1057F00025F903460136B44203F15403F3D10448BA
:10580000BD46BDE8F08719F0FF01AED1F7E700BF54
:105810004409046008B50520FEF7EEFB10B1D0F88E
:105820000930186908BD00BF08B5FEF7ADFC0520BA
:10583000FEF7E2FB10B1D0F80930186908BD00BFCF
:1058400008B5FEF7A1FC0920FEF7D6FB10B1D0F891
:105850000930186908BD00BF4FF0405393F841313B
:105860004A78D0F8090003491B049200C068194423
:1058700013F0E4B86808016008B50620FEF7BCFB29
:1058800010B1D0F80930186908BD00BF08B5FEF79F
:105890007BFC0620FEF7B0FB10B1D0F80930186988
:1058A00008BD00BF8200014813F0C8B8A01700204F
:1058B000F0B4D0F809300B4E1C6906F130073546BC
:1058C0000FCDBD4220606160A260E36006F110066A
:1058D00004F11004F3D107CE20606160A260F0BC37
:1058E000704700BFA017002008B5FEF74DFC0A2046
:1058F000FEF782FB10B1D0F80930186908BD00BF6F
:105900002DE9F043002ADDE907EC21DD4C2707FBF8
:105910000EC7013901EB020811F8016FBEF1000F4B
:105920004FEA8606C6F10A064FEA66060CDD6446B3
:1059300010367600A519EA7993F800904C3469F393
:10594000C702A742EA71F5D1414503F10103E3D152
:10595000BEF1000F09DD4C2303FB0ECEC0B28CF864
:1059600025000CF14C0CF445F9D1BDE8F08300BFE3
:10597000F0B40024D0F80D70D0F801C07D7BDCF8C5
:10598000380005F01F0505F00306B601AD0804F167
:10599000100300EB43039979DA7901F03F0122F01B
:1059A0000702013431432A43112C9971DA71EED187
:1059B000002290F84A3080F8482023F01F0380F836
:1059C0004A3080F84920BC783D7863007A789CF8AA
:1059D0000010DBB2EE18C6708270047144718571DC
:1059E00000297FD00A3A1344C371002401254FF0E7
:1059F0004053447685763A7983F8E8207A7983F8BB
:105A0000E920BA7983F8EA20FA7983F8EB20BA7AA8
:105A100083F8EE203A7B83F8EF209CF8062083F889
:105A20008E2093F8892042F0300283F8892093F881
:105A3000A12064F3041283F8A1209CF8032083F8CA
:105A4000A920002952D183F8981093F88B2042F0B6
:105A5000010283F88B204FF04053012200210424DF
:105A60004FF4F97083F88D4083F8B02083F8C510A7
:105A700083F8812083F880209CF8044083F88440D8
:105A80007C7C83F89F40BC7C83F89E4083F89C100C
:105A9000A3F8CA0083F8CD20FA7C83F800219CF893
:105AA000072083F805219CF8082083F80A219CF838
:105AB000092083F810213A7D83F8DA2093F8A32097
:105AC000B97D61F3061283F8A32093F8A320F97D32
:105AD00061F3020283F8A3207A7D83F8A020F0BC52
:105AE000FEF77EB8033A1344C3717EE783F89850FB
:105AF00093F88B2064F3000283F88B20ABE700BFA0
:105B00002DE9F04FB0F1000885B0D2F801A046DDD4
:105B100099464FF0000B4F1E4C239AF80160CBF1D1
:105B2000210404EBD4740BF00305012E4FEA640446
:105B300003FB059517F8011F34DC324602A812F06A
:105B400059FF46B3029B3F2B1946A8BF3F21039A3A
:105B5000002B134401F03F01B8BF00213F2B184632
:105B6000A8BF3F20002B00F03F004FF00002B8BF5D
:105B7000002004F1100C05EB4C0C4AB3A3181033B1
:105B800005EB430393F806E061F3050E83F806E0A6
:105B90000132B242F1DB0BF1010BD845BCD105B0AB
:105BA000BDE8F08F3046019105F0B0F8044106FBE6
:105BB00004F40F2C019906DD012202A812F01AFF4D
:105BC0000126029BBFE7324602A812F013FFB9E795
:105BD0009CF8063060F305038CF80630D8E700BF68
:105BE000F0B5D0F809308BB01968D0F80150DE68F4
:105BF000D0F80D4021B102462D4B0620FFF780FF63
:105C00006B7953B14EB101272A7DE968284D207C7C
:105C10003346CDE90075FFF773FE0022E378CDE946
:105C20000722012B8DF8242016D1224807AD0DF153
:105C30002506002303EBC301415C0133082B42EA34
:105C40000102F7D105F8012BAE4200F1010001D0AD
:105C50002A78EEE79DF81C2007A80023144D01E0E8
:105C600010F8012FE9180133092B0A72F8D149F60F
:105C70004041A0786378227803EB4003134400206E
:105C8000053301225B00A226042591FBF3F4029068
:105C900009490A480491039007AB0596CDE90052E3
:105CA000114664200794FCF72BFC01480BB0F0BDB3
:105CB000C8070460642E0020589D0100449D010027
:105CC000F0B50546B3B068B3421E022A01D933B01D
:105CD000F0BD03AF1C46BC4603F1400E664620688B
:105CE0006168A268E368103474450CF1100C0FC6AB
:105CF000F4D15E26389B13AC186859689A68DB6843
:105D00000FC4389B186959699A693B4607C4389A89
:105D10001A49908B2A4620800C68009600210120A9
:105D2000A047D4E70E46144603AF0146BC223846CE
:105D300012F08FFE31683846802212F07FFE246810
:105D400023AE04F1300C354620686168A268E36830
:105D50001034644506F110060FC5F4D1206861685F
:105D6000A268BC2407C60022044800943B4604688D
:105D700011460120A04733B0F0BD00BF8CC7010021
:105D8000002370B5104C1946236063603C220F4815
:105D900012F05FFE00F0DCF94FF480610C4A0D4D0B
:105DA00092680D4B0D4C986091606B682468984721
:105DB000AB68064698470234024631462046BDE8A5
:105DC000704012F03BBE00BFC8290020C82E002042
:105DD000580A00208CC701001C200020080A00205F
:105DE0002DE9F04F264C0E46217885B081420546BC
:105DF000DDE90E899246DDF840B020D0A378AB42B1
:105E000002D005B0BDE8F08FE378002BF9D07F22F7
:105E10001C4B00921C4900226420FCF7B9FB2DBBEF
:105E20004FF4F0600121F368184C24680E902A4664
:105E30000846A446039405B0BDE8F04F60471F46EE
:105E40006378002BDAD077220E4B00920E490022A5
:105E50006420FCF79DFBCDF800B04B4608F1100222
:105E600007F110012846FFF72BFFC7E76B1E022B37
:105E7000C7D84FF470700121044C5346D5E700BFDA
:105E8000C8290020D09D0100E09D01008CC70100C1
:105E90002DE9F04F564C89B06479DDE9125714B9F9
:105EA00009B0BDE8F08FCDE904238946A022002186
:105EB0008046504812F0CDFD9B224F4B00924F4937
:105EC00000226420FCF764FB00224D4C944692466D
:105ED000484BDFF834E105F1FF3B039744E000282D
:105EE0000CBF012002204FF487651A70587038F9F2
:105EF00012000CF1010C05FB00F08EFB006505445F
:105F0000C017C0EBE52040F62415588039F912007F
:105F100005FB00F08EFB00650544C017C0EBE520D3
:105F20009880049830F91200A3F808A0FE28C8BF92
:105F3000FF20D8800598A3F80AA030F91200FE28A7
:105F4000C8BFFF2098810398805C987338F91200CD
:105F5000208039F91200608001320A2A217103F190
:105F6000100304F1060433D01BF8011F2079002927
:105F7000B5D10028F0D04FF48766B4F90050B4F9D9
:105F8000020006FB05F540F6241606FB00F08EFB2A
:105F9000056706978EFB00674FF003065E70069E4E
:105FA00007972E443746079E1A700644C017C0EB69
:105FB000E620039EED17B65CC5EBE725D980198175
:105FC000598199810CF1010C5D8098809E73C3E723
:105FD0000C4BCDF848C01B6803220393039C02219D
:105FE0000120A446034B09B0BDE8F04F604700BF55
:105FF000C8290020E0170020D09D01001C9E010050
:10600000C82E00208CC701008100088010B584B024
:1060100003F080FA174B42791978914216D04479EF
:10602000154AE4B21C70136803938CB94FF4817263
:10603000124B0092124922466420FCF7A9FA022171
:106040000094234622460846039CA04704B010BD96
:10605000FA220A4B00920B4900226420FCF798FABE
:1060600000230221009308460122039CA04704B0AC
:1060700010BD00BFDC1700208CC70100D09D0100BF
:106080009C9D0100849D010010B582B003F042FA8E
:10609000437F93B140F213120446094B0092094921
:1060A00000226420FCF774FA0023074863771A463D
:1060B0000468009319460220A04702B010BD00BF3B
:1060C000D09D01000C9E01008CC70100F0B587B087
:1060D00003F020FA104CC37F22789A421AD0012292
:1060E000002540F22717C67F0C490D4B0092049102
:1060F0000393114623460597CDE901556420267088
:10610000FCF7FEF9074922782B460C68009506211A
:106110000220A04707B0F0BDDD170020D09D010090
:10612000BC9D01008CC7010010B582B0FFF7ACFF29
:10613000FFF76CFFFFF7CAFF0023044900930C68C8
:106140001A4604210120A04702B010BD8CC70100EF
:1061500000487047801800204FF48060704700BFEF
:10616000FAF790B812F06ABC12F073BC0F2330B586
:10617000012583B0054C00930022054B054964209E
:106180002570FCF705FA03B030BD00BF9D27002045
:10619000C09E0100D09E01003C23F0B505460E468E
:1061A0001446144F8BB0009300223B4612496420E2
:1061B0000994CDE90756FCF7EBF94FF03F0C0121AC
:1061C000002004220D4BCDE9011000920393CDE98C
:1061D000047C07AB03226420FCF792F9003418BF5B
:1061E0000124074B03EB450203F8156054700BB014
:1061F000F0BD00BFC09E0100649E0100989E01009A
:10620000C8290020162330B583B00446009300222D
:106210000B4B0C496420FCF7BBF90B4A40F2F1210F
:106220001346104623F8021B0C2125686468C2F847
:1062300002505C6003B0BDE8304003F09FB900BF7E
:10624000C09E0100449E01002C3100200048704790
:10625000EC9E01001EF0040F0CBFEFF30880EFF37B
:1062600009808169004A10470DE60000684620F069
:1062700007018D4601B401BC8546704772B61EF019
:10628000040F0CBFEFF30880EFF30980004A1047BA
:106290000564000072B61EF0040F0CBFEFF3088017
:1062A000EFF30980004A10470964000072B61EF03F
:1062B000040F0CBFEFF30880EFF30980004A10478A
:1062C0000D64000072B61EF0040F0CBFEFF30880DF
:1062D000EFF30980004A104711640000684620F07F
:1062E00007018D4601B401BC85467047684620F021
:1062F00007018D4601B401BC85467047684620F011
:1063000007018D4601B401BC85467047684620F000
:1063100007018D4601B401BC85467047684620F0F0
:1063200007018D4619B507232B4CB020237308F0C5
:1063300023F90021294A2A4BA1709A420CD2111D3F
:1063400003335B1A23F0030326480B4450F8041B65
:1063500042F8041B9A42F9D1234A244B9A420CD2A8
:10636000111D03335B1A23F0030321480B4450F83B
:10637000041B42F8041B9A42F9D11E4A1E4B9A4252
:106380000AD20020111D03335B1A23F003030B44D0
:1063900042F8040B9342FBD1EFF30882174B9A4269
:1063A00005D94FF0CD3143F8041B9A42FBD84FF684
:1063B000FF72094B1A8707F0DFFF07F0E9FF10496A
:1063C000002007F08BFF044600F04EF8844200D016
:1063D000FEE709F00BFDFBE700001050005600201F
:1063E0009856002080000000000000203412002099
:1063F00038C8010034120020682900203032002003
:10640000FCFB0100704700BF704700BF704700BF32
:10641000704700BF014B93F821007047C0FB01009B
:10642000014B187E704700BFC0FB0100014B587E36
:10643000704700BFC0FB0100014B987E704700BF52
:10644000C0FB0100014BD87E704700BFC0FB0100BC
:10645000014B986A704700BFC0FB0100014BD86A2E
:10646000704700BFC0FB0100014B1868704700BFB8
:10647000FCFB01002DE9F04F4FEA820B83B00BF1DA
:106480000A0525F0070500AFADEB050D6D463B6035
:106490004B68D1F80080064614468A467B60C047A8
:1064A0005A462846002112F0D4FA012202FA06FBCD
:1064B0001BF1FF3B17D37B6898478146BBF1000F68
:1064C00000D0C047002CF3DDAC4600215CF8043B53
:1064D00059F8042B013113448C424CF8043CF5D19B
:1064E0001BF1FF3BE7D2002C09DD2946002251F8C1
:1064F000043B01323341944241F8043CF7D1DAF8CD
:1065000008302946204698473A68DAF80C30294680
:10651000204698470C37BD46BDE8F08F01322DE983
:10652000F04191FBF2F404FB121282B0DDE90A673C
:10653000DDE90C4512B102B0BDE8F08120228046B1
:1065400000921846DDE90812012304F045FBB8F17A
:10655000000FF0DD04EB48020FFA87FE0FFA86FC0D
:1065600008E0634655F8041B944203FB101345F8FA
:10657000043CE0D034F9023BB342F2DCBB42B8BF8A
:106580007346EFE72DE9F04F14469846D31D85B0CA
:1065900023F0070300AFADEB030D95007960834650
:1065A000002168463A6012F054FA05F10A0323F01C
:1065B000070341462046EA46ADEB030DBB6B984707
:1065C000FB6B9847E94601462A46484612F036FAE0
:1065D000002C40F38880434608EB040113F8012B9C
:1065E00001328B4203F8012CF8D141463868BB6B6D
:1065F0009847FB6B9847043D04384D44A9F10403C8
:10660000514642464FF0FF0C4FF0010E08E0AB42FE
:1066100081F800E01C6001F1010102F1010211D0DA
:1066200050F8044F53F8046FA642F0DB1478AB42E5
:1066300004F1FF3481F800C0147001F1010102F18E
:106640000102EDD13B685E1E56440AF1FF334FF064
:10665000000A1D46C4461C46012209E078688842AB
:106660000FDB00228CF80010B4420CF1010C0ED0AC
:1066700014F9011F0029F7D09CF8000001448B4554
:10668000ECDDB44284F800A00CF1010CF0D182BB27
:10669000C7E9023241463868BB6B9847FB6B9847A5
:1066A000D7E9023284469E4605E049F82200AC4212
:1066B00002F1010215D015F9011F0029F7D05CF88D
:1066C000220059F822308342EFDB18F80200AC4276
:1066D000A0EB010108F8021085F800A002F1010208
:1066E000E9D17346B5E7BB6B414638689847FB6B09
:1066F00098471437BD46BDE8F08F00BF2DE9F04F35
:10670000012683B00138B2F100080D4600AF9B4668
:1067100006FA00F640F39880013B03EB0800F1B263
:1067200003F8011F8342FBD1761000F09D804FEAF1
:10673000880AAAF10409C7F804A07C6BD7F830A036
:1067400059464046D047A047B8F1000F13DD5B46DD
:106750005FFA86FC011F00EB090E51F8040F1A784E
:10676000A842A2EB0C00D6BF624418701A707145A3
:1067700003F10103F1D17610E2D1594640463B6B5B
:10678000D7F804A098477B6B98470AF10A0323F0D7
:106790000703ADEB030DB8F1000F02466C465CDD5C
:1067A000043C161F20463146AAF1040A02EB0A0CEB
:1067B00051F8043F5B1B8C4540F8043FF8D1D946A3
:1067C0005B46304602EB0A0E50F804CF1978AC4510
:1067D00001F1FF3CD6BF013183F800C0197070454C
:1067E00003F10103F0D1594640463B6B7A6098476C
:1067F0007B6B98477A68924456F8043F54F8042F0C
:106800005B1B002A83EAE371A1EBE371B8BF52423C
:106810008A420ADA99F80020002B02F1FF31D6BF34
:10682000013289F8001089F80020B245236009F18F
:106830000109E1D1594640463B6B98477B6B98472D
:106840000C37BD46BDE8F08F76107FF470AF3B6B20
:106850005946404698477B6B98473B6B59464046A4
:1068600098477B6B9847E5E7594640463B6B98470E
:106870007B6B98474FEA880A0AF10A0323F0070363
:10688000ADEB030D02466C468AE700BF2DE9F04FE1
:1068900083B00D9EDDE90F9C002E40DDDFF8848083
:1068A000DF021D0388FB073B88FB05380E9BFF17A3
:1068B000ED17013B5200C5EB6815002400EB010801
:1068C0004FF47A7E41F2301AA7EB6B171E44411A3F
:1068D00001921AE008FB00FB59F82400019A3818CD
:1068E00090FBF2F00EFB00F090FBF5F00EFB0BFBC3
:1068F0000AFB00F00C9A9E4202FB10B090FBF1F0F4
:106900004CF8240004F1010409D013F8010F002809
:10691000E0D19E424CF8240004F10104F5D103B00B
:10692000BDE8F08F1F85EB512DE9F04F17469A46D1
:106930000646850097B02A46DDE920490846884684
:10694000002112F086F82A460021384612F081F81C
:1069500072000021504612F07CF82A464846002179
:1069600012F077F8002E40F38B800023CE4602937E
:10697000239B221FC3EBC3730F925B002A44CDF805
:1069800018A00B9711920E93CDF81C800F9B53F813
:10699000041F0F934FEA116BC1F307435B450C9142
:1069A0004ED80123239A25989A400BFB02020392AA
:1069B000DDE923200BFB02020892029A93400A931E
:1069C000CBB20193C1F307230D930D99019B99421B
:1069D00027DB089B4FF0010C5E18DDF82C8005E0EA
:1069E000900650D4019B01398B421ADC16F801291C
:1069F000029B9A42F4D1039B079C33F91120236830
:106A0000069D01FB023328882360D8F80030013945
:106A10000BFB0233C8F80030019B10448B422880E6
:106A2000E4DD039A0E990C9B0A4403922399089A79
:106A30000BF1FF3BC3F30743521A5B450892C4DDD9
:106A4000069BB3F900205AB107990B685B0293FBD0
:106A5000F2F30B600B990B685B0293FBF2F20A6096
:106A6000029B0F9A01330293069B02330693079B06
:106A7000043307930B9B04330B93119B934285D1F3
:106A800017B0BDE8F08F00234FF601701C464A4D49
:106A900016AF2D7847F8040D04952498474D0593BB
:106AA000149500EB010A02F00F05099245FA03F074
:106AB000C2071AD514AAD056239A584402FB00A044
:106AC00013F90790049A10F809900CFA09F091450F
:106AD00040EA040009D2A04207D0059A044616A84D
:106AE0001044013200F80C9C05920133042BDDD1D7
:106AF000DDE909231C423FF475AF039B33F91130E4
:106B00000993D30613D49DF808307370079D099834
:106B10002B68069F01FB00333A882B60D8F80030C1
:106B200002440BFB0033C8F800303A805AE74FF0BC
:106B30000009059B0DF14B005A1E914500EB030720
:106B40000DF14C0A1846CDF840B01CDA09F10109E4
:106B5000484514DD54469AF800B0049214F8013FF9
:106B60009B452ABF1D465D465B465EF825200CFA14
:106B700003F31343A7424EF82530EFD1049A914511
:106B80000AF1010AE2DB059BDDF840B0032B0BD0D4
:106B9000042B05D0022BB9D1099B5B100993B5E7F3
:106BA000099B9B100993B1E74AF6AB23099A03FBB3
:106BB00002F35B140993A9E7049F0100000001FFA1
:106BC0000288014B1A807047841C00202DE9F04197
:106BD0004FF4614C4EF2B057184C069E94F800806A
:106BE00094F801E006EB410611F1FF3123D336F9A9
:106BF000024D002CF8D053F8215032F9214068B9E9
:106C000005F5807504F58074B8F1000F01D0C5F565
:106C1000F055BEF1000F01D0C4F580440CFB05F522
:106C200007FB04F42D14241442F8215043F82140AA
:106C300011F1FF31DBD2BDE8F08100BF841C0020E0
:106C40002DE9F843984604460F46164602F062FCCA
:106C5000437A40F6FE72022B14BF0D25002544F244
:106C6000507E49F64E3CC5F57F6108EB04030F31B9
:106C7000A2EB050814F1FF341FD313F8010D00280F
:106C8000F8D037F9140036F914900CFB00F000141A
:106C90009042A8BF10460EFB09F94FEA29494D451D
:106CA00020EAE0700BDA4945D8BFC14627F8140046
:106CB00026F8149014F1FF34DFD2BDE8F883A9461A
:106CC000F4E700BF0288014B1A807047881C00203F
:106CD00000231849184A70B41848194E194D1A4C17
:106CE000C1E900330B81C2E9003318491381184A06
:106CF000C6E90033C6E902333361C5E90033154EF6
:106D0000C5E902332B61C4E90033C4E902332361CE
:106D1000C0E90033C0E902330361C1E90033C1E9CE
:106D200002330B61C2E90033C2E9023313613370ED
:106D300070BC7047A81F0020D01E0020681F0020D4
:106D4000DC1E0020F01E00202C1F0020181F002039
:106D5000041F0020A41F00202DE9F04F8BB09DF8E8
:106D60005460794CCDE9026027786578774C0193BF
:106D70002478029B92469C4238BF744A0E468DF896
:106D800024708DF8255038BF1370149D092404F029
:106D90009BF9039B0490DFF8CC91DFF8CC81DFF8FE
:106DA000CCB12544123603F1120739E018F804205B
:106DB0000AAB0B4413F804CC0132D2B264489445B8
:106DC00008F804204FEA440330F914003BF914E0BA
:106DD000009745D20022297808F8042009F8041009
:106DE0005C4AD0525C4A5A4822F803E0009AB2F951
:106DF0000020C252B6F9002058482BF803203AF977
:106E00001420C252019A564832F91420C252013C51
:106E1000631C05F80119A7F10207A6F1020639D093
:106E200004F0FEFE58B13AF91430002B07DDB6F934
:106E30000030B3F5007FBCBF01238DF8243019F872
:106E400004102B788B42B1D1002308F80430630082
:106E50003F4A3BF903E0D05E039A1A440092BFE731
:106E6000002ABDD02A781AB9384A1278012A18D0D7
:106E700038803BF903203280384A0198D25E2AF8E4
:106E80001420374AD25E20F8142018F80420002A73
:106E9000BDD1DDE7029B0BB92C4A13700BB0BDE8E6
:106EA000F08F049A132AE3DC2A4AD25E00922A4A1F
:106EB00032F903C0009A002A42D0009A821A002AAE
:106EC0000692B8BF52420592AEEB0C0200920792B6
:106ED000059A772A05DC009A002AB8BF5242772A21
:106EE000C6DD41F6CC0CA0F1C90292B26245BFD812
:106EF0006FF4C87243F24A6C724492B26245B7D8DA
:106F000041F65C2C069A02EB420202EBD27200EBD5
:106F100062020092013A6245AAD8079A02EB420C3B
:106F20000CEBDC7C0EEB6C0E43F66A1C0EF1FF32B0
:106F300062459DD8BDF800203A80A6F800E09BE7A6
:106F4000BCF1000F94D0B8E7881C0020A41F0020DB
:106F50002C1F0020DC1E0020F01E0020181F002027
:106F6000041F0020A81F0020D01E0020681F002042
:106F7000F8B505461A4C0146B022204611F05EFDD8
:106F80002E1D04F15C0C0FCEACE80F000FCEACE868
:106F90000F0096E8030005F1300704F188068CE83D
:106FA00003000FCF0FC60FCF0FC697E8030086E888
:106FB000030005F18807261D0FCF0FC60FCF0FC6A0
:106FC00097E803005C35303486E803000FCD0FC42A
:106FD0000FCD0FC495E8030084E80300F8BD00BF9F
:106FE0008C1C00202DE9F84F92460F461D460446A2
:106FF00002F090FA834604F067F89BF80920012A12
:1070000032D0414E05EB440506F1300906F1040883
:1070100014F1FF3428D335F9023D002BF8D057F88E
:107020002430B26D93423DDA9BF8091002295FD1FA
:107030007F209B1A00FB03F302EBA31247F82420E6
:107040005AF824103368994210DA9BF80920022A72
:1070500046D17F20C91A00FB01F103EBA1134AF8C6
:10706000243014F1FF34D6D2BDE8F88FF36AC1F5AD
:10707000E0519942CCDA9BF80920022A42D008B2AA
:10708000494603F015FE5AF82410F36AC1F5E051A1
:10709000C91A00FB01F103EBA113C3F5E0534AF851
:1070A0002430B5E7D6F88420C3F578539342C7DA85
:1070B0009BF80910022923D018B2144903F0F8FDF7
:1070C00057F82430D6F88420C3F578539B1A00FB78
:1070D00003F302EBA312C2F5785247F82420AFE77E
:1070E00008B2414603F0E4FD33685AF82410B1E7D2
:1070F00018B2074903F0DCFDB26D57F8243098E769
:107100007F20E3E77F20C3E78C1C0020141D0020B4
:10711000E81C00200346997A254A0078012930B4FA
:1071200010701FD0197C01290BD009B921480170BA
:1071300053F8120F20491B79C2F812000B7130BCB2
:107140007047D089D989884220D0194651F80C0F50
:107150001A4C8988D060A1800120022415491C7432
:107160000870E5E710891989884214D0194651F84A
:10717000025F13484C680989C2F8025044600181DB
:10718000002002240B499C720870CBE790899989F2
:107190008842DAD1E0E7D088D9888842E6D15088A1
:1071A00059888842E2D1908899888842DED1E7E701
:1071B0003C1D0020B02D00204E1D0020481D002049
:1071C0003E1D002010B4314C314B04FB00F49C42B6
:1071D00029DB4FF4876202FB00F02E4AA2FB00324B
:1071E000801A02EB5002D20A40F6241303FB01F18D
:1071F000284B294CA3FB01032078C91A03EB510348
:10720000DB0AD0B9A27C002A36D0B4F813209A4207
:1072100038DCB4F8152010BCC2F5126204329A4270
:10722000B8BF032070471D4AE31782FB04021444D1
:10723000C3EBE42404F58762D6E71949097891B9CC
:10724000E18891421BDCA188914201DD642B19DCAD
:10725000218991420DDCA27C012072B1B4F8132087
:107260009A42D6DD0EE0A18991420BDCE189914280
:10727000F1DD022010BC7047104610BC70476188D9
:107280009942E0DA032010BC704700BFC8FBFFFF43
:107290001E32DEFF010110003C1D0020810008802D
:1072A000B02D0020F0B49DF81840079D022C25D089
:1072B000032C19D0012C02D00020F0BC70473B4BAE
:1072C0005B5D002B41D10922394B3A4EA3F10A05EF
:1072D00013F8011D022908BF9455AB4202F1FF3299
:1072E000F6D1F0BC01207047304B5B5DA3B1324B4F
:1072F0005B5D023B012B0FD90420DEE72B4E765D50
:1073000086B12D4E765DB71E012F2DD92B4A042054
:1073100052F82530013314E00122264B03205A5540
:10732000F0BC7047264C274E24F815002648274C01
:1073300020F815300220012324F815201F4A26F8D2
:10734000151042F82530F0BC70471B4B5B5D022BDB
:10735000C7D11A4B53F825302F2BC2DC1C4A1D4BCA
:1073600054551C702046A8E7032EDBD044F6C466B3
:10737000144A134B32F9152033F91530891A01FBE1
:1073800001F1C01A00FB00100C4AB04252F825105F
:1073900001F1010308DD2F2906DC01210D480C4C09
:1073A000017061550420CCE72046CAE7D42D0020A7
:1073B000EA290020EC310020E0290020182F0020CD
:1073C000D4310020F8310020042F0020B42D0020FB
:1073D000C82D0020283100202DE9F04F00248FB067
:1073E000CDE90C23804BCDE90A011C7002F092F824
:1073F000437A002B56D17D4B1A78002A4FD00023B8
:1074000009931C460A9B189DA3F102090B9BA3F14B
:1074100002080C9BA3F1020B0D9BA3F1020A22E0D0
:10742000734A125D022A00F097800023714A1355B7
:107430006F4A13552B78704A1355BDF81430013438
:10744000A9F80030BDF818300A2CA8F80030BDF8B3
:107450001C30ABF80030BDF82030AAF8003005F839
:10746000016B00F09180002739F9023F059338F94C
:10747000023F06933BF9023F07933AF9023F089314
:10748000199B1F555D4BE7542E78002E32D15A4B75
:107490001B5D002BC4D1564A1E461355CBE79B7C7F
:1074A000002BACD10023564ADFF860E1DFF860C161
:1074B000544F524E4E4D504C4E48534902F1140811
:1074C00022F8023B42452EF8023B2CF8023B27F8FB
:1074D000023B06F8013B05F8013B04F8013B00F8CC
:1074E000013B41F8043BEBD10023099309980FB00D
:1074F000BDE8F08FBDF81810BDF81400FFF762FE6C
:107500000A23199ACDE90204DDE90501CDE900322B
:10751000DDE90723FFF7C6FE042830D0012804D98F
:107520003E46334B18552B7885E7314B1B5D022BBC
:10753000F7D10128F5D1334B344933F91430344AAB
:1075400008932F4B31F9141032F9142033F9143009
:10755000069107920593E4E72B4A52F824202F2A3C
:107560003FF763AF234A125D002A7FF45EAF1E46E9
:1075700009930123199A13551B4A137055E71C4BA5
:107580001B5D022BCDD1D6E7174B1B78002BADD05E
:10759000DDE90ACEDDE90C89DDE918AB002301271E
:1075A000164A174E194D1A4C164812F8011B11B9FC
:1075B0001BF8031089B136F913102CF8131035F9A4
:1075C00013102EF8131034F9131028F8131030F993
:1075D000131029F813100AF8037001330A2BE4D1B1
:1075E00009980FB0BDE8F08F283100203C1D002025
:1075F000E0290020EC310020D42D0020C82D0020EF
:10760000D4310020042F0020182F0020F831002052
:10761000B42D002001465422014811F00FBA00BFDA
:10762000E80700200021044B03F1780299600C3335
:107630009342FBD1704700BF5C3100202DE9F04F31
:107640003F4F85B03C68DDF83880012C08BF002230
:1076500000295AD04FEA400A0AEB0001394D89004F
:107660006E18B4680A2C59DDD3F800C00AEB00018B
:1076700005EB810149680AEB00094FEA89090446D4
:1076800055F809001E46D8F80030ACEB0000591A36
:107690000028B8BF40420029B8BF4942039203F016
:1076A000B1FA039A834607EB0217D7E902237968F8
:1076B0003F69009703F090FA05EB090700283BD0DB
:1076C000326855F8093002FB0BF203FB00230BEB89
:1076D000000251100B4493FBF2F33360D8F80030F2
:1076E0007F6803FB0BFB07FB00B0084490FBF2F044
:1076F000C8F8000033685444A4002B51D8F8003077
:107700002C44636005B0BDE8F08F0E4B00EB4000E9
:1077100003EB8000816005B0BDE8F08F0134B460F8
:10772000012CD3F800C0A1D145F801C0D8F8001051
:107730007160D3F800C09EE7D8F80000D8E700BF1A
:10774000E80700205C31002030B40546064C69682B
:10775000AA68EB6800680FC428696969AA69EB69BF
:107760000FC430BC704700BF541D00202DE9F04706
:10777000DFF8C0800021D8F804208146920011F083
:1077800068F9D8F80430D8F81020581EA0EB630030
:107790009047D8F814309847D8E9006486B3671E3C
:1077A000002C37D009EB8404013ED8F818309847F4
:1077B00082469FB3D8F804007D1EA5EB6000D8F880
:1077C00010309847FE4202D0D8F814309847D8F8C5
:1077D0001C30504698470022831E3E3033F9021F6A
:1077E00098420A44FAD154F8043D2F469A42B8BF51
:1077F0001A466B1C2260D8D1D8F80440002ECED196
:1078000004EBD4706410D8F81030C4EB6000BDE80D
:10781000F0471847013EF3D0013EBFE7D8F80420F7
:10782000D8F81030501EA0EB620098474FF0FF359B
:10783000C8E700BF541D00200E4BF0B45F68022F54
:1078400015DD00EB87070C3F0438024600230A4988
:1078500000F10C0652F8045F11F9014B964205FB4A
:107860000433F7D11B1140F8043F8742EDD1F0BC3F
:10787000704700BF541D0020601D0020DFF868C065
:10788000F0B4DCF804600024002E0ADD01EB86066B
:10789000043E0B1F53F8045FAC42B8BF2C469E4217
:1078A000F8D1DCF808304610A34214DA002818DDBD
:1078B00000236FF00045043951F8044FAC42B8BFC3
:1078C0001F4603F10103B8BF25469842F4D1B81B07
:1078D0001560F0BC704751F826300020F0BC1360F2
:1078E00070476FF00045F2E7541D0020F0B40446E5
:1078F000074E00F13007354620686168A268E368EA
:107900001034BC4206F110060FC5F4D1F0BC70472C
:10791000741D00202DE9F047DFF8E89002EB4005E8
:1079200099F82C3099F82D2082B0441E0F468DF81E
:1079300004208DF805304E464FF0000A4FF06408E1
:1079400000E0013C631C17D035F9023D002BF8D054
:10795000314637F9140003F0ABF9B5F9003098421D
:107960003EDBD9F8282008FB03F302FB00F2934228
:10797000C8BF4FF0020AE4E71F4B1878BAF1000FB6
:1079800013D11E4AC2F800A060B91D4999F82E40D3
:107990000A680132A2420A6004DD01221046C1F8E1
:1079A00000A01A7002B0BDE8F0870546AAF10200F7
:1079B000B0FA80F04009854217D0104C02A9226825
:1079C000014411F8041C01328A42226011DD0022B8
:1079D0001870226000220A4B1A6002B0BDE8F087DE
:1079E0000020054B1D788542E7D10022034B1A6029
:1079F000F0E72846EEE700BFC01F0020B41F0020BC
:107A0000BC1F0020741D0020014B1870704700BF80
:107A1000C01F0020034B1B781BB9034A13680133B6
:107A200013607047C01F0020BC1F00200278014B6C
:107A30001A7070473C0800200022034B83F8F020A6
:107A400083F8E421704700BF402F00202DE9F04F5C
:107A5000614D97B02C78002C69D000296BD0F424AC
:107A600004FB00F4DFF874811E4608EB040C9CF85C
:107A7000F0301746FF2B68D00133DBB28CF8F030C2
:107A8000D2F800E0D6F8009004F1D00B012BCDE93C
:107A900004E9C34461D00DF1100900234FF4807A4A
:107AA0005A460EA808EB040B4946CDE9063303936A
:107AB00000F096F80EAA06A9584600F045F9039B77
:107AC00059461A46CDF800A00123484600F092FA24
:107AD000012304F134011A460A904144CDF800A074
:107AE000484600F087FA04F168010B9041444FF4D6
:107AF000C8730222CDF800A0484600F07BFA04F1DA
:107B00009C010C90414449F640430122CDF800A06D
:107B1000484600F06FFA06AA0D900AAB594608A82D
:107B200000F026FADDE908232C783A60336020461D
:107B300017B0BDE8F08FF422284B02FB003320463B
:107B400083F8F01017B0BDE8F08F1268336804F1C5
:107B5000D00BCDE90423C3449DE74FF0000A6146F2
:107B6000524653468CF8F1A08CF8F2A00132042A58
:107B7000C1F800E0C1F80C904B600B618B60C1E96B
:107B80000533C1E90733C1E90933CB6201F134019F
:107B9000ECD1F4214FF4C863FA2201FB00800DF10F
:107BA000100902634266C0F89820C0F8CC208361B7
:107BB000C3648365C0F88030C0F88C30C0F894305E
:107BC000C0F8B430C0F8C030C0F8C8304946584694
:107BD00000F0A6F861E700BF3C080020402F00201D
:107BE000F0B413680F684E685568DC1BAD1B002CA1
:107BF000B8BF6442002DB8BF6D422C44C82C84B07D
:107C000004DC4EF660251389AB4274D90125C2E924
:107C10000076D1E90034341B2E46FF1A002FB8BF7E
:107C20007F42002CB8BF64423C44134694FBF5F5F8
:107C3000002123F8086F02F11C0633F8024FA1421D
:107C4000B8BF21469E42F8D1937FA942B8BF2946CA
:107C5000082B02EB43048CBF002301330529658107
:107C6000937722DD27294ADC294B4A1F03FB02F2C6
:107C7000284BD41783FB02531344C4EB631303F262
:107C8000CA341429009413DD31293DDC6FF0D10290
:107C9000143902FB01F1204ACB1782FB01520A443E
:107CA000C3EB221303F28E3304E040F2CA34009493
:107CB00040F28E3301934FF42F730146CDE9023326
:107CC000164F00F1280601ADC4F57A7287FB02C396
:107CD000A3EBE2739BB200F1080220F8023B824260
:107CE000FBD121F80A4B8E4202D055F8044BEBE74A
:107CF00004B0F0BC704701339EB2354695E74FF4AF
:107D00002F7431290094C1DD4FF42F73D2E700BFE7
:107D1000F2FEFFFFEBA00EEA89888888565555557C
:107D200070B4D1E90062034600256424C0E9006212
:107D300000F11C0223F8085F23F8024F9342FBD1A5
:107D400070BC0023837770472DE9F04F0C469246B4
:107D5000CFB003900146D0221AA8A4F1020B10F074
:107D60006DFE5D46D6465046A046804F0AF1080695
:107D7000002213461AA930F833C00C6B0133042BD0
:107D800004FB0C2201F13401F5D1B2F5FA6F34BFD6
:107D90000122A7FB023200F1020028BFC2F38F12BA
:107DA000864225F8022FE3D144460023A11D8C46CC
:107DB000CDE90633CDE908330AF1200A0DF1240993
:107DC0000DF1680806AA15464F465C467646D8F877
:107DD0003010029236F8022B34F8020F01FB02F247
:107DE000B2FBF0F2A445134445F8043B47F8042FD6
:107DF00001D02B68EEE70EF1080EF24508F13408C9
:107E000009F11009069BDDD1002108460C461AAD88
:107E100005F1D00C2A6B2F68EE683435AC4511445F
:107E200007FB024406FB0200F4D194FBF1F490FB43
:107E3000F1F1039A10461460D160934604229046F3
:107E4000CDE9040300218C460F460E460C46084639
:107E50000AAB019303EB080E1AAA00915EF8103BDF
:107E60001168D2F8089001FB0300D168D2F814A081
:107E700001FB0344516809FB03CC01FB0366116954
:107E8000343201FB0377009995420AFB03130093F8
:107E9000E4D1194606AB53F8083008F1040890FB0A
:107EA000F3F094FBF3F496FBF3F697FBF3F79CFBEC
:107EB000F3FC91FBF3F1B8F1100FCBF83400CBF8E1
:107EC0004040CBF83860CBF84470CBF83CC0CBF8DE
:107ED00048100BF1340BB5D1DDE904430399D031DF
:107EE00003910025A846AE46AC462F462E46DDF847
:107EF00004901AA9009359F8100B8B69D1F82CB093
:107F000003FB0066CB690BFB005503FB00770B6A94
:107F100003FB00CCD1E9093A34318A4203FB00EE7D
:107F20000AFB0088E7D1009B96FBF3F697FBF3F77B
:107F30009EFBF3F09CFBF3FC98FBF3F195FBF3F550
:107F4000019BC4E9066704330193039BC4E908C09D
:107F5000C4E90A153434A34204D0029951F8043F0D
:107F60000291BEE74FB0BDE8F08F00BFD34D621065
:107F70002DE9F0438C460C460026DFF87480971EEE
:107F8000043B063237F802EF53F8045FBA4205FBB0
:107F90000EF5A8FB059ECCF8305006EB9E160CF1B2
:107FA000340CEFD101250A46D031136B3432B3FBC8
:107FB000F6F3002B08BF2B4642F8043C9142F4D163
:107FC00000210D460E46236BD4F800C0E768343418
:107FD000A24219440CFB036607FB0355F3D196FB41
:107FE000F1F695FBF1F1C0E90061BDE8F08300BF57
:107FF000D34D62102DE9F04FD2B28BB0012A01921D
:10800000044600F05881C0F02881022A00F09D80CB
:1080100000234FF480629C461F461D469E469B46A9
:108020001E46984699469A46CDE907330592039332
:108030000293069304930093039AD4E90004A4EBFB
:10804000090406FB04290BFB0433A0EB0A0043F3ED
:10805000951308FB00EE06FB00550BFB007708FBB1
:1080600004CC49F39519C1E90493029B4FEAAE2E63
:108070008B61019B45F3951547F395174FEAAC2C9F
:10808000C1E900E5C1E9027C002B00F0E080009A24
:10809000059B764203FB02F3069A002B4FEA822AE5
:1080A000009AB8BF03F2FF3306FB02AABAF1000F31
:1080B0004FEAA323B8BF0AF2FF3ACB614FEAAA23E3
:1080C0004B62019B022B00F037810023C1E90A3388
:1080D0000B6204FB04F400FB0040A94B984200F340
:1080E000AE80642404FB00F0149BA64A90FBF3F4DA
:1080F0006310934200F3A38042F21071A24AE41786
:1081000082FB0302C4EB223201FB12309F4D561C4E
:1081100080EAE07401FB1633A4EBE07435F8160036
:10812000002B00FB04F035F81220B8BF5B4202FBC5
:108130000300974FA7FB0030400B01FB00F0149B9E
:1081400090FBF3F00BB0BDE8F08FD1F82090D1E9AF
:1081500006073D1809EBD970D1E90ACED1F824A061
:1081600005EB60050EEBDE7809EB0C064FEA6808BC
:108170000CEBDC7B3D4406EB08024FEA6B0B5744EB
:10818000554404925F445D4402EBD27B8A684F44BD
:1081900003924A69674409920A687344914605EB61
:1081A0006B05079307EB080300932B4648680AEB1F
:1081B0004C0A0290029AF24409EB2219039ACDF874
:1081C00018A009EB621A099AD1E9036006EB2016A0
:1081D00006EB6219002D149AB8BF05F10F0302EBEC
:1081E00023134FEA851898FBF3F8009A149396012D
:1081F000049AC8F580634FEA821B149A059396FB94
:10820000F2F69BFBF2FB029A03FB05F31546099F6E
:10821000002B3844F444039AB8BF03F2FF338001C3
:10822000CDF820C003909812099B1544AD0102902F
:1082300097019B014FEA8A2E4FEA892CFCE642F215
:108240001070149B90FBF3F00BB0BDE8F08FC1E908
:108250000733C1E90933CB623BE78869149A0344C9
:108260001846002BB8BF03F10F0002EB20124FEAB3
:10827000831898FBF2F81492C8F5806202FB03F0B1
:1082800000230028D1F800A0D1F80C90B8BF00F26C
:10829000FF3005928212CDE902231F461D469B4600
:1082A0001E46CDE907330693049300934FEA8A2EC6
:1082B0004FEA892CC0E6486AD1E9065605EB460E1E
:1082C000864403440693734632184D6800920A6848
:1082D0000F6902EB251ACA68BEF1000F02EB2719DD
:1082E000149AB8BF0EF10F0302EB23134FEA8E1856
:1082F00098FBF3F81493C8F5806303FB0EFE059317
:10830000009BBEF1000F4FEA8316149BB8BF0EF21C
:10831000FF3E96FBF3F600234FEAAE220292BA012B
:10832000AD0103921F469B46CDE9073304934FEA04
:108330008A2E4FEA892C7FE6DDE9042303FB02F352
:10834000089A002BB8BF03F2FF334FEA822C9B122E
:10835000049A0B62079B06FB02C6049A9B020BFB66
:10836000123B002EB8BF06F2FF36BBF1000FB8BFBC
:108370000BF2FF3BB6124FEAAB238E62CB62A8E64C
:1083800014AE47016F110100AD8BDB68109F010037
:108390005917B7D130B40546044C00686968AA681B
:1083A000EB680FC42869206030BC7047A41D002012
:1083B0000268014B1A607047B81D002030B40546B2
:1083C000044C00686968AA68EB680FC428692060DB
:1083D00030BC7047BC1D00202DE9F0430746032246
:1083E00000204FF0010803FB07F6079D104C2944BD
:1083F0008E5D94F80090DFF83CE0DFF83CC006F0BA
:108400000F0646FA02F4E4070CD512F90E4012F9F1
:108410000C503C4403FB0414645D4C453CBF08FA1B
:1084200004F4204312F1FF32EBD2BDE8F08300BF29
:10843000089F0100209F0100289F01002DE9F04FB7
:10844000814299B083468A4613921193DDF89C903D
:1084500001DA8B468246239B119933F91B60229BDC
:10846000239853F82B4030F91A5051F82B7051F8DB
:108470002A0004FB06F4229907FB06F751F82A109C
:10848000249B01FB054100FB057053F82B2006914E
:1084900053F82A304FEA8A010E914FEA4A015FFAF7
:1084A00082FE5FFA83FC14914FEA8B0105900F91D5
:1084B000A8194FEA4B01F44507900C92159103D28D
:1084C00011466CF307010C91C3F30721C2F3072097
:1084D000884203D20C9861F30F200C90C3F307413C
:1084E000C2F30740884203D90C9861F317400C90FF
:1084F0001B0EB3EB126F03D90C9A63F31F620C923D
:108500000C98C0F30747020E974259DC0123299CBF
:1085100007FA03F109FB01410132039128990892FE
:10852000C2B207FB0916099203FA0BF1C0F3072246
:1085300003FA0AF30B430A924FEA49020B92CDF871
:1085400010B05FFA8BF2CDF858A09B46CA460D9149
:108550001792099C0A9A944224DC02F101080CE06B
:1085600019F0100F06D10D9B834200F0A480002863
:1085700000F0B7800134A04514D016F8049019F02B
:10858000200FF7D0289B269A009321465346384661
:10859000FFF722FF8345E3D19DF8103033550134B6
:1085A000A045EAD1039B0B9A013713440393089B20
:1085B00056449F42CDD1D146DDF810B0DDF858A029
:1085C000249B0F9A19460C9B8B500E9A8C58C4F31F
:1085D0000740250E854218D3289BE6B209FB0031DF
:1085E000C4F30724771E013521443F1BA64208DC53
:1085F0007B1813F8012F924508BF83F800B0994209
:10860000F7D1013085424944F0D1059B079D1A46B8
:10861000069B92FBF5F01A4692FBF5F1119A229C0B
:1086200016460F9A0023B05026460E9CB15025994D
:10863000159E0C192399139F8D530AF10100149D67
:1086400087424B530EDD259B01261946259B8958F1
:108650009D18226806FA00F313400130194387423F
:108660002960F6D10023259A0E999A45535077DD5B
:1086700001220F98259F02FA0AF138440646CC439E
:10868000154602FA0BF006E00243224047F8232089
:1086900001339A4564D057F823200A42F8D09B450D
:1086A000F2DCF2DA326805FA03FC42EA0C023260CC
:1086B00057F82320E9E79DF8103007983355039BBE
:1086C00033F9143004FB03F107FB03F21844059B54
:1086D000079003EB41230593069B03EB422306938C
:1086E00048E709F00F03109603251E46CDF8488091
:1086F00046FA05F3DB072CD51B4B269A15F90380A8
:108700001A4BB84415F90390289BA14400934046A6
:1087100049465346FFF760FE83451AD1289B179AB6
:108720000AFB0838109B08F809201946039B0A55D4
:1087300033F91430079804FB03F107FB03F21844E4
:10874000059B079003EB41230593069B03EB422314
:10875000069315F1FF35CBD2109EDDF8488009E76E
:1087600019B0BDE8F08F00BF209F0100289F0100D5
:108770002DE9F04FDFF8C4B089B09BF80C40002C15
:1087800059D0002857DD00251F4637F9153005F16F
:10879000010A002B914688460646544649DD564557
:1087A00003DC48E00134A6423BD037F91430002BFB
:1087B000F8DD59F8243059F8250058F82510C01A6A
:1087C0004EF2B05358F82420891A0029B8BF494204
:1087D00003FB01F14FF461430028B8BF404203FBA3
:1087E00000F00914001402F00DFADBF81030834297
:1087F000D8DD179B21460793169BCDF80090069372
:10880000159B32460593149B28460493139B013411
:108810000393129BCDE901734346FFF70FFEA64277
:10882000C3D1554637F9153005F1010A002B5446DE
:10883000B5DC5645F5DC09B0BDE8F08FBC1D002065
:108840002DE9F04F634C91B0E47B34B3002824DD74
:108850001F4690468A4681464FF0000B37F91B3081
:10886000BBB158F82B201D9902F58072521201FB02
:1088700002F65AF82B301E9903F5807331445B12CF
:10888000C95C55485945057820D0A94209D38806C6
:108890006DD40BF1010BD945E0D111B0BDE8F08FDB
:1088A00077461F9BCDF8008007931E9B4A46069390
:1088B0001D9B584605931C9B04931B9B03931A9B7B
:1088C000CDE901735346FFF7B9FDE2E74FF0FF3002
:1088D0006FF0FE1E844603243E49CDE9085789689F
:1088E000CDF83CE00C913D490DF1380E0E911F99E9
:1088F00001EB46010B9159000A910FAE1CEB020CE3
:1089000018442CD400282ADB1C99614527DD1D99C9
:10891000814224DD01FB0CFC1E99089D6144095C29
:10892000A9421CD20A9F8B4507EB4C0C17D0642739
:108930001F9D35F90C500D950B9D35F913C00D9DFC
:1089400007FB05F50C9F07FB0CFC654507DD64255F
:108950000B9F37F9100005FB00F0604537DC24B1B0
:10896000013C14F90EC0A057C8E7099F91E71A9877
:1089700050F82B00C0F307249C4224D0C0B2984288
:108980000BBF032401244FF0020C4FF0000CBE4635
:1089900001F00F001E990B4440FA04F1C9070DD5F0
:1089A0000F491D9F61560F4E114407FB0131A65719
:1089B000895DA94202D259457FF472AF013C6445FA
:1089C000EADA774665E703244FF0020CDFE7099FF8
:1089D00067E700BFBC1D0020089F01000101FFFFE9
:1089E000209F0100289F01002DE9F04F83B0DDE9B1
:1089F0000D4704FB02FE07EB0E04E65C864245D001
:108A00008E4243D016F0200549D000250324AA4603
:108A10004FF0010BDFF8A4C006F00F069CF80090A1
:108A2000019307EB030C46FA04F7FB0715D5214F1A
:108A3000214BE75714F903800D9B174403FB07C72D
:108A400017F808800BFA08F7C84547EA050704D26B
:108A5000AF421CBF3D460AF1010A14F1FF34E2D2D5
:108A6000012202FA00F002FA01F10843A842019B38
:108A700019D0284010D05B0003EB4E0E0F9B33F94A
:108A80000E0090FBFAF003B0BDE8F08F5B0003EB43
:108A90004E0E0F9B33F90E0003B0BDE8F08F284651
:108AA00003B0BDE8F08F934003EB4E0E0F9B33F9FC
:108AB0000E00F1E7209F0100289F0100089F0100A0
:108AC0002DE9F04FB74CA9B0A47B1A94002C00F00C
:108AD0000E81002800F0038116930023CDE91812BF
:108AE0000E93431E12901D930E9B1D9A934280F28B
:108AF000FE80339B0E9A194651F82230511CCB4010
:108B00004FEA82021B9113920D9300F04881129B51
:108B100019461B9B994240F342810C9300230E9A05
:108B20001C93169B03EB420317930BE00C9B0D9ACF
:108B3000013352080C930D9200F02D81129A9A4243
:108B400000F029810D9BDB07F0D5189B13991C467B
:108B50005858199B0C9A1D4654F82240595855F8FC
:108B60002230051B0A940B93CC1A85EAE573A3EB1C
:108B7000E573149384EAE473A3EBE4731593169EF0
:108B8000179B36F91220B3F90030002C40F0F98021
:108B9000002D40F011814FF4007BDDF868800A9EC3
:108BA0000B9F34463D4604FB03F402FB004405FBE7
:108BB00003F5134494FBF3F402FB015595FBF3F525
:108BC000329B139A9C469A5820941446CDE9216111
:108BD00000260C9B1F905CF82330D0B2D9B28142A2
:108BE00038BF61F30704C2F30720C3F307218842AB
:108BF00038BF61F30F24C2F30740C3F30741884233
:108C00004FEA136388BF61F31744B3EB126F88BF59
:108C100063F31F642395230EC4F307459D422497F5
:108C2000CDE92566279600F3CD8001330F93E3B29B
:108C30001093C4F30723119325AF109C119A94420B
:108C40005CDC9DF838306E02099333464646984600
:108C50009DF830A002F10109379B2A460393369B09
:108C600051460293359B09980193349B0093234608
:108C7000FFF7BAFE00283DDDDDE90A324FEA442C59
:108C80000221ACEB030E0EB30BFB0EF3A2EB63233E
:108C9000A3EB0803002BB8BF5B42B3F5007F09DAF2
:108CA000C3F5007300FB03F357F8212002EB6323A5
:108CB00047F82130F1B101391FAB53F8213022AA16
:108CC00052F82120ACEB030E002EDDD1A8EB0202FE
:108CD0000BFB02F2A3EB6223A3EB0C03DAE76FF0CA
:108CE0000043314C3149324A23600B60106029B097
:108CF000BDE8F08F01344C45AED1B0460F9B013535
:108D00009D429AD1DDE92642DDE91401259B6425C7
:108D10009A42A8BF1A4605FB04F4154601F0AAFFC3
:108D20002D2801DDC0F15A001E4A0CCA03FB00F3D6
:108D3000C0F12D0002FB00321E4B83FB0231D31722
:108D40000A44C3EB621305FB03F3A342BFF6EEAE86
:108D5000379B129A0793369B0C990693359B0E9876
:108D60000593349B0493339B0393329B0293169B8E
:108D70000193199B0093189BFFF760FB1A9B1C93B0
:108D8000D4E6DDE91467BE4216DA6D0295FBF4FB0A
:108D9000DDF8688003E71C9B002B7FF4A5AE1B9BCE
:108DA0000E93A1E6BC1D002060080020640800208E
:108DB000E81F0020B7600BB6640294FBF5FB4FF090
:108DC0000008ECE6DDE9140101F054FF2D287FF7DF
:108DD000ADAE00252C46A5E72DE9F04F634C8BB0D6
:108DE000647B002C68D0002866DD1E4691468846CC
:108DF00083460025DDF850A036F91530002B58DDEC
:108E0000002401E036F91530002B4FDD36F914301F
:108E1000002B4BDDAC4249D059F8242058F82430BF
:108E200059F8251058F82500891AC01A01F0EAFEF1
:108E300059F8242059F8251058F82430074658F8D6
:108E40002500891AC01A0029B8BF49420028B8BFB6
:108E5000404201F00FFF64232D28C8BFC0F15A0023
:108E600003FB00F3C0F12D0003EB8010404B3AF9F7
:108E7000142083FB00313AF91530014403EBC3039E
:108E8000DB10C0170A3302EBC202C0EB611003EB28
:108E9000E20303FB00F3B7EBA31F07DA36F9153043
:108EA000002B03DD36F91430002B08DC0134A34518
:108EB000A8D10135AB459FD10BB0BDE8F08F1A9B0F
:108EC000CDF800900793199B5A460693189B2146AC
:108ED0000593179B28460493169B0393159BCDE996
:108EE00001634346FFF7AAFAAC421FDD159836F935
:108EF000153050F8250059F8252058F82510029013
:108F00001A9808AF06901998059018980490179829
:108F1000039009A8CDE90070284601F03DF8DDE98D
:108F2000080101F06FFE2AF81500BFE7159836F921
:108F3000143050F8240059F8242058F824100290D6
:108F40001A9808AF069019980590189804901798E9
:108F5000039009A8CDE90070204601F01DF8DDE975
:108F6000080101F04FFE2AF814009FE7BC1D002005
:108F7000B7600BB684B038B5174D04AC84E80F0069
:108F8000202240F21461154804AC00F087F80FCCA1
:108F900028606960AA6003CC1822286169612846AC
:108FA0004FF4B871EB6000F079F80D494FF4606050
:108FB00000F0C2F80B494FF4905000F0BDF8642067
:108FC00000F0A8FC632000F0A5FCBDE8384060205C
:108FD00004B000F09FBC00BF9C290020EC1F0020C3
:108FE000380A0020480A002084B030B402AC84E87B
:108FF0000F000A4B9DF808209DF80A109DF81250AA
:109000009DF813401A7099709D72DC7230BC18463E
:1090100018224FF4B87104B000F06AB89C290020FF
:1090200070B40446174D00686168A268E368164E84
:109030000FC520696169154A03C57368A569207F5A
:1090400051692B4373600870A37F657FCB71E17F0B
:1090500093680F480570197094F820000D495870F6
:1090600094F821500C489D7094F82250DD70D3681C
:10907000A28DD4E909651A811E605D60086070BC2C
:10908000704700BFB02E0020880C0020100C00207C
:1090900034200020EC29002055960000F8B5134B31
:1090A0000C0A53F824606EB1F468CFB2013C05E0BD
:1090B00073681B5DFB1A002B05DA2C46631C04F158
:1090C000FF35F5D1F8BD1546B368326833F8143072
:1090D000014652F824002A4618440FF0AFFCB3684A
:1090E00033F814202A4423F81420F8BD680A00201D
:1090F000104BF0B40C0A53F824706FB1FB68CEB279
:10910000013B05E07C68E45C341B002C06DA2B464E
:10911000591C03F1FF35F5D1F0BC7047BC683968C4
:1091200034F8134051F82350A41A01462819F0BC12
:109130000FF084BC680A0020044B000A53F820207A
:109140001AB9142898BF43F820107047680A002005
:1091500000232DE9F043036069B3CE68D2B206F173
:10916000804C06F100470CF1FF3C013F06F1FF3E49
:10917000B342A7EB0308AEEB0305ACEB030915D034
:109180004C680133645D141BF2D40D6855F82990C6
:10919000B9F1000F07D08D6835F818502D1B002D40
:1091A000E6DD0560A1444846BDE8F0834FF00009C4
:1091B0004846BDE8F0838946F5E700BF0023B1F5D6
:1091C000704F70B4C1F30724036028DA132C1FD941
:1091D000144D06466A68E86889B2431E02EB4002F5
:1091E00004E032F8020D081A07D52346581C03F193
:1091F000FF34F6D1002070BC7047AA68296852F885
:10920000232051F82330121A3260184470BC704782
:10921000054B8AB253F8241070BCFFF799BF18466B
:10922000E9E700BF580A0020680A002000B583B0B3
:10923000014601A8FFF7C2FF044B186008B1019B6B
:109240001844034B186003B05DF804FB282000208D
:109250002C20002070B50E4E024635681DB10D4B16
:109260001C68A54206D31446084600210FF0F1FB06
:10927000204670BD641B8442A8BF044608462246AF
:10928000294625440FF0DAFB3560204670BD00BF4B
:10929000282000202C20002070B50B4E35681DB111
:1092A0000A4B1C68A54202D30024204670BD641BF3
:1092B0008442A8BF04462846224625440FF0BEFB40
:1092C0003560204670BD00BF282000202C200020E3
:1092D000B0F5C06F16D0B0F5047F03DC0F4B5B69AF
:1092E000B3B118470E4B1B7803F07F0303F50473EB
:1092F0008342F3DB42189342F0DA10B500F036F8FF
:10930000012010BD0029E9DB064B1A78A02A01D004
:1093100000207047052201201A707047B02E0020EF
:109320007C200020080B0020024B1B6903B118476A
:1093300018467047B02E0020084B094A5B78DBB214
:10934000012B137006D0022B03D10122054B5A705A
:1093500070477047044B1B68184700BF1C0B002068
:1093600074200020080B0020B02E002008B50A4B06
:109370001B78012B0CD0022B02D10022074B5A7014
:10938000074A137803F080036FF3C713137008BD07
:10939000044B5B689847F3E774200020080B00201B
:1093A0007C200020B02E00202DE9F843254EDFF868
:1093B000A8903378244DDFF89C80244F012B06D0F1
:1093C000022B1BD06A78934238D1BDE8F883D8F8D5
:1093D000083098470446B9F1000F28D1D8F8043076
:1093E0009847D8F800309847DFF870906B7832785B
:1093F000DBB2934209D1002CE0D1E6E71A467C7833
:109400006B78E4B2DBB29342F5D0012A12D0022A83
:1094100002D100220D4B5A700D4A697813783170D1
:1094200003F080036FF3C7131370BDE8F88309F1ED
:10943000FF39DBE7074B5B689847EDE71A46012ADF
:10944000E5D1F7E7742000201C0B0020080B00205A
:109450007C200020B02E0020FF2C0100FE2C0100FB
:1094600038B5194C2378012B17D0022B0CD0174A92
:109470005278934206D0164A137803F080036FF3B4
:10948000C7131370002038BD124B104A5978527818
:10949000022AF7D000225A70EDE70F4DAB689847CB
:1094A00018B16B6898472B6898470A4B0749227890
:1094B000587849789142E5D0012A02D16B689847E3
:1094C000D9E7022AE6D0D6E7742000201C0B002042
:1094D0007C200020080B0020B02E0020A023034A8F
:1094E00013701378A02BFCD0704700BF080B00202E
:1094F000014B1878704700BF1C0B0020014BD87837
:10950000704700BF1C0B0020014BD870704700BF94
:109510001C0B002000487047200B0020014B98785E
:10952000704700BF1C0B0020014B9870704700BFB4
:109530001C0B002008B5FFF793FF08B9014B18601A
:1095400008BD00BF782000200A46F8B5094F0A4C34
:109550003B6826689B79B51803EB830103EB410355
:109560009D4200D9FFDE0146B86830440FF066FA2C
:109570002560F8BD5C0B00207820002070B50D46FA
:109580000646FFF711FF094A094C1378094963F0B1
:109590007F0365F306038D80A5681370A660FFF74F
:1095A000CBFEFFF701FFA56070BD00BF7C2000204F
:1095B0005C0B0020680B0020F0B50D46002185B043
:1095C0002E79CDE9011103919DF828C0044638B3E6
:1095D0005EB31F4E3178814224D09DF8051060089B
:1095E00060F300019DF80470C4F3800E64F38201FF
:1095F0006EF3C30162F303070A466CF307176EF3B9
:10960000041201A80C21ADF809308DF805208DF861
:109610000470FFF799FF012334702B7105B0F0BD82
:109620002EB90B4E347005B0F0BD094ED5E79DF84C
:10963000043001A862F303036CF307130C218DF8C7
:109640000430FFF781FF024E2C71347005B0F0BD7D
:10965000CA2000202DE9F04F89B099469DF85C4062
:109660009DF8603006460F46904602933CB1FFF7E6
:1096700061FF002800F0DE8009B0BDE8F08F6F4B7D
:109680001D460393FFF790FE2C600024A642CDE90F
:109690000544079440F3AC80DDF850B04FF0010A68
:1096A000674D67E037F914E0B5F9001038F9140098
:1096B000714500F0B9809DF81610159A4FEA2E2CCE
:1096C0006CF303018DF817E08DF8180012F804E030
:1096D0000012129A60F307119DF8143004F1010C86
:1096E0008DF8161032F914106CF30303FE296AF397
:1096F00007138DF81430C8BFFF239DF815C039F843
:109700001400C8BF8DF81B30139B4CF0010CADF852
:10971000190053F824006EF3410CD8BF8DF81B10CC
:109720008DF815C0C1B2C0F3072CC0F30743ACEBF2
:109730000101C3EB106399424FF04D024EDD02FB75
:1097400001F189118DF81E108DF81F300C2105A82C
:10975000FFF7FAFE37F914109BF80030298038F92A
:10976000141069800134A6422B710BF1010B05F135
:1097700006053DD09BF80030002B93D12B79002BB0
:10978000F0D0B5F900E09DF816109DF814304FEABE
:109790002E2060F30301601C60F30303B5F902009F
:1097A000159A9DF815C08DF81800001260F3071186
:1097B000105D0CF0FE0C6AF3071360F3410C8DF89A
:1097C000161005A80C218DF814308DF817E08DF8CF
:1097D00015C0FFF7B9FE9BF80030C3E702FB03F3A7
:1097E000ACEB00009B118DF81E308DF81F00ADE72B
:1097F0000222B9F814300298009212490B22FFF7A6
:10980000DBFE039B1B68002B3FF436AF0E490F486D
:109810000A78838002F07F0263F306020A70FFF782
:109820008BFD09B0BDE8F08FB5F9021081427FF4DD
:1098300042AF97E7014B039327E700BF7820002052
:1098400080200020C42000207C200020680B002005
:10985000F0B4224C82B025788DF80720854202D0E2
:1098600002B0F0BC7047FF261D4802AD076B15F82B
:10987000012DBF681B4892000361C0E902151A4B15
:109880003A81069A26701A608A7822B30B79087892
:109890004E7902FB003006F07F06144B06FB00F009
:1098A0009F6838608B795BB10022013B01EB830537
:1098B0006D89013B2A445D1CF8D102FB06023A6027
:1098C000A0230B4A13702378FF2BFCD005231370C1
:1098D00002B0F0BC70474A78D8E700BFCC20002027
:1098E000680A0020880B00201C200020580A002055
:1098F000080B0020014BDB6858817047100C0020DA
:10990000034B1879A0F10100B0FA80F040097047CC
:10991000DC20002000B583B00146202268460FF00D
:1099200069F801230099064A019802EB8102D2F8F6
:10993000051083400B43C2F8053003B05DF804FB0B
:10994000DC200020014B1878704700BF840C0020F9
:1099500070B4184A184B90601960827802B9427846
:1099600003790178457902FB013105F07F05134B3E
:1099700005FB01F19E68316083795BB10022013BF8
:1099800000EB83046489013B22445C1CF8D102FB98
:1099900005123260A024FF2309480A4A04700A49CC
:1099A000137002E00B78022B02D11378FF2BF9D051
:1099B00070BC7047780C00201C200020580A002042
:1099C000080B0020840C00201C0B00200246024BD8
:1099D0000068516803C37047D01D002000230B4965
:1099E0000B4A0C4810B4C1E90033C1E90233C2E9A3
:1099F0000033C2E90233C0E90033074C0B61136145
:109A00000381C4E90033238110BC7047401F00204C
:109A10007C1F0020D01F0020F420002009232DE906
:109A2000F04F324C85B0656824688646039530480F
:109A30000294304FDFF8C090DFF8C0A01A440091C4
:109A400037E006784FEA430C3EF91350002E36D02B
:109A500039F913B0FC5CA5EB0B0101910299884622
:109A60000399002C18BF884644460199E4B20029A6
:109A7000B8BF49428C422ADD009931F913803AF986
:109A80001310A8EB0108B8F1000FB8BFC8F1000827
:109A900044451CDD34462EF813B03AF90C500099B9
:109AA00021F81350013B591C00F8014902F1FF3223
:109AB00019D01478002CC4D1DC551478F2E7009941
:109AC00029F8135031F913502AF81350EAE7009996
:109AD00029F80C5031F913404FF00101F9542AF8DC
:109AE0000C401478DEE705B0BDE8F08FD01D0020F3
:109AF000D91F0020F4200020401F00207C1F0020E0
:109B000030B40546044C00686968AA68EB680FC465
:109B10002869206030BC7047D81D0020014B1878A0
:109B2000704700BFFE200020014B1868704700BF3F
:109B3000002100202DE9F04F6FF000444FF0000E9F
:109B4000A446F2464FF0640987B03D4ECDE90312BA
:109B50003C4ADDF84880146072680092B268019255
:109B600032690292F268059210F1FF304AD33478DC
:109B7000002CF9D033F91050009A95424CDD109A20
:109B8000019932F910208A4246DD4FF00101A246C8
:109B9000119A115458F82070C7F307215FFA87FB18
:109BA000C7F30742A1EB0B01C2EB1762013201318F
:109BB0009142B5BF09FB01F109FB02F291FBF2F200
:109BC00092FBF1F271786245BCBFA646944600292B
:109BD000CAD002998D42C7DD039951F820400499FB
:109BE000A4F50074A4B2B4F5705F51F8201018D930
:109BF00005999142B8DD4FF00101119A115410F10D
:109C0000FF30B4D2BEF1000F15D150460E4B83F891
:109C100000A007B0BDE8F08F4FF00001119A115479
:109C2000B8E7A1F5007189B2B1F5D05F9CD905996B
:109C30009142E0DC98E7034BC3F800C0E5E700BFC2
:109C4000D81D002000210020FE2000202DE9F04F2B
:109C5000C3F307461C0E8BB0A642DDF85090DDE939
:109C600017E856DC06FB09FC12B2A2EB4622029270
:109C7000621CDDB209920AB2079505926544159AF5
:109C8000C3F307276B1ED3180193169B089703EBAA
:109C90004C0C4FEA490301370693079B08998B4206
:109CA0002ADC029A019D002AB8BF5242039204E0C6
:109CB0008A0631D40133BB421ED015F8011F814200
:109CC000F6D13CF91340002CF4DD059AA2EB4321B8
:109CD00081EAE172A2EBE172DEF80010013304FBCD
:109CE0000211CEF80010D8F800200399BB4201FB06
:109CF0000422C8F80020E0D1069B01369C44019B59
:109D00004B440193029BA3F500730293099B9E426F
:109D1000C3D10BB0BDE8F08F0022159C01F00F01FC
:109D200004EB030B049341FA02F4E3070BD5094C4F
:109D3000094B145712F903A0344409FB04B414F876
:109D40000A40A04204D00132042AECD1049BB1E7BE
:109D5000049BB6E7249F01002C9F0100F0B4044649
:109D60000F46124E00F1300C354620686168A2683B
:109D7000E3681034644506F110060FC5F4D13D4682
:109D8000206861680A4F03C605F130063C46286822
:109D90006968AA68EB681035B54207F110070FC46F
:109DA000F4D12868696803C7F0BC7047042100201B
:109DB0003C2100202DE9F04F824693B01F46BDF9AB
:109DC0008C30840007939DF890308846914600219E
:109DD00022461C9806930EF03CFE22461D98002158
:109DE0000EF037FEBAF1000F64DD0024DFF8A4B1F5
:109DF00002E00134A2455DD037F91430002BF8DDC4
:109E00000025229E1E9B12A853F8243040F8245DA2
:109E100059F8242058F824100296219E04900196A7
:109E2000209E08A80390009620460895FFF70EFF95
:109E3000069B012B41D058F824005946C0F3080076
:109E4000B0F5807FC8BFC0F5007000F031FF064656
:109E500059F824004C49C0F30800B0F5807FC8BF12
:109E6000C0F5007000F024FF1D9B054653F8241038
:109E70001C9B53F8240000F0C5FEDBF82C30834215
:109E80005DDC4020064637F914C0DDE9082302FBFB
:109E900006F603FB00F34FEA8C1C96FBFCF693FBE3
:109EA000FCF31C9A42F824601D9A42F824300134D5
:109EB000A245A1D113B0BDE8F08F37F91410DDE948
:109EC000083293FBF1F392FBF1F11C9A0A9442F8E9
:109ED00024301D9BB42543F824101C9B58F82420E3
:109EE00053F8240059F82430C2F30802C3F30803DE
:109EF000B2F5807FC8BFC2F50072B3F5807FC8BFDE
:109F0000C3F50073CDE90B010D920E9300F07AFEBC
:109F10000026012104220F901C481D4BCDE90405A9
:109F200037F91450CDE90116079E009203930822D9
:109F30000AAB6420CDE91065F8F7E2FA59E7DBF8DF
:109F40002830079A37F914C09A4202DC40200646AE
:109F50009BE7C6F14003DBE90C1260460093002347
:109F600000F03AFE084B37F914C0D3E90C12C5F1E2
:109F70004003009306440023604600F02DFE37F9AD
:109F800014C0284481E700BF3C210020309F01001D
:109F9000389F0100042100202DE9F047002688B0F9
:109FA0001C1EDDE91087C8F800603E604FDD8A4660
:109FB000169D08AB43F8046D0295159D0DF1180C24
:109FC0000195149DCDE903C30095129B9146069619
:109FD000FFF73CFE1F4ECAF30800B0F5807FC8BFF4
:109FE000C0F50070314600F063FEDFF86CA0C0F1F0
:109FF0004003316BDAF834200546009320460023F5
:10A0000000F0EAFDC9F30809B9F5807FC8BFC9F5BA
:10A01000007905441049484600F04AFEDAE90C127E
:10A02000C0F14003064600932046002300F0D4FD13
:10A03000DDE90623304403FB00F302FB05F0A40135
:10A0400093FBF4F390FBF4F4C8F800403B6008B0D5
:10A05000BDE8F087042100203C210020F0B4044634
:10A06000094E00F13007354620686168A268E36850
:10A070001034BC4206F110060FC5F4D120686168A7
:10A0800003C6F0BC704700BFEC1D00202DE9F0476F
:10A09000061E1FDDDFF840A04FF064085746941EEF
:10A0A00004EB4606A1F102095D1E34F9020F3946A0
:10A0B00000F0FEFDDAF82C2039F9023F02FB00F037
:10A0C00008FB03F38342B4BF00230123B44205F825
:10A0D000013FEAD1BDE8F087EC1D00202DE9F047F3
:10A0E000061E1FDDDFF840A04FF064085746941E9F
:10A0F00004EB4606A1F102095D1E34F9020F394650
:10A1000000F0D6FDDAF8282039F9023F02FB00F012
:10A1100008FB03F38342B4BF00230123B44205F8D4
:10A12000013FEAD1BDE8F087EC1D002000283BDDAF
:10A130002DE9F043002637468C1E04EB4008951E9F
:10A1400034F902EF35F902CF7745B8BF7746664557
:10A15000B8BF66464445F3D100254FF06408A946D0
:10A16000124CD4E90CC404FB06F60CFB07F7079C61
:10A17000013C04EB000E14F8010F78B131F915C061
:10A1800008FB0CFCBC4505DB32F9150008FB00F0B0
:10A19000B04203DA84F8009003F80590A64505F173
:10A1A0000105E8D1BDE8F083704700BFEC1D002039
:10A1B000034610B4034C59689A680068DB680FC402
:10A1C00010BC7047241E002070B500242826144BB4
:10A1D000144A1548C3E90044C3E902441C61134B07
:10A1E000134D2146C2E90044C2E902441461C0E9AA
:10A1F00000443246C0E902440461C3E90044C3E9B3
:10A2000002441C610B48C5E900442C810EF021FC7E
:10A2100032462146BDE8704007480EF01ABC00BF28
:10A22000541F0020901F0020C4210020D8210020AE
:10A23000DC1F00209C210020742100202DE9F04F1C
:10A24000840004F10A0589B0824625F0070507302D
:10A2500020F0070000AFADEB050DE846ADEB000DBB
:10A2600068467D6EB961E91D21F00701ADEB010D76
:10A270007A61002152463B61C7F804803860FE6E67
:10A280000EF0E7FB2A464FF0FF3168460EF0E1FB87
:10A290002246396E4046C7F80CD00EF0CFFBBAF11B
:10A2A000000F68DD7B6D4FF0000803F1FF3B0BEB07
:10A2B0000A03FB6104E0FB6908F101089B455AD0E1
:10A2C0001BF8013F002BF6D03B6E002D53F82810F1
:10A2D000554B5B6803EB4103EDDD3A6FC7F808B0FF
:10A2E0004FF0FF3A0024A2F102099B4602E001343C
:10A2F000A5421DD039F9021F0029F8D0FB6D56F890
:10A30000241033F918E0BB6DA1EB0E0133F918C02E
:10A31000BB6E53F82400A0EB0C0000F073FC584512
:10A32000B8BFA24604F10104B8BF8346A542E1D1FB
:10A33000BAF1FF3F5B46D7F808B0BCD0FA6812F913
:10A340000A10481C65D07A6852F821008342B2DABC
:10A350004FF0010E4FF0000C42F82830FB683C68CB
:10A3600003F80A80FB6904F801C09B4504F808E083
:10A3700008F10108A4D1002D47DDD7E91CECD7E98D
:10A380001E40FB68013D1D440022AB46591ED7F814
:10A390006880F961F96911F9013FF961591C25D00B
:10A3A000D8F8001035688946B96921F813907969A1
:10A3B00094F8009021F81350BEF90050396921F843
:10A3C0001350BCF900A0B96C056821F813A0F96C12
:10A3D00001F80390396D41F82350C8F8002032602D
:10A3E000AEF80020ACF8002022700260FB6908F192
:10A3F00004085B4506F104060EF1020E0CF1020C96
:10A4000004F1010400F10400C4D12437BD46BDE8C5
:10A41000F08F01217A6842F82830FB6803F80A803F
:10A420003B6803F8081046E7241E00202DE9F04F92
:10A4300004469BB006AFD7F884500730073525F0A7
:10A440000705ADEB050D20F0070006ADADEB000DE7
:10A450000DF1180BC7E90D21584622460021FD6079
:10A460009846BB600EF0F5FA0022D7F884107A64A3
:10A47000914252DDBE4EC7F83CB006E07A6CD7F888
:10A48000843001329A427A6445DAD7F8903033F951
:10A490001230002BF2DD0023D7F8A0209C42C7E940
:10A4A00012237A6C40F35F814FF0FF3904E0FB6CBC
:10A4B0000133A342FB6420DA38F913100029F6DDDA
:10A4C000B86B796B31F9131030F91330D7F88C0071
:10A4D00050F82250D7F88800691A50F82200C01AA4
:10A4E00000F090FBBB6C0546834200F3F880FB6CE8
:10A4F0007A6C0133A342FB64DEDB4FFA89F301215E
:10A50000F8688354FB6B013203F80910D7F88430E4
:10A510007A649A42B9DBD7F83CB0002C40F3DB8078
:10A520000026013C0BEB0402D7F884303A61FA684C
:10A53000013B0BF1FF3BD318B2463B63D94604E025
:10A540003B6901364B4500F0C68019F8013F002BEE
:10A55000F6D0BB6833F91680BB6B33F916207B6BE2
:10A5600008FB02F233F91630BA6208FB03F3FB6210
:10A57000BB6F33F916B0FB6F9B5D7B62D7F8803001
:10A5800053F82600D7F88430002B40F38480FA6813
:10A59000C7F804900023013AC7F82080D7F88890C4
:10A5A00003E0396B0133914271D012F9011FB142BE
:10A5B000F7D1D7F89000D7F8801030F913C0D7F84A
:10A5C0008C0051F8264050F8230051F82310F86110
:10A5D000E0B2B861D7F894005FFA81FE30F9135009
:10A5E000F8697D613D6AFC6365443D6259F823501A
:10A5F000A846BD6A08FB0C55BD62FD6A00FB0C5500
:10A600007869FD62D7F898508344ED5C786A2843F6
:10A610007862B869704503D920466EF30700F86385
:10A62000C1F30725C4F3072CAC4503D2F86B65F3DF
:10A630000F20F863C1F30745C4F3074CAC4503D9B9
:10A64000F86B65F31740F863090EB1EB146F03D98B
:10A65000F86B61F31F60F863D7F88C1049F823A0FA
:10A6600041F823A0D7F89010F86B21F813A0D7F881
:10A67000941021F813A0D7F8981001F803A0D7F888
:10A680009C1041F823A0396B013391428DD1D7F84A
:10A690002080D7F80490BB6AFA6A93FBF8F392FB28
:10A6A000F8F2B96821F81680B96B21F816307B6B87
:10A6B00023F81620BB6F23F816B0FB6F1A4697F8E5
:10A6C00024309355D7F8803043F826003B69013693
:10A6D0004B457FF43AAF5437BD46BDE8F08F4FF499
:10A6E000317200920022334622496D2093464FF08A
:10A6F000040ABD64D7F84C900125F7F749FF40F2F2
:10A70000C5231D4A0593039229462A4607F14403AF
:10A710000496CDE9015BCDF800A06420F7F7F0FEC8
:10A7200040F2C623154A2946039205932A4607F1AB
:10A730004C03CDE9015BCDF800A004966420F7F747
:10A74000DFFE40F2C7200E4B05900393CDE9015B7D
:10A75000CDF800A004962A46294607F14803642054
:10A76000F7F7CEFEC3E64FF0FF339946C7E600BFCA
:10A77000449F0100509F01005C9F0100609F010009
:10A78000649F01002DE9F84FB0F1000840F3958077
:10A7900092469B46894600253BF91530002B40F335
:10A7A000888000244FF0FF360D9FAC4213D03BF958
:10A7B0001430002B0FDD5AF825105AF8242059F8D0
:10A7C000250059F82430891AC01A00F01BFAB84243
:10A7D000BCBF074626460134A045E6D1731C68D0AD
:10A7E0003BF9160059F826203BF9151002FB00F33F
:10A7F00059F825200C1802FB013292FBF4F249F8BB
:10A8000025205AF826305AF8252003FB00F302FBD6
:10A81000013292FBF4F20A990C9B4AF825202BF89E
:10A82000154053F8252031F8150031F816400A9FDD
:10A83000044410460B9953F82630895D27F81540DB
:10A840000B9F5FFA82FC5FFA83FE79557400B100BA
:10A85000F4453E44C2F3072CC3F3072788BF6EF3C9
:10A860000700BC4538BF67F30F20C2F3074CC3F3A2
:10A870000747BC454FEA136388BF67F31740B3EB44
:10A88000126F88BF63F31F600C9B4FF0000243F808
:10A890002500002349F801304AF801300A9B2BF8C3
:10A8A00004201A534FF0000333700C9B1A46002308
:10A8B00053500135A8457FF46FAFBDE8F88F00BF56
:10A8C0002DE9F04FB0F1000B83B0DDE910C9DDE9EF
:10A8D00016A83FDD00264FF0FF34DFF880E002E0ED
:10A8E0000136B34536D01EF806000028F8D10134F1
:10A8F00008EB040002E00134A4452BDD077805468F
:10A900000130002FF7D06445019523DA129859F8E9
:10A91000247050F8240021F8167022F816001398BD
:10A920000C9D30F914701598005D23F81670149F73
:10A9300037F9147025F816700D9D0E9FA8555AF81A
:10A9400024500198007847F826500F9DA8550136ED
:10A95000B345C8D103B0BDE8F08F00BFDC1F0020B5
:10A960002DE9F04F8FB00446894692461E460EAF41
:10A97000386CDFF818C1434D0090786CCDE9035C6A
:10A98000D7E90E23FD6ADFF808E1DFF808B101908E
:10A99000B86CD7F828800C953D6BCDE905EB796B49
:10A9A00002900A20CDE90749CDE909A6CDF82C800F
:10A9B0000D95FFF743FC344A0021D2E90232386D8D
:10A9C0000092642200F008F93B6B0A900993FB6A3D
:10A9D0008346CDE90783BB6CCDE905A602937B6C6A
:10A9E000CDE9034901933B6C796B00930A20D7E9C9
:10A9F0000E23FFF71BFD3B6D63B13B6BCDF80CB035
:10AA00000293FB6A5246CDE900834946334620460D
:10AA1000FFF7B8FED7E90F12FB6C0A20FFF736FBF1
:10AA2000E31D23F00703ADEB030D0DF1380B5B467F
:10AA3000424631462046FFF751FB3B6B796B0A9348
:10AA4000FB6ACDE906A6CDE90883FB6CCDE9044994
:10AA50000393BB6C0A2002937B6CCDF82CB001935E
:10AA60003B6C0093D7E90E23FFF72AFFFB6CFA6BD0
:10AA700000930A20D7E91013FFF758FB0437BD46AF
:10AA8000BDE8F08FDC1F0020241E0020C421002020
:10AA9000D8210020742100202DE9F04F0026013A32
:10AAA0003446174683B032468046434DDFF818B12E
:10AAB000DFF81891DFF818A10E461BE0002340F8DC
:10AAC000243038F91430002945D101202BF81430F6
:10AAD00036F91410394B2AF8141038F9141029F8E3
:10AAE000141036F91410285523F8141001320134CB
:10AAF0000A2C2CD017F8013F3148295D002BDDD1FD
:10AB00002F48DFF8B8C0DFF8CCE00029EFD050F8CC
:10AB10002410DEF800E0013140F824103CF8140065
:10AB20007145ADF8040039F814002BF81400BDF895
:10AB300004002AF81400DADD224929F814302CF830
:10AB400014302B5541F8243001340A2CD2D1104650
:10AB500003B0BDE8F08F36F914C03AF914103BF990
:10AB60001400ACEB0101181A019200F04BF838F90F
:10AB7000143039F91410DFF84CC0591A03EB610393
:10AB80000E492BF8143036F9143031F914E04CF832
:10AB90002400A3EB0E0E03EB6E032AF8143038F9F1
:10ABA0001430387829F8143036F91430019A2855C1
:10ABB00021F814309AE700BFDC1F0020901F00200E
:10ABC0009C21002074210020C4210020541F00205B
:10ABD000D8210020241E0020884210DB904210B4AF
:10ABE0000ADA441A0198521AC01A04FB00F494FBC2
:10ABF000F2F210BCD0187047019810BC704718468C
:10AC0000704700BF81EAE173A3EBE17318B300283A
:10AC1000B8BF4042F1B198421FDA820192FBF3F2D1
:10AC2000402AA8BF402211498A5CC2F15A028AB167
:10AC30000F4910B4C2F15A0431F8122031F814103F
:10AC400003FB02F300FB01F01B1403EB2043184647
:10AC500010BC70470346184670479A0192FBF0F209
:10AC6000402AA8BF402201498A5CE0E754A00100C5
:10AC700098A0010088420ADB40B1890191FBF0F005
:10AC80004028A8BF4020094B185C7047704751B15D
:10AC9000800190FBF1F14029A8BF4021034B595C92
:10ACA000C1F15A0070470846704700BF54A0010028
:10ACB00070B40E680C89022E25DDA04223DB0B4602
:10ACC0000125013E02E0844206DC15466A1C9642DC
:10ACD0009C8903F10403F6D101EB8505AE88ED886C
:10ACE000A6420DD001EB8201CB88001B5D1B00FB4F
:10ACF00005F0A41B90FBF4F41C4420B270BC704718
:10AD000028B270BC704700250122E5E77F280CDCE3
:10AD1000402824DA0F2824DC082827DA022829DB37
:10AD20000428B4BF012002207047B0F5806F08DA14
:10AD3000B0F5007F1CDAB0F5807FB4BF0720082093
:10AD40007047B0F5805F05DAB0F5006FACBF0B203F
:10AD50000A207047B0F5005F0CDA0C20704706201F
:10AD600070472028B4BF0420052070470320704797
:10AD700009207047002070472DE9F04F056889B021
:10AD80001446ADB1394D3A4F3A4E4FF480722B46CE
:10AD90000092394600226020F7F7FAFB40F20112D8
:10ADA0002B460092314622466420F7F7F1FBECE790
:10ADB000314A81461368084601338A4613600DF014
:10ADC0002DFEC9F8000020B12C4B00EB0A029A427C
:10ADD0003CD9264F0025B846DFF8B0B040F20B1240
:10ADE00043460092264900226420F7F7D1FB04264F
:10ADF000012240F20F13D9F80000114600EB0A0CB3
:10AE00000593069006ABCDE903B7CDE90155009651
:10AE10006420CDF81CC0F7F773FB01224FF4887350
:10AE200018490593CDE9025107AB114600960497E6
:10AE300001956420F7F764FB40F21112434600923B
:10AE4000214600226420F7F7A3FBC7E70E4A2B46F2
:10AE5000114602E00133322B05D051F8044B002C8F
:10AE6000F8D142F8230009B0BDE8F08FFC9F010043
:10AE700004A0010008A00100B422002030460020F8
:10AE800028A0010048A00100EC2100203CA0010006
:10AE90002DE9F04F8046006889B08946C0B12F4D3A
:10AEA00000232A4602E00133322B1DD052F8041B46
:10AEB0008142F8D1002445F823400DF0B7FD284A1F
:10AEC000C8F800401368013B136009B0BDE8F08F7B
:10AED0004FF491730A4600932249234B6420F7F7FD
:10AEE00057FB09B0BDE8F08F1F4E00243746DFF84E
:10AEF00080B0DFF880A04FF497723B4600921B4968
:10AF000000226420F7F744FB042501224FF49873D4
:10AF1000D8F80010642007910593114607ABCDE9DE
:10AF200003B6CDE901440095F7F7EAFA40F2311291
:10AF30003B460092494600226420F7F729FB4FF474
:10AF400099730A2205930095CDE903A6CDE9014442
:10AF50001146024B0020F7F7D3FACCE7EC21002092
:10AF6000B4220020A09F0100FC9F0100C09F0100AF
:10AF70004CA00100E89F0100134B1B68002B22DD51
:10AF80002DE9F041114C4FF000082746104E114DAD
:10AF900086B040F23F123B460092294600226420D0
:10AFA000F7F7F6FA01224FF4A071042305910093FC
:10AFB000CDE90364CDF8088001921146024B64206C
:10AFC000F7F79EFAE5E77047B4220020FC9F0100E6
:10AFD0006CA1010050A1010010B50446FDF7EEF987
:10AFE00004F14C0104F11400FEF7B8FE04F18400F2
:10AFF000FBF7BEFF04F59A70FBF7E2FD04F59C70C9
:10B00000FEF77EFD04F5A670FCF770FC04F5BE703B
:10B01000FFF724F804F5DA70FFF7CAF804F5E270D8
:10B02000FDF7C6F904F23D2001F09CFB04F5E57044
:10B03000FCF7FCFC94F8CA310BB9FCF7FDFC04F5F5
:10B04000E670FCF7E7FA04F50870FEF7BFFC04F5BC
:10B050000A70FDF79FF904F5107000F0D9FD002289
:10B06000014B1A6010BD00BFB81F002038B9064A56
:10B07000136801338B4205DD106001207047002307
:10B080001846014A13607047B81F002008B5FBF747
:10B090001FFEFEF7A3FCFFF797F8FCF7CDFCFCF7CB
:10B0A000C1FABDE8084001F055BB00BF0022014BCA
:10B0B0001A607047B8220020024A136801331360F7
:10B0C000704700BFB8220020014B1868704700BFCE
:10B0D000B8220020014B33F8100070477CA101001A
:10B0E00038B500240A4B0B4D21464FF42072C3E9BA
:10B0F0000044C3E902441C6107482C600DF0A9FC20
:10B100002146BDE838404FF4967204480DF0A1BCCA
:10B11000B4290020C0220020C422002044250020A1
:10B120002DE9F04F00261F460D468FB00DF118088F
:10B1300081461446314640462022CDE903660296F8
:10B14000CDF813600DF085FCBB10DFF8ECB00A2BD6
:10B15000B8BF0A23B542CBE90066CBE902665ADDE7
:10B1600002AF4FEA490AC9EBC97E009607EB050C0E
:10B17000019604EB0A024FEA4E0EB9F1000F14DDFE
:10B18000002102EB0E0030F9024B9C4207DD3E78B5
:10B1900011F80850013601353E7001F808500229B7
:10B1A00001F1010131DD9042EDD101376745524493
:10B1B000E3D1009B93BB9DF818509DF80830002602
:10B1C0003046374631460DF109020DF117040BB137
:10B1D000012630448B42C4BF19460127944202D055
:10B1E00012F8013BF3E71FBBFEB900210B460DF13E
:10B1F0001D020DB101210B44904502D018F8015FEA
:10B20000F7E779B90FB0BDE8F08F01250095019DF2
:10B2100025440195C7E733463546D0E7019BCBF877
:10B220000C30C8E7CBF80830ECE7CBF80000DCE7DF
:10B23000CBF80410D8E700BFD02900202DE9F04F4B
:10B2400095B000AFC7E90432D7E91ECED7F89430E5
:10B250000028BB61D7F89830F961D7F8B840D7E932
:10B260002C517B607862386240F37181BF4EC04BD5
:10B270003068994603EB8013786A023A4000B86060
:10B28000023B02EB000832F9020F904523F8020F4F
:10B29000F9D12368FB60FB69002B19DD3B6932683B
:10B2A000A3F102084346B348C2EB021200EB42028C
:10B2B000F869023A08EB400633F9020FB34222F86C
:10B2C000020FF9D13B6A002B40F36281A84B9946EB
:10B2D0000022C7F8B84047F6FF764C46C7F8B410CE
:10B2E000DFF8A88279697A6200234FEA420B786A14
:10B2F00004EB0B09C34439F940ABCB455344FAD1B5
:10B30000824678629C4880FB0309DB17C3EBA903E4
:10B310001BB2002B21F81230994602DD504618442A
:10B3200078629E42A8BF1E469C450CDAB5F808908C
:10B330002B6809F10109A5F8089031F91290A9EBE1
:10B340000C0A53442B60CE450CDDB5F80A906B68AF
:10B3500009F10109A5F80A9031F91290A9EB0E093B
:10B360004B446B60022A40F327813B6A01329342CF
:10B37000BADCD7E92D14FA68AE8115467F4B786A9E
:10B3800083FB0553A3EBE2732360E3683A6AFB6037
:10B39000FB6990FBF2F0002B40F3E3803B69A3F1E3
:10B3A0000208002247F6FF7C96464646714DDFF8BC
:10B3B000C881D7F8049038612846002305F5967BAC
:10B3C00030F91EAB83455344FAD188FB03A0DB1749
:10B3D000C3EBA0031BB29E45B869B8BF9E469C450F
:10B3E000A8BF9C46834226F8023F0CDD0B89086803
:10B3F00001330B817862B6F90030B869A3EB000A1B
:10B40000786A50440860994509DD4B8948680133E2
:10B410004B81B6F90030A3EB090A50444860012A79
:10B4200023EAE37002DD0E2A40F0C1806369034421
:10B430006361FB690132934205F10205BCD13869B1
:10B440000FFA8EFE0FFA8CFCBD68A1F80EC02B46D9
:10B45000083323F00703ADEB030DFB69A1F80CE003
:10B46000A3F1040C3B6A6946002B38DD7B6900269A
:10B470009A1E154440F24458A946A1F1020E32F931
:10B4800002AF256AAAEB000323EAE3731BB2AAF119
:10B49000970AAB421FFA8AFAC8BFC4E90763C245DC
:10B4A0002EF8023F06F1010602D8A3690133A36119
:10B4B0009145E4D1B1F90030002B10DDA36A3A6A5E
:10B4C0001A441046013304E031F9022F002A40F3F8
:10B4D000968098421D4603F10103F5D1A06247F61C
:10B4E000FF70FB680326984293FBFCF1B8BF184637
:10B4F0000023234AC7E90E33C7E91033C7E91233E3
:10B50000204D214BA16000B207F12801C7E90C23AF
:10B51000C7E90A65FFF7CCFBE2686369012A1146B7
:10B52000B8BF01219B0193FBF1F323EAE373984237
:10B5300009DAE369B34206DD41F287339A4202DC5D
:10B54000012384F824305437BD46BDE8F08F2368CA
:10B55000FB60FB69002B40DD3B6A044E5B00BB6077
:10B560009CE647F6FF7C4FF0000E6DE7C0220020FE
:10B57000C42200204425002067666666565555554E
:10B58000E8034000F4013200D007400044250020C9
:10B5900047F6FF72AA81FA681A4B104683FB000334
:10B5A000A3EBE2732360E3680020FB60F9E6FB682D
:10B5B0000344FB60E3603CE731F91290F868D7F888
:10B5C000B830B9F1000FA8BF48445B68F8609944EF
:10B5D000D7F8B830C3E90009C7E647F6FF70FA6943
:10B5E000084BA2F1040CFA68A88183FB0263E068AF
:10B5F000A3EBE273044A2360F860CA606FE7A562B8
:10B600006DE700BF565555550000FF7F0020F0B490
:10B61000384E8C1E186058609860D86018610431EC
:10B620001D1F34F9020F002821DD87B207F1FF3C0E
:10B63000BCF1090F11D9A7F10B0CBCF1090F1CD9F2
:10B64000A7F1150CBCF1090F1FD800EB400040001A
:10B65000A6FB0070C008033080B2A14245F8040F79
:10B66000DFD1F0BC2449DA600A791A617047002002
:10B67000A14245F8040FD4D1F3E74010053080B261
:10B68000A14245F8040FCCD1EBE7A7F11F0CBCF1A8
:10B69000090F0BD9A7F1290CBCF1090F11D8C00073
:10B6A000A6FB0070C008043880B2D6E7C0EBC0002B
:10B6B000A6FB0070A1424FEAD00045F8040FB0D1BC
:10B6C000CFE7A7F1330CBCF1090F0BD93D3F272F72
:10B6D000C3D8C0EBC0004000A6FB0070C0082638ED
:10B6E00080B2BAE700EBC000A6FB0070C0080938C2
:10B6F00080B2B2E7CDCCCCCCB429002084B08DE8A8
:10B700000F00174A0299D3782BB9462825DD1E2948
:10B7100023DD0123137013792BB96E281ADD1E293E
:10B7200018DD0123537053790BB104B0704740F218
:10B73000DC53984205DD1E2903DD012304B093701C
:10B74000704741F288330E999942F6DC002304B029
:10B750009370704700235370E5E700231370DAE716
:10B76000B429002084B02DE9F047002482B081463E
:10B770000BA880E80E00524D9DF85070DFF86C81E8
:10B78000504EDFF86CA115F8013BD3B9119B122B79
:10B7900002DCB9F1000F34D04FB34FF4CD72334611
:10B7A0000092494900224920F6F7F2FE002305F8ED
:10B7B000043C0134032CE6D102B0BDE8F04704B0EC
:10B7C000704708EB4403DB880B9A9A4202DD0D9B1D
:10B7D0001E2B3BDC40F2AD12334600925146002254
:10B7E0004920F6F7D5FE002305F8043CE1E74FF4C5
:10B7F000CF723346009235493A464920F6F7C8FEE3
:10B80000D7E740F281122F4B009231494A46492036
:10B81000F6F7BEFE129B062BCBDD002F44D1109B0A
:10B82000B3F57A7F36DD159B052B33DC139BB3F51F
:10B83000FA7F2FDA40F28D123346009225493A46BC
:10B840004920F6F7A5FE05F8047CB2E740F2A31202
:10B850001C4B0092204900224920F6F799FE012353
:10B8600005F8043C67B140F2A712334600921B4929
:10B8700000224920F6F78CFE002305F8043C98E7E7
:10B880004FF4D5723346009215493A464920F6F7EF
:10B890007FFE8EE74FF4C9723346009211490022B1
:10B8A0006420F6F775FE84E74FF4C37233460092C6
:10B8B0000D494A464920F6F76BFE05F8049C78E7E7
:10B8C000B72900203CA20100FCA2010038A301001E
:10B8D00050A20100A0A201006CA3010088A30100F6
:10B8E000B8A30100C4A2010078A201007CA101005C
:10B8F000C8A3010082B000B583B0069A0593012A5F
:10B9000023D0E8B1591001EB4301914202DCD91E6A
:10B91000032926D9023A032A12D8079A012A0FDDF1
:10B92000023B032B0CD840F2DD12134B009213495B
:10B9300000224920F6F72CFE0022114B5A709A7013
:10B9400003B05DF804EB02B07047042BD9DC40F281
:10B95000CD12094B00920B4900224920F6F718FE40
:10B96000EAE740F2D512044B009207490022492031
:10B97000F6F70EFEE0E700BF3CA201000CA20100BA
:10B98000B4290020A0A10100E0A101002DE9F043AD
:10B99000204C214FDFF88490DFF8848083B0E61CD0
:10B9A000E07814F8015BB8B9E5B163790133DBB233
:10B9B0000A2B63710BD94FF4FD73012502460093E6
:10B9C00060713B4641466420A570F6F7E1FDB44244
:10B9D000E6D103B0BDE8F08345B10023B442237241
:10B9E000DED1F6E7B4426571DAD1F2E7237A0133AA
:10B9F000DBB2282B2372EAD94FF401723B46009246
:10BA000049462A466420A570F6F7C2FDB442257265
:10BA1000C6D1DEE7B42900203CA2010004A4010045
:10BA2000F4A301002DE9F0438DB06C4614A951F840
:10BA3000389B07AE1F4690460FC986E80F001BAD26
:10BA40000FCD0FC44FF0000C95E8070084E8070005
:10BA50006C46134D17AEA5F800C085F802C096E8F5
:10BA60000F001AADFFF74AFE0FCD0FC495E80F0087
:10BA700084E80F00384696E80E00FFF773FE23AB0C
:10BA800093E80700229B8DE807004A463946404666
:10BA9000FFF730FF0DB0BDE8F043FFF777BF00BF01
:10BAA000B42900202DE9F04FA1B00025DDE93B8746
:10BAB0006E4681468A4615AC139220462C22002100
:10BAC0009B460CF0C6FFCDE90F74CDF838800DF120
:10BAD000D00C0DF11C0EBCE80F00AEE80F009CE886
:10BAE00007008EE807000DF1B40CBCE80F00C8F8A1
:10BAF0000050C8F80450C8F80850C8F80C50C8F8EE
:10BB000010503D607D60BD60FD603D610FC69CE8EA
:10BB100007002C9B86E8070051462B9A4846FFF702
:10BB20008DFB2E4B0EAF0FCB87E80F0003AE0FCC73
:10BB30000FC60FCC0FC694E8070086E807002C9CC0
:10BB4000139A02942B9C264E01942A9C5B460094E7
:10BB500051464846FFF766FF33682B9901330A2B9D
:10BB600014BF1C462C4648463D9B159A3460FFF78F
:10BB70004DFD3D9B1B4AD9683E98D37881828DF854
:10BB80005350E3B9117918465279F1B91ABBF8B993
:10BB900001224FF41A710023134C14480591CDE98A
:10BBA0000133CDE90304009211460DF153036420E3
:10BBB000F6F7A6FC9DF8530021B0BDE8F08F0120F8
:10BBC0001179034652790029E0D043F0020312B9FB
:10BBD0008DF85330DCE743F00403F9E7D029002067
:10BBE000C0220020B42900203CA20100B8A201001C
:10BBF00030B9064B187810B10138C0B218707047D0
:10BC00001423024A18461370704700BFBC2200205C
:10BC10000146982201480CF011BF00BF341E0020DD
:10BC2000014B1878704700BF7826002001464FF47A
:10BC3000707201480CF002BFF029002000487047E4
:10BC4000F02900202DE9F04FC3B0CDE9000180229A
:10BC5000002102A822AE4E9C4D9F0CF0FAFE304609
:10BC6000802200210CF0F5FE4FF0000E444BDFF86F
:10BC7000188104F1FF3993F801C093F9024008F5E7
:10BC8000707A19F8015F4046002301E0202B21D093
:10BC900030F9022FA24209DA02A951F8231002F169
:10BCA000050B59440DF1080B4BF82310944506DAA7
:10BCB00056F82310A2F1050B594446F823101F2D06
:10BCC00003F10103E2D1A242E0DA002FC8BF96449B
:10BCD000202BDDD108F14008C245D2D14FF0000839
:10BCE0004FF000406FF00044254B21AA9F88B3F924
:10BCF00006C0B3F9089001AD41AE52F8043F55F8C3
:10BD0000041F002B07DDBB4205DA8C4503DDF1453E
:10BD1000B8BF08F101088C42A8BF0C469842B8BFD2
:10BD20001846B242E9D1164A937A434503DAB2F98A
:10BD30000C30A34206DB00231846124A136043B0BE
:10BD4000BDE8F08FB2F9103000998B42F3DDB2F903
:10BD5000123001998B42EEDAD38911468342EADA36
:10BD6000084A09784F9813680144994203DD01336A
:10BD700013600020E3E7002301201360DFE700BF2A
:10BD8000341E002070260020EE290020F0B5284C3B
:10BD9000BDF91860A78BBDF91CE0B842BDF924506D
:10BDA000BDF928C003DAB4F92000984230D000224F
:10BDB000A18C8E4203DAB4F92610714521DB0020F4
:10BDC000218D8D4207DAB4F92A10614503DAE18D3D
:10BDD000089DA94226D0B4F914209A4208DA154ADF
:10BDE000A1691368994208DC002318461360F0BD6E
:10BDF0000022104B01201A60F0BD013313600120B6
:10BE0000F0BDA08D0599401AB0FA80F04009D7E73F
:10BE1000B4F91E008842CADA618C8A1AB2FA82F238
:10BE20005209C5E7002AD6D00028D8D1D3E700BFF1
:10BE3000341E0020742600202DE9F04F8BB0DDE980
:10BE40001C9607961F9E9846DDE914450896169F96
:10BE5000BDF95CC0BDF960E0DDF864A0BDF968B073
:10BE6000BDF96C309DF8806020BB19BB4146DFF8FE
:10BE70007880104698F8002009920ABB089B039628
:10BE80000293079B2246CDE900932B46FFF7DAFE8B
:10BE900088F80000099B83420FD0FDF73BFB98F820
:10BEA00000300246CBB983770E480BB0BDE8F04FA7
:10BEB000FAF786BE00220C4B1A700BB0BDE8F08F6B
:10BEC000CDE904B3CDE902EACDE9007C2B46224658
:10BED000FFF75CFF88F80000DCE701230348937755
:10BEE000E3E700BF8CC2010078260020DCC301001C
:10BEF0002DE9F843C51D25F00705CC1D24F00704E6
:10BF000000AFADEB050DEC46ADEB040D6C4690B10A
:10BF100065464FF001084FF00009013A02EB000EB0
:10BF200012F8016F01351F2E0CBF05F8019C05F8B2
:10BF3000018C7245F4D179B322464FF0010E4FF0D7
:10BF40000008013B5E1813F8015F01321F2D0CBF82
:10BF500002F8018C02F801ECB342F4D100291BDD98
:10BF60000026451ED7F820E004EB010865444FEA9F
:10BF7000400900280CDD72460CF1FF3313F8011F55
:10BF800009B1217801B916809D4202F10202F5D172
:10BF900001344445CE44ECD1BD46BDE8F88300BF32
:10BFA0002DE9F04F264F0228B7F830A0B7F932B08C
:10BFB000B7F83480B7F936604FF000093ADDCC4667
:10BFC000A1F1040E0EEB400E31F9024FA4EB08056F
:10BFD000002DC8BFAC44A41B48BFA1448E45F3D17B
:10BFE000E24527DA0120022AB7F838E0B7F93A80AB
:10BFF000B7F83CC0B7F93E504FF0000713DD3E469E
:10C00000191F01EB420233F9021FA1EB0C04002CB3
:10C01000C8BF3619491B48BF7F189A42F3D1B645AD
:10C0200001DABDE8F08FB845D4BF002000F0010070
:10C03000BDE8F08FCB45D4BF00200120D3E700BF7F
:10C04000341E0020034B1B6C9842D4BF00200120FB
:10C05000704700BF341E00202DE9F04F013883B037
:10C06000002801916CDD012872D04FF000094FF0DB
:10C07000010C09EB000303EBD3735B1032F91310CF
:10C0800032F910404500A14204DD22F813400C466D
:10C0900022F8101032F919104FEA490BA14202EBB5
:10C0A0000B0A04DD22F81940515332F9191032F904
:10C0B00013408C4205DD22F8131022F80B4032F9B0
:10C0C000134006460BF10201555E02EB4C0E22F8BE
:10C0D0001350545232F90B503EF9028F0CF1010CFF
:10C0E000A845F9DB711E02EB410301E00E46013960
:10C0F0001F4633F90249AC42F8DC8C4507DCAEF848
:10C100000040A7F800800E46BAF90050E4E7019B12
:10C1100022F80B408B423D8018DBE14616DD484596
:10C120000EDD09F1010C8445A3D102EB4909400061
:10C13000B9F90030115E8B42C4BFA9F80010135248
:10C14000019B32F9130003B0BDE8F08FB01EE6E7A3
:10C1500091460220ECE700BF2DE9F04F013800EBDB
:10C16000D07383B05B10002801936CDD012872D07E
:10C170004FF000094FF0010C09EB000303EBD37300
:10C180005B1031F9132031F910404500A24204DD63
:10C1900021F81340144621F8102031F919204FEAF4
:10C1A000490BA24201EB0B0A04DD21F819404A5366
:10C1B00031F9192031F91340944205DD21F813209B
:10C1C00021F80B4031F9134006460BF102028D5E57
:10C1D00001EB4C0E21F813508C5231F90B503EF903
:10C1E000028F0CF1010CA845F9DB721E01EB420332
:10C1F00001E01646013A1F4633F90249AC42F8DC29
:10C20000944507DCAEF80040A7F800801646BAF95E
:10C210000050E4E7019B21F80B4093423D8018DB7E
:10C22000E14616DD48450EDD09F1010C8445A3D138
:10C2300001EB49094000B9F900300A5E9342C4BFDE
:10C24000A9F800200B52019B31F9130003B0BDE89F
:10C25000F08FB01EE6E789460220ECE7831A042B34
:10C2600010B413DDDC1EB1F90430002A0B804B80C2
:10C2700031F9143008DD4000A0EB42020A440144C9
:10C2800021F8023D8A42FBD110BC70475C1E032C92
:10C2900008BF9C1EE7E700BFF0B40446049E0846B2
:10C2A000DDE90551A642DDF81CC019DD04F10044AA
:10C2B000AF1E013C07EB460705EB44058E1C06E06C
:10C2C0009C42B8BF1C46BD4226F8024F08D035F943
:10C2D000024F9442F4DD1446BD4226F8024FF6D1D7
:10C2E000F0BC6246FFF7BABFF0B400280F46DDE9A4
:10C2F0000561DDF81CC014DB013006EB40048D1C29
:10C3000006E09842B8BF1846B44225F8020F08D09C
:10C3100034F9020D9042F4DD1046B44225F8020FC4
:10C32000F6D13846F0BC6246FFF798BF2DE9F043DE
:10C33000B1F9009002284FEA4918DDE90767C2E920
:10C340000088DDE909CE21DD8C1E5B0176017F01CD
:10C35000043204EB4000023103E0A84631F9029CAC
:10C360000432B1F90050B1F9024006FB05F503FBB8
:10C370000454156802310CFB054407FB094408FB13
:10C380000E4481424FEAA4245460E6D1BDE8F08314
:10C390002DE9F041884684B04C00083404AFBD6BF1
:10C3A00024F00704ADEB040DBE690395FD6904ACF0
:10C3B0000195009602947D6BFFF76EFF3B6B214663
:10C3C0000293FB6A03950193BB6A40460093D7E949
:10C3D0000823FFF7ABFFBD46BDE8F0812DE9F04132
:10C3E000884684B04C00083404AFBD6B24F00704C9
:10C3F000ADEB040DBE690395FD6904AC0195009693
:10C4000002947D6BFFF770FF3B6B21460293FB6A42
:10C4100003950193BB6A40460093D7E90823FFF7D1
:10C4200085FFBD46BDE8F0812DE9F04F8FB00AAF22
:10C430007D6D9A461B1A023300F103088B46591989
:10C44000FB6B18EB050804461646FB6000F0AA805B
:10C450004FEA8809002934D109F10A0929F00709AE
:10C46000C7F808D0ADEB090D08953E6D0DF1280910
:10C470000796FE6C13460696BE6C5A4605967E6C71
:10C48000414604963E6C0396BE6BCDF80890CDE90C
:10C4900000A6FFF7A3FF002C0DDBFE680235013478
:10C4A00009EB850906EB440459F8043B5B1124F8B9
:10C4B000023DA642F8D1D7F808D01437BD46BDE8F2
:10C4C000F08F8B000A3323F00703C7F804D0ADEBDD
:10C4D000030D08953A6D0AAB0792FA6C09F10A0947
:10C4E0000692BA6C29F0070905927A6C04923A6CAC
:10C4F0000392BA6BCDE900A2BB605A460293334661
:10C50000FFF746FFADEB090D0895396D0DF12809D0
:10C510000791F96C33460691B96C5A460591796CCE
:10C5200020460491396C0391B96BCDF80890CDE9A0
:10C5300000A14146FFF752FF631C9A4511DDFE68DA
:10C54000BA68E91CB31E02EB810103EB4A0A06EB51
:10C55000440251F8043B5B1122F8023F5245F8D1E6
:10C56000FE60002C0DDDFE68E91C09EB810106EB85
:10C57000440251F8043B5B1122F8023D9642F8D187
:10C58000FE60BB68023559F8252053F82530134466
:10C59000FA689B1122F81430D7F804D01437BD463E
:10C5A000BDE8F08F8B000A3323F00703E946ADEBBB
:10C5B000030D08953E6D0DF128080796FE6C134695
:10C5C0000696BE6C5A4605967E6C04963E6C0396A3
:10C5D000BE6BCDF80880CDE900A6FFF7D9FE544523
:10C5E00012DAFA6804F10044013C0335931E02EBB1
:10C5F000440608EB850803EB4A0A58F8043B5B1134
:10C6000026F8023FB245F8D1CD461437BD46BDE805
:10C61000F08F00BF2DE9F04788B099464FEA4308F4
:10C6200008F1080424F0070408AFADEB040DD7E9C6
:10C630000D563C6BCDE90656BD6AFE6A059403951E
:10C640003C6A7D6A049608AECDE901650094FD6BF5
:10C65000FFF7EAFEB9F1000F10DD023CA044A6F19D
:10C66000020A34F9023F3AF9022F9B1AAB42CCBFBF
:10C670005B1B03EAE37344452380F2D1BD46BDE86A
:10C68000F08700BF1E232DE9F041264E86B00D46EF
:10C690008046009324493346642014460022F5F76F
:10C6A00077FF00274FF01F0C012204211F482B4663
:10C6B000CDF814C000910390114664200496CDE992
:10C6C0000177F5F71DFF4FF0240C0120184AA5EB68
:10C6D00008014909009003920496CDE90177434689
:10C6E000CDF814C020226420F5F70AFF294651F83E
:10C6F000043BA342FBD02B2700220124C5F11F03DA
:10C700000C481944CDE901220390049649092B46AF
:10C710000597009420226420F5F7F2FE06B0BDE8EC
:10C72000F08100BF14A4010020A4010034A4010082
:10C7300040A4010058A401000B68934209D070B5D1
:10C740000D4614460646224629463046FFF79AFF14
:10C75000F9E770470022024BC3E900221A817047B3
:10C76000F42600200278014B1A707047CC1E00207E
:10C77000314B1B78002B5AD02DE9F04F16462F4A2B
:10C7800087B08946804600242D4F1368DFF8B4B087
:10C79000DFF8B4A0013E14E03D5D38F91410022D1D
:10C7A0002BF8101005F1010E39F914109CBF5FFA37
:10C7B0008EF53D55032D2AF8101017D001340A2CA0
:10C7C0000CD04FEA440C0CEB0401C81816F8011FFA
:10C7D0000029E1D1395501340A2CF2D10133022B61
:10C7E000C8BF0023136007B0BDE8F08F0CEB040353
:10C7F0005B000BEB03010868534402901868B1F822
:10C8000004C09B88049002A928460192ADF8143018
:10C81000ADF80CC0FFF7A0FC04A928F814002846C6
:10C82000FFF79AFC019A29F814001368C6E7044A36
:10C83000C2E9003313817047CC1E0020002700207E
:10C84000F42600207C260020B8260020F0B48300C7
:10C850000A3323F00703002800AFADEB030D30DDF2
:10C860006B4600260439B20002F1804292F880C281
:10C8700092F8815292F8824292F883225FFA8CFCFD
:10C88000EDB2E4B2D2B2013683F800C05D709C70A4
:10C89000DA70BCF1000F03D00CF1FF3C83F800C04C
:10C8A0001E2D9CBF01355D700CB1013C9C700D2AA2
:10C8B0009CBF0132DA7053F8042BB04241F8042FC8
:10C8C000D1D1BD46F0BC704792F83230002B43D135
:10C8D000F0B500288BB00E460546144610DD936A6D
:10C8E00042189A4210DB00231A4684F8313094F83B
:10C8F000243093429CBF012384F830300BB0F0BD4C
:10C90000F1D1D36A8B42EEDD2C2294F83130134FF3
:10C91000013384F8313012493B46009264200022F2
:10C92000F5F736FE4FF0320C0020012104220D4BAA
:10C93000049794F83170CDE901100092039303221B
:10C94000CDF814C007AB6420CDE908650797F5F76B
:10C95000D7FD94F83120CAE7704700BF6CA40100EE
:10C9600080A40100A8A401002DE9F04F98468DB0E5
:10C97000DDE91653012DA946B8BF4FF00109012B7F
:10C980009C464FF00004B8BF4FF0010C189E09926E
:10C990003788B6F804E01268D8F8006005FB072570
:10C9A00003FB0E66002895FBF9F596FBFCF6CDE936
:10C9B0000A442ADDA446A146A246023901EB400002
:10C9C0000894CEF1000B079031F9023F5A1B22EA7E
:10C9D000E272334403EAE37397420EEB030403DC91
:10C9E0000120D21B089092445B4505DC4FF0010CFE
:10C9F000002CB8BF6442A144079B9942E4D1089B34
:10CA0000002B49D1BCF1000F49D101240026042597
:10CA10005A22244FDDF82490234B059221462246CA
:10CA2000CDE90337CDE901464B4600956420F5F783
:10CA300067FD5B201D4B224621460590039304971A
:10CA40004346CDE9014600956420F5F759FD5D2088
:10CA5000174B224621460590039304970AABCDE974
:10CA6000014600956420F5F74BFD5E20114B2246F0
:10CA70000590039304970BABCDE901460095214641
:10CA80006420F5F73DFDDDE90A23C9F80020C8F868
:10CA900000300DB0BDE8F08FCDF828A0B2E7CDF89A
:10CAA0002C90B2E76CA40100B8A40100C8A4010056
:10CAB000D8A40100ECA4010070B19A4215DC0F4A21
:10CAC0001368C72B01DC013313600D4B187808B1D4
:10CAD00081F0010019707047084B1A68C72AF4DD0D
:10CAE0001860074B0120197070470022034B1A6031
:10CAF000034B18780028EDD0EAE700BF0827002094
:10CB0000142700202DE9F04FBF48ADF2344D1093AB
:10CB1000DDF870440378CDE90E121193002C00F07B
:10CB2000B984B2AB1D460DF1A80B3C22002158463A
:10CB30000D930BF08EFF7822002128460BF089FF21
:10CB400020462946FFF782FE0123DDF87044129348
:10CB500020220F23DDF8681494AE0591DDF86C14E3
:10CB6000CDE9023204910D992046009176AA58A988
:10CB700001965B46F9F7D8FEDDF87014002940F302
:10CB8000D3845B4600200BEB410133F9022B02B149
:10CB900001308B42F9D11490012340F20A22002483
:10CBA00000939A4B05920493994B202203930F21F3
:10CBB000DDF86C346C20CDE90144F5F7A1FC2022AE
:10CBC0000F23DDF86814CDE902320591DDF86C140D
:10CBD000DDF8700404910D99019600915B4676AAE8
:10CBE00058A9FBF72DFEDDF87004A04208DD5B4676
:10CBF0000BEB400133F9022B02B101348B42F9D126
:10CC0000139420250F24DDF868340D9F0593DDF87B
:10CC10006C3476AA049358A95B4601960097CDE937
:10CC20000245FBF74DFFDDF8683458A90593DDF8A0
:10CC30006C34DDF870040493CDE90245CDE900764B
:10CC40005B4676AAFBF794FDDDF87014002940F3EB
:10CC50006F845B4600200BEB410133F9022B02B1DC
:10CC600001308B42F9D11590002440F23E2201237D
:10CC7000664905920491664900930391DDF86C348E
:10CC800020220F216C20D0AFCDE90144F5F738FC0C
:10CC90000DF56E782146782238460BF0DAFE2146F3
:10CCA000782240460BF0D5FE20210F22594BDDF8AB
:10CCB00070041D68DDF894346D78B3F9243008955C
:10CCC000DDF86854CDE903210695DDF86C5407932F
:10CCD00005950D9D5B46CDE90078029576AA58A989
:10CCE000FDF768F8DDF87034A34240F3258439ABD2
:10CCF0009A46B94645460C9355F8041B59F8040B5F
:10CD0000FDF780FFDDF870340134A3422AF8020BEE
:10CD1000F2DC0F212024DDF86804DDF894240C9D5A
:10CD2000B2F924200690DDF86C04CDE903140590D7
:10CD30000D980792019076AA184658A95B4602966C
:10CD40000095FCF749F85B4676AA58A9DDF870040F
:10CD5000FAF748F9DDF8701476AB58AA0020CDF840
:10CD600000B0F9F733FF0120DDF87014CDF800B002
:10CD700043463A46F9F72AFFDDF8700400280CDD37
:10CD80002A46662405EB4001B2F9003004FB03F3A8
:10CD90009B1222F8023B8A42F6D10D9B76AA02939F
:10CDA0000C9B58A9009318AB01935B46FCF7C2FE9D
:10CDB000FCF7B0FB0446FEF733FF002840F050813B
:10CDC000154E164A1199A379022918BF1646002B51
:10CDD00000F043815A460C99DDF87004FAF79AFD89
:10CDE00048AC254684460E4F0FCF0FC50FCF0FC559
:10CDF0000FCF0FC597E8030085E80300BCF1000FD3
:10CE000000F081830EE000BF5D1600206CA40100DD
:10CE100000A50100340A0020CCB40100D4C20100F6
:10CE2000788C010000262046FDF718F9DDF87034F3
:10CE30002660B34200F31C81012240F2BA21002592
:10CE40000420B24BB24E0090CDE9046103936D20F3
:10CE5000CDE9012511460DF58E63F5F751FBDDF89F
:10CE60007004A84239DD0C9F5E46DFF8A492DFF81B
:10CE7000B482DFF8B4A203E0DDF87004A8422CDD30
:10CE800040F2C12337F9020BB6F900C0002200932B
:10CE90004146C4E900504B464120C4F808C0F5F7AC
:10CEA00077FB36F9023B0135002BE5D040F2C32079
:10CEB000002201214FF0040C954B0590CDE903A30E
:10CEC000CDE901124120CDF800C023460322F5F739
:10CED00017FBDDF87004A842D2DCDDF8B034109EF8
:10CEE0000A93DDF85C3476AA0993DDF8643405967C
:10CEF0000893DDF8603458A90793DDF85834069399
:10CF00000F9B04930E9B03930D9B029318AB01930D
:10CF10000C9B00935B46FDF723FDDDF87024002A8F
:10CF20002FDD0025DDF85834B71EA3F10208DDF827
:10CF30005C3440F2DB2BAA46DFF8F0915E1E01E084
:10CF4000AA421EDD38F9023F37F9021F636016F866
:10CF5000013F2560A1600135002BF1D001210423A0
:10CF60006B4A0093CDE90392CDF814B00322CDE9CA
:10CF7000011A23464120F5F7C3FADDF87024AA42CE
:10CF8000E0DC0F9F0E9E3946DDF85C243046FDF74D
:10CF900083FD3946DDF85C2482463046FFF7E8FB26
:10CFA000FEF73EFE119B0025022B08BF40F001005A
:10CFB000A6F10209C3B2A7F1020BDDF85C64554F7C
:10CFC000DFF86C810D9339F9023F3BF9022F31787C
:10CFD00016932093179222600C96002900F0B480DB
:10CFE0006FF4E170A3F1E10C03444B4810F805E045
:10CFF00041F69C00844541F2D86002D8E42A00F34F
:10D000005B82834200F29A8043F2D450A2F5E67329
:10D010009BB283428CBF00230123BEF1000F00F0BE
:10D020005F82002B00F090804FF000003A4A58F8E1
:10D0300025305055AA000C92002B40F08D80364BC5
:10D040005B5D002B00F088800A233B60234620AA0A
:10D0500000212846FAF7FAFC8AE03046FCF7FEFF8A
:10D0600048AC0026DDF870342660B3427FF7E4AEAA
:10D07000DFF8C0A0DFF8C090DFF8948040F2B5225E
:10D0800043460092254900227020F5F781FA0125D8
:10D0900040F2B62204231E4921480491CDE90260E2
:10D0A000059229462A460093702023460195F5F7FC
:10D0B00027FA40F2B72002272368154905900C98FB
:10D0C000CDE903A100EB43032A46294670200195D0
:10D0D00002960097F5F714FA4FF42E7023680C4966
:10D0E0002A46CDE9039105900BEB4303CDE900758A
:10D0F000029629467020F5F703FA2368DDF87024BC
:10D100002B4493422360B9DB96E600BF38A50100AB
:10D110006CA40100182700200427002008A50100A6
:10D120005C9F010044A5010054A5010064A5010015
:10D130000C27002020A501002CA50100BEF1000F46
:10D1400002D10123C54A535558F82530AA000C9244
:10D1500013B900297FF473AF3B68092B3FF776AF13
:10D16000234620AA2846FAF771FC002800F0BC816B
:10D1700017AB317800220093284616ABFAF75EFA17
:10D1800057F8041B22681698C1F10A0302FB03FE3C
:10D1900000FB01FC179A209802FB01E200FB03C38D
:10D1A000AF4880FB02EC80FB03E0D21716F801EBDE
:10D1B000DB17C2EBAC02C3EBA003A9F80030ABF85D
:10D1C0000020BEF1000F00F01981BAF1020F00F348
:10D1D0005781A24B5B5D002B40F024810D9B002BFF
:10D1E00040F0AE81BAF1020F40F02F810C9B48F85D
:10D1F00003E0002D00F0148102250E9B5F190F9BA8
:10D200005E19DDF85C3403F1010837F9020F36F9D5
:10D2100002CF18F8011F20AB009400222090C4F820
:10D2200000C02846FAF70AFA0135209A23680A2D29
:10D230003A803380E9D1BAF1000F40F35D810025D7
:10D240002822002120A80BF004FCDDF870242560C2
:10D25000AA4249DDCDF830A040F25D3B2B46DFF815
:10D260001C92DDF864A404E0236801339342236038
:10D2700037DADDF85C14CB5C002BF5D001260027F3
:10D280004FF00408774B784A31460493CDE9027297
:10D290000196324623466D20CDF814B0CDF80080BB
:10D2A000F5F72EF940F25E302368314600966D4E58
:10D2B000424605900AEB83036D20CDE90177CDE965
:10D2C0000396F5F71DF92368DDF870245AF823104A
:10D2D000013320A8934240F82510236005F1010591
:10D2E000C7DBDDF830A0EDB240F265330127002640
:10D2F0009DF850105B4A9DF85400CDE904238DF849
:10D300005C105A4B9DF84C10CDE9016600970393D1
:10D310008DF85D1017AB39468DF85E0004226D2044
:10D320008DF85FA0F5F7ECF840F26630504A4D4BAF
:10D330003946CDE90166009704930590DDF89434F1
:10D3400003926D209A22F5F7DBF84FF45A7102220E
:10D35000484B4448CDE90176CDE90401009203939E
:10D360002022DDF868340F216D20F5F7C9F840F26E
:10D3700069323C48404BCDE9016600970490039325
:10D380000592DDF86C3420220F216D20F5F7B8F8F6
:10D3900031463E220DF591700BF05BFB202742F2E7
:10D3A0000F0C8226DDF86834214600932A4620AB14
:10D3B0000320A4F800C0A7706671FCF749FA0E9C20
:10D3C000DDF85C3401950093DDE90F52DDF8583447
:10D3D00029462046F9F7C0FCDDF85C2429462046A2
:10D3E000FCF71CFBDDF85C342A4621460A20F9F7DD
:10D3F00027FC12980DF2344DBDE8F08F0D9B0BB158
:10D40000092911DD0C9B48F803E0BAF1000F7FF405
:10D41000F0AE47F804AC48F803A0002D7FF4ECAE62
:10D420000125D0E5092969DC013147F8041CBEF16A
:10D43000000FE7D0BAF1010F3FF7D8AE074B5B5DA5
:10D44000002BDFD10D9B002BDCD157F8043C002BC7
:10D45000C4BF03F1FF3347F8043CD3E7042700209F
:10D46000676666666CA401007CA5010094A50100B6
:10D4700098A5010024B1010000A5010080A50100CC
:10D4800009293FF7B3AE013147F8041CBEF1000F84
:10D49000D0D1B7E7B2AB1D460DF1A80B3C22214617
:10D4A00058460D930BF0D5FA2846782221460BF00A
:10D4B000D0FA1294FFF74CBB834228D843F2D450E1
:10D4C000A2F5E6739BB283428CBF00230123BEF119
:10D4D000000F7FF4A6AD43F6870082427FF734AE9B
:10D4E0000122194842559CE531780246009420AB50
:10D4F0002846FAF7A3F83BE6002560E7BAF1020FE9
:10D500003FF474AE7EE73046FCF7A8FDA9E5BEF116
:10D51000000F7FF419AE43F687039A427FF714AEEB
:10D520000123094843550FE600231493FFF734BB4A
:10D5300000231593FFF798BB39AA0C92FFF7E9BBBC
:10D5400009297FF771AF75E7042700202DE9F04F17
:10D55000C7B2C0F3072883B0474501900C992BDC74
:10D560009DF806A052000AF100499DF807B009F1A4
:10D57000FF390AFB023301EB490901EB4B0C0D9912
:10D5800008F1010801EB470EDA4518D849461C4658
:10D590000C4D34F9170031F9026F8542B8BF0546CA
:10D5A0008642B8BF08808C451444F2D12DB20137B1
:10D5B00047452EF8025BE7D103B0BDE8F08F014D7F
:10D5C000F5E700BF0080FFFF2DE9F04F05468FB063
:10D5D0004FEA410A08AF18467A6088465246002151
:10D5E0006C00BB60D7F844900BF033FA2246386CDD
:10D5F00000210BF02EFA002D64DD0AF108033E6CC9
:10D6000023F0070B4FEAA8033B617B683119F960EF
:10D610009C1EC7F814D0ADEB0B0D08ABA51C18462B
:10D62000294652460BF00AFA396902464046FEF78F
:10D6300013FDB8F1000F014650DD002022460346DD
:10D6400032F902CF8C4508BF184601339845F7D10F
:10D650000522ADEB0B0D152340F23E6C4FF0290E69
:10D6600007926FF42472009508ADCDE9015306923C
:10D67000CDE903E3A1F11E02CDF814C03C314346CD
:10D68000FEF7D2FEBA68023D0AEB040134F9023F0C
:10D6900035F9020F1B1AA3EB0903002B238006DDCB
:10D6A00010889BB2184410803088034433808C4229
:10D6B00002F10202EAD1FB6802369E42D7F814D08A
:10D6C0000C46A6D100237A68C8EBC8084FEA480880
:10D6D0001C3722F80830BD46BDE8F08F6FF4247285
:10D6E0004FF0050E152340F23E6C2920ADEB0B0DDB
:10D6F000CDE9062E08AA0390019204930293A1F1AA
:10D700001E0200953C31CDF814C043460020FEF7C0
:10D710008BFE04EB0A01CEE72DE9F04F9FB08A00A3
:10D7200008AF7A61083222F00702ADEB020DB86152
:10D730004E0008A800297963B860FE6119DD4FF436
:10D74000004E47F6FF7C0025B11ED7F88420014427
:10D75000D7F88C00023A96190DF11E04023822F80F
:10D76000025FB24221F802EF20F8025F24F802CFF4
:10D77000F5D1B969786B4A0000FB02F2083222F059
:10D780000702ADEB020D08AA00297A6040F3E3809E
:10D790007A6400223A6300EBD07222F00102043B6B
:10D7A0000A32D7F88010BB6322F007033B617B6924
:10D7B0000439CB18F9603B653B69C7F82CD0ADEB59
:10D7C000030D08AAADEB030D08ABBB647B6BFA64D9
:10D7D000002B40F33981D7F890200023013A1446FA
:10D7E00047F6FF797A629046D7F88C209A46951EC4
:10D7F0007A6CC7E90F33CB46FE68D7F838E0A2F160
:10D80000020C3C620BE0FC6C4A4524F8130002DA7F
:10D8100001468146FB633A6D0133964221D056F8AA
:10D82000040F5EF8042F35F8021FC2EBA01211445A
:10D83000298018F8014F10B2E4072CF8020F49466E
:10D84000C7F854B0DFD4BC6C5A4524F81A0003DA88
:10D8500083467865C7F840A03A6D0AF1010A9642FE
:10D86000DDD1C7F828A015254FF0000B05266FF471
:10D87000247840F23E694FF0290AFA6C3C6A009223
:10D88000F86B6431CDE9066B0395CDE9015A4FF091
:10D890000042CDE90498FEF7BDFECDE902A5CDE931
:10D8A000066BCDE904980195BE6C4FF000420096DE
:10D8B000796DBB6A6431386CFEF7ACFE796B7B6ABC
:10D8C000FD6C0B44594618467B6C14F8012F02334B
:10D8D000D2074BBF35F81B2036F811200BF1010B96
:10D8E0000131844223F8022CEFD17A6CF9693B6B49
:10D8F0000A447A647969BA6B01330A44BA63BA6933
:10D900003B639A42D7F82CD07FF456AFD7E90C8905
:10D910007A68FB69A2F1020CBA6800269E4692461C
:10D920009D1E1544B9F1000F11DD29466046AAF18C
:10D93000020230F9023F31F9024F9C42B8BF0B801E
:10D9400032F9024F9C42C8BF1380AA42F1D101367E
:10D950004645F444E6D17B6B002B71DDBB68D7F8FC
:10D9600088109C1E2646FA69881ED7F88C10A2F1F2
:10D97000020CD7F81880023903EB0C0500EB020EFD
:10D9800035F8023F36F8022F9B1A20F8023F31F992
:10D99000023F704593FBF8F30B80F1D1D7F8843048
:10D9A000991E0A46BB6803EB0C0534F9023F32F9B5
:10D9B000020F002BB8BF5B42984200DA1380A542E9
:10D9C000F3D1BB68084663449C46FB690B441A4686
:10D9D0003CF9023F30F9024F002BB8BF5B429C423A
:10D9E000B8BF03809042F3D16FF00044D7F8903075
:10D9F0002646581E7B6B03449C46034604E0944233
:10DA0000A8BF14469C450AD013F8015F31F9022FD4
:10DA1000ED07F4D49642A8BF16469C45F4D1D7F83A
:10DA2000842010F8015F118815F0010FA1EB0405A7
:10DA30000ABF891B15801180834202F10202F0D1D6
:10DA40005C37BD46BDE8F08F0024152505266FF430
:10DA5000247840F23E694FF0290AFB6C204600937F
:10DA600007942346CDE90586CDE90359CDE9015A4E
:10DA70004FF0004248F26301FEF7CCFDCDE90664A9
:10DA8000CDE90498CDE902A50195BB6C2046009331
:10DA90004FF00042234648F26301FEF7BBFD24E746
:10DAA000002824DDF0B400258E1EAC464FF0FF3771
:10DAB00000E01D4636F9024F6B1C944203DD6445BD
:10DAC000C4BFA4462F469842F3D17B1C11D07B00E3
:10DAD00031F917001FB1CA1832F9022C1044AF42B5
:10DAE00003DA1944B1F902301844F0BC7047002041
:10DAF00070470020F0BC704770B40024061E1C6004
:10DB000020460EDD023901EB460631F9024F944200
:10DB100002DD1D6801351D60A042B8BF2046B1423C
:10DB2000F3D170BC704700BF2DE9F04F8246164616
:10DB30005246002589B000AF8846B86C52000021DB
:10DB4000BC6D99463B61C7F808A00AF082FF0AEB5A
:10DB5000DA7323F001030A3323F00703ADEB030D5F
:10DB6000C7F818D0AA45ADEB030D2561C7F814D04E
:10DB700025606560A560E56084F811A0257440F318
:10DB8000DB80534647F6FF7EFA6CCC46501E321FB0
:10DB900002EB8303FB60BB6C3860AB467146786078
:10DBA0008246A8F10408A3F10209FD61BC6511E0F9
:10DBB0007345A8BF7346D7E9064524F81500A8BFEA
:10DBC0001846FC698646F86801349042FC610CF105
:10DBD000010C31D0386952F8043F20B19CF80000A4
:10DBE00000FB0333DB1158F8040F3D6DC3EBA013AA
:10DBF00047F6FF708342A8BF034652480E46834251
:10DC0000B8BF034618B229F8020F1AF8014F2C5773
:10DC1000002CCDD18B42A8BF0B467C691E4624F850
:10DC20001B00A8BF18460146F868734690420BF1E6
:10DC3000010B0CF1010CCDD1D7E916429342A8BFDC
:10DC400013469642A8BF16460FFA83FB534236B2DC
:10DC50009B45B8BF9B469E42B8BF1E46BA683B680C
:10DC60004FF0000C13449A464FF000407B6D3E612C
:10DC7000C7F80CB0E046D3E900E662466FF0004515
:10DC8000D3467968F861D7F848903CE0BB69F868FA
:10DC900033F8183008F101081B1A1BB229F81230AA
:10DCA000734518DDB4F808A023680AF1010AA4F846
:10DCB00008A039F912A094F91100AAEB0E0A5344F6
:10DCC000236094F910309042C8BF62749342B8BF89
:10DCD000227439F912309E420ADD6389606801338B
:10DCE000638139F91230A3EB060A8244C4F804A018
:10DCF000F86901329842B8BF18469D42A8BF1D4638
:10DD00008B45F86110D011F8013F386DC356002BD8
:10DD1000BCD17B69386933F81C300CF1010C1B1A3B
:10DD20001BB229F81230BBE72BB205B22437A5810C
:10DD3000E381BD46BDE8F08F4FF0FF334FF0004068
:10DD4000F4E700BF0080FFFF2DE9F04786B0824670
:10DD5000DDE9129816461C460D46149FF4F796F816
:10DD60001423159A0397CDE90423D0F801300F98B6
:10DD7000153332462946CDE9010300940E9B5046E7
:10DD8000FFF7D2FE00254FF02E0C01210227184884
:10DD9000184E2346CDE9030652466920CDF814C03B
:10DDA000CDE901150097F4F7ABFBAA4528460FDD36
:10DDB000A31E03EB4A0A33F9021FA1EB0902002A52
:10DDC000C8BFAD18B1EB080148BF40185345F2D1A8
:10DDD000109BAB4207DB119B8342D4BF0020012084
:10DDE00006B0BDE8F087012006B0BDE8F08700BFAF
:10DDF00024B10100B0A50100002820DDF0B48E1E82
:10DE000006EB4006B14218D0571C38460B46B1F914
:10DE1000004033F9025FAC4207DD0D801C8092F9AF
:10DE2000004090F9005015700470B34200F10100F9
:10DE3000EDD10231B1423A46E6D1F0BC70477047AD
:10DE40002DE9F04F8046450005F1080485B000EB50
:10DE5000D07A24F0070407302AF0010A00AF20F03E
:10DE60000700ADEB040D08F1090424F00704EB46AC
:10DE7000ADEB000D0AF10A0020F007006E46ADEB95
:10DE8000040D6C46ADEB000DE946C7E902210AF12D
:10DE9000020A08F102021F2120467B600AF0D9FD28
:10DEA0005246484600210AF0D4FDB8F1000F7B68C5
:10DEB00007DD324606EB0800911B02F8011B824287
:10DEC000FAD14FF0FF3A2A46F96858467B600AF0CB
:10DED000B5FD594632464046FFF78EFF023D08F138
:10DEE000FF3E7B6806EB0E01AB44013EB14218D009
:10DEF0003BF9025911F901299D4202F1010C10DB95
:10DF0000A05C22441F28927860D01E2860D81E2A68
:10DF100096BF4FF0FF3204F80C0004F80C20B14219
:10DF2000E6D1B8F1020F04F1010113DD0B46FF2029
:10DF3000A64402E0013373450CD05A781F2AF9D168
:10DF40001A781E2AF6D89A7801331E2A98BF1870BC
:10DF50007345F2D1B8F1000F2EDDFB6804EB080623
:10DF6000F96004E00134A64203F1020323D0627891
:10DF7000FF2AF7D1257894F802C039F8150039F84E
:10DF80001CE08346704528BFF346B3F90020B96B07
:10DF90000A449345E6DA704538BF7046013465455A
:10DFA0008CBF29F81C0029F81500A6420AF1FF3A97
:10DFB00003F10203DBD1F9684246B8680AF03EFD7E
:10DFC0000AF101001437BD46BDE8F08F1F2A06D0C4
:10DFD0001E2A88BF6FF0690204F80C2086E70AF158
:10DFE000010A04F80CA029F81A507FE7FFF728BFB0
:10DFF0000048704798080020014B036020207047BC
:10E00000D0A50100014B03600F207047F0A501006F
:10E01000014B03600F207047C0A5010030B44FF0E2
:10E02000804300220E211F2020250F2483F8082181
:10E0300083F80A2183F8090183F80B111A739A7384
:10E040005873D9731D725C72DA7793F8211041F01E
:10E05000010183F8211093F8211062F3410183F844
:10E06000211030BC704700BF10B44FF0804485B021
:10E070000DF1100C0CE90F00BDF800302382BDF843
:10E0800002306382BDF90430A382BDF90630E38219
:10E09000BDF808302383BDF80A306383BDF80C3027
:10E0A000A38305B010BC70474FF08043988370473E
:10E0B0004FF08043988B70474FF0804383F82000E7
:10E0C000704700BF0123002110B50A4A0A4C23778C
:10E0D000917210B94FF08042D3704FF0804301220B
:10E0E000987000211A700A2000F094F90022024B67
:10E0F0001A7710BD202700200000105001234FF098
:10E100008040102110B4034A034CA372436010BC3A
:10E1100011607047A40C00202027002001234FF03D
:10E120008040102110B4044A044C6372C0F80431DA
:10E1300010BC1160704700BFA40C002020270020F5
:10E14000E022002101480AF084BC00BF80010040A9
:10E150002DE9F04105461F4B1F4886B06A1E13F893
:10E16000011B834202F8011FF9D101242B464FF015
:10E17000A90C002702262868184AC11782FB00E272
:10E18000DFF8648002441648C1EB222243F8242BB6
:10E190002146CDF814C02246CDE90308CDE9014758
:10E1A00000966220F4F7ACF94FF0AA0C0D48CDF8B8
:10E1B00010800390CDE90147009605F12603224621
:10E1C0002146CDF814C06220F4F79AF906B0BDE8F4
:10E1D000F08100BF280000405400004089888888F2
:10E1E00074C6010004A6010000A6010070B5E0227B
:10E1F000064600210B480AF02CFC002401234FF0B6
:10E200008042094D09492B770A208C729370214670
:10E21000137000F0FFF82C773046BDE87040FFF730
:10E2200097BF00BF80010040000010502027002051
:10E2300010B50446FFF78CFF2E234FF0804004F109
:10E240004E0203F1600150F82110013B1F2B22F810
:10E25000021DF6D14FF0804004F1960203F16001F7
:10E2600050F82110013B22F8021D591CF6D110BDB7
:10E270004FF0804270B5037909B201FB03F1948B32
:10E280008B11A342B8BF2346012500240221068832
:10E290009BB24380A2F80C61A2F80E31074E084BE6
:10E2A000357709205C7282F8035182F80211214609
:10E2B000A2F8005100F0AEF8347770BD00001050A5
:10E2C000202700204FF0804393F81401704700BFCF
:10E2D0004FF0804393F81701704700BF0023094AAD
:10E2E00082F832305064916472B6012382F8403073
:10E2F00000BFB2F852309BB2002BFAD062B6B2F82F
:10E3000050007047000010502DE9F04750221020B7
:10E31000202130244FF0400A4FF060094FF00108EF
:10E320004FF4807E4FF4007C4FF480674FF400661A
:10E330000825104B83F8040383F8081383F800437F
:10E3400083F8034383F805A383F8092383F80A239A
:10E3500083F80B2383F80F93C3F8008018601960CB
:10E36000C3F800E0C3F800C01F601E601D60BDE878
:10E37000F08700BF00E100E04FF40042034BC3F818
:10E380008020BFF34F8FBFF36F8F704700E100E035
:10E3900000220121034BA3F86E20A3F86A20A3F802
:10E3A000681070470000105010B5174C84B094E806
:10E3B0000300029002A88DF80C1000F061F800F044
:10E3C00069F8FFF7A1FF62B600F014FAA36804A889
:10E3D00040F80C3D00F008FA00F050FA00F05EF949
:10E3E00000F0C0FA094B1A6922F004021A61BFF367
:10E3F0004F8F0721064A82F824105A6942F0100212
:10E400005A6104B010BD00BFB08C010000ED00E007
:10E410000000105008B500BF72B6084A135C3BB943
:10E4200000BF30BF62B600BF72B6135C002BF7D0DE
:10E430000023135401B1884762B608BD202700208D
:10E4400000200A4B0A4913F8012B10448B42C0B23A
:10E45000F9D1064B1A78AA2A01D000207047DB7B3D
:10E46000181AB0FA80F04009704700BF80004000E1
:10E470008F0040004FF0A04301225A74704700BF44
:10E480000246034B0068127918601A71704700BF8A
:10E490003027002070B5FFF7D3FF01220021334B56
:10E4A000D9705A72DA7200285CD0314AD278D2B26E
:10E4B0001A72002201242F492C4B8D789A725A73BC
:10E4C0001D734D780E781E751D77CD78097983F808
:10E4D000215083F820105A749A741C749A7018B3DF
:10E4E000234A51781A78C9B2D2B28A4208D08A42F5
:10E4F000B4BF013202F1FF32D0B28A421870F6D1B5
:10E500001B4B1A491A794B78D2B2DBB29A420AD025
:10E510009A4203F1010096BF03F1FF33C3B2DBB2AD
:10E520009A424B70F4D170BD1A78D2B2B02A08D09A
:10E53000AF2AD4BF013202F1FF32D1B2B02A197032
:10E54000F6D10A4A5378DBB2082BECD0072B03F143
:10E5500001018ABF03F1FF33CBB2DBB2082B53704A
:10E56000F4D1E0E7E0221A72A3E700BF00001050E8
:10E57000800040003027002007490B78DBB283423F
:10E5800008D09842CCBF013303F1FF33DAB28342A3
:10E590000A70F6D1704700BF0000105008B5FFF7B1
:10E5A0004FFF18B1024B5878C0B208BDB02008BD6B
:10E5B00080004000014B1878704700BF00001050E9
:10E5C000084A5378DBB283420AD0984203F1010132
:10E5D00096BF03F1FF33CBB2DBB283425370F4D169
:10E5E000704700BF00001050014B5878704700BFC3
:10E5F0000000105010B50446FFF73CFF4FF0A04359
:10E6000020686168A26807C310BD00BF38B54FF02D
:10E61000A044E37DDBB2042B28D0082B19D0022BB9
:10E6200009D00123184A137000BF4FF0A0421373A2
:10E6300000BF537338BD154D15496079FAF72CFEAC
:10E6400061792868FAF770FE62792B6813442B60B1
:10E65000E7E7104BD0E9051259609A60236A5BBA6C
:10E660000A4A18461360FAF7E1FDDAE7074D0A494E
:10E670002079FAF7EFFD21792868FAF729FE227947
:10E680002B6813442B60CCE720270020382700207C
:10E69000200000503420002024000050274B00228E
:10E6A000D3F8801041F00101C3F88010196C21F0FB
:10E6B00001011964196841F001011960D3F8801053
:10E6C00021F00201C3F88010196C21F002011964D5
:10E6D000196841F002011960D3F8801041F010016F
:10E6E000C3F88010196C41F010011964196841F0E9
:10E6F00010011960D3F8801021F02001C3F88010B8
:10E70000196C21F020011964196841F02001196089
:10E71000D3F8801021F04001C3F88010196C21F06B
:10E7200040011964196841F040011960C3F80821DB
:10E73000C3F80421C3F80021704700BF0000025055
:10E74000034BD3F8C03018420CBF012000207047A3
:10E750000000025038B54FF040540125642084F881
:10E76000245000F0D1F900F07FF900234FF47A70C3
:10E7700084F8253084F8815000F0C6F9BDE83840AF
:10E7800000F072B910B501234FF04054642084F8B2
:10E79000253000F0B9F900F067F9002384F824303F
:10E7A00084F8813010BD00BF14200122002130B553
:10E7B0000A4D89B02D780A4C05900A4808AB03F839
:10E7C000015DCDE90111CDE90304009211466420F9
:10E7D000F3F796FE9DF81F0009B030BDB70040006A
:10E7E00018A6010020A601000268014B1A607047BC
:10E7F0003C27002038B5FFF723FE0F23F0B94FF078
:10E8000040524FF00104D9B2013B072B82F82B1084
:10E8100082F8284082F82800F5D1042382F82F30AE
:10E820004FF040530121002283F8281083F828205C
:10E830004FF47A70BDE8384000F0F6B94FF040511F
:10E84000012500240C4806E081F82B20013B81F8CB
:10E85000285081F82840027A0E2A8EBF0F22027AB1
:10E86000D2B29342DAB2EFDA4FF04052024B5B7A07
:10E87000DBB282F82F30D3E780004000F8B5FFF715
:10E88000DFFD4FF0405401250026074684F825603F
:10E890004FF47A7084F8205084F8275000F0C4F9BF
:10E8A000642084F8255000F0BFF984F824506420D7
:10E8B00000F0BAF984F8256007BB06231C4D84F8E4
:10E8C0002730EB7884F826302B7884F842304FF0EC
:10E8D000405401230022697840F24C4084F84610ED
:10E8E00084F8442084F8453084F8413084F840307E
:10E8F00000F09AF9AB7884F84430F8BDFFF754FF84
:10E900000C4B9B7A88B94FF04052DBB2084D84F82B
:10E910002730E978074B82F82610DB7A29780B44F8
:10E920000B3BDBB282F84230D1E7053BEBE700BF9F
:10E930003C2700208000400020B9064A064B1060AA
:10E940001860704703490548034B054A08601A6080
:10E95000704700BF442700204027002055E70000F3
:10E9600085E700004FF04053F0B406240122002553
:10E970000A26FF2083F8D64093F8D7100F2764F3B8
:10E98000030183F8D710042183F8D86083F840216D
:10E9900083F8D00083F87F5093F88C004FF0050C7B
:10E9A000104383F88C0093F88C00072640F0020097
:10E9B00083F88C0093F8910064F30300032483F838
:10E9C000910083F8901083F88D1083F8A02093F8BD
:10E9D000A10065F3010083F8A10083F8947093F817
:10E9E0008800104383F8880093F88900104383F867
:10E9F000890083F8F12083F8874083F88E4083F8FC
:10EA0000D22083F8D52083F8ABC083F8AD5083F8CB
:10EA1000AC4083F8AE1083F8AF1093F88B1041F040
:10EA2000700183F88B1083F8936083F8B020F0BCFA
:10EA3000704700BF00220521034B04481A6058604C
:10EA40009A601960704700BF10E000E0FFFF0F0000
:10EA50000022044B98681A60C0F57F2000F6FF7012
:10EA6000704700BF10E000E0002382B0002801934F
:10EA7000B8BF0730019BC010984206DD00BF019B64
:10EA800001330193019B8342F8DB02B0704700BF62
:10EA9000054A0649937CD27801335B00934000FB22
:10EAA00003F091FBF0F070470000105000B4C40474
:10EAB000054A937AD27ADBB20AB101339840034B0C
:10EAC00093FBF0F0704700BF0000105040420F0071
:10EAD000054A937AD27ADBB22AB10122134402FAB0
:10EAE00003F390FBF3F0704700001050054A00EB71
:10EAF0008000937CD27801335B009340000190FB4F
:10EB0000F3F0704700001050124B00EB80001B7BAD
:10EB10000001DBB25A1E062A0DD9082B12D0092B90
:10EB200015D0A3F10B02032A0ED90F2B0CBF012322
:10EB30004FF0FF3300E00133064AD278934090FB58
:10EB4000F3F070470A23F7E7063B9B00F4E70C233A
:10EB5000F2E700BF00001050034B044A5B7C03F057
:10EB6000010352F823301847000010502CA6010072
:10EB7000034B044A5B7C03F0010352F8233018472F
:10EB80000000105024A6010008B5044B1868FFF7D8
:10EB9000EFFFBDE8084000F0A1B800BF4C270020FF
:10EBA00038B50C4B054693FBF1F00C46FFF7ACFF74
:10EBB0003A2303FB04F39B1103FB00F090FBF5F0F9
:10EBC000834203DB462404FB00F4A411024B1C60C7
:10EBD00038BD00BF40420F004C27002070B5012215
:10EBE00000244521042688B008AB43F8040D0B4DE2
:10EBF0000B48CDE901240591CDE9030511460096A6
:10EC00006420F3F77DFC074B07985C7100F042F835
:10EC100021460520FFF7FEFB08B070BD34A60100B9
:10EC20003CA601002027002008B5FFF795FFBDE8AE
:10EC30000840FFF7D3BF00BF08B5044B1860FFF7CB
:10EC400097FFBDE8084000F00DB800BF4C2700203A
:10EC5000002000F049B800BF012000F045B800BF17
:10EC600000F030B8012830B44FF000024FF0020439
:10EC700038BF01200121054B054D1A702A719C7087
:10EC80009860DA605A70197030BC70470000085004
:10EC90002027002001284FF000024FF0010138BF6B
:10ECA000012010B4054B064C1A706271997098607F
:10ECB000DA605A70197010BC704700BF000009502C
:10ECC00020270020012000220249034B08711A70FE
:10ECD000704700BF2027002000000850014B9860BB
:10ECE000704700BF0000085010B40B4A0B4983B0B6
:10ECF000CDE9001202AB03EB800353F8082C9378A4
:10ED0000DBB2012B04D10021054C043023541170D7
:10ED100003B010BC704700BF00000950000008504D
:10ED200020270020034AD2F8803023F00103C2F8E4
:10ED30008030704700000250034AD2F8803043F020
:10ED40000103C2F88030704700000250034BD3F833
:10ED50008000C04300F00100704700BF0000025077
:10ED6000002822DDF0B5DCF80460002496F80EE0FF
:10ED70000CE0DCF800703F5D07FB033305FB03F399
:10ED80005B1242F824300134A0420DD051F8043B0C
:10ED9000356ABEF1000FECD103FB05F39B1042F87E
:10EDA00024300134A042F1D1F0BD7047002822DDAB
:10EDB000F0B5DCF80460002496F80EE00CE0DCF816
:10EDC00000703F5D07FB033305FB03F35B1242F862
:10EDD00024300134A0420DD051F8043B356ABEF115
:10EDE000000FECD103FB05F39B1042F824300134F3
:10EDF000A042F1D1F0BD7047002822DDF0B5DCF86B
:10EE00000460002496F80EE00CE0DCF800703F5D32
:10EE100007FB033305FB03F35B1242F82430013494
:10EE2000A0420DD051F8043B356ABEF1000FECD181
:10EE300003FB05F39B1042F824300134A042F1D1CA
:10EE4000F0BD7047002822DDF0B5DCF80460002436
:10EE500096F80EE00CE0DCF800703F5D07FB033332
:10EE600005FB03F35B1242F824300134A0420DD0BD
:10EE700051F8043B356ABEF1000FECD103FB05F3FA
:10EE80009B1042F824300134A042F1D1F0BD70470C
:10EE9000DCF80830F0B49C7BBCB9002813DDDCF84A
:10EEA0000430D3F80D301B681E89DD8851F8043B0F
:10EEB000013403FB06F393FBF5F3A0424FEA8313FF
:10EEC00042F8043BF2D1F0BC70470028FBDDDCE9DE
:10EED0000043D3F80D30013C1B6820441F89DE88B5
:10EEE00014F8015F51F8043BA04205FB033307FB14
:10EEF00003F393FBF6F34FEA630342F8043BEFD1CD
:10EF0000F0BC7047704700BF00280BDD10B4002430
:10EF100051F8043B01349B01A04242F8043BF7D175
:10EF200010BC7047704700BF00232DE9F041DCF8AA
:10EF30000C5088B00793D5F809200028644617685C
:10EF40000EDDDCF80820D2681618013E013A12F8EE
:10EF5000011F795C96420B440793F8D193FBF0F3C1
:10EF6000606807934288002A53D00689921B1102D9
:10EF70009B1B91FBF3F3B3F5DC7FA8BF4FF4DC736D
:10EF80000362D5F80D504FF0020E2989002603FBCD
:10EF900001F31912FF29A8BFFF2101224FF0AB088E
:10EFA0001E4FDFF884C0698100EB0E03CDF800E04E
:10EFB000CDE903C71146CDF81480CDE90166642080
:10EFC000F3F79EFA01254FF00408AC22144B05928A
:10EFD00029462A460393049707AB02960195CDF87C
:10EFE00000806420F3F78CFA4FF0AD0C63680D4895
:10EFF00004970390CDE90156CDF8008020332A46CE
:10F000002946CDF814C06420F3F77AFA08B0BDE8B9
:10F01000F0814FF480730362B3E700BF40A60100A4
:10F0200068A6010070A601004CA6010000232DE98E
:10F03000F041DCF80C5088B00793D5F8092000287F
:10F04000644617680EDDDCF80820D2681618013E09
:10F05000013A12F8011F795C96420B440793F8D1EC
:10F0600093FBF0F360680793C288002A52D0868829
:10F07000921B11029B1B91FBF3F3B3F5DC7FA8BF3E
:10F080004FF4DC730362D5F80D504FF0020E29895E
:10F09000002603FB01F31912FF29A8BFFF2101225B
:10F0A0004FF0F4081D4FDFF880C06981831DCDF853
:10F0B00000E0CDE903C71146CDF81480CDE9016623
:10F0C0006420F3F71DFA01254FF00408F522144BD4
:10F0D000059229462A460393049707AB02960195A9
:10F0E000CDF800806420F3F70BFA4FF0F60C63685C
:10F0F0000C4804970390CDE90156CDF800802033E9
:10F100002A462946CDF814C06420F3F7F9F908B06F
:10F11000BDE8F0814FF480730362B4E740A60100BC
:10F1200068A6010070A601007CA6010000232DE95D
:10F13000F041DCF80C5088B00793D5F8092000287E
:10F14000644617680EDDDCF80820D2681618013E08
:10F15000013A12F8011F795C96420B440793F8D1EB
:10F1600093FBF0F3606807934288002A54D0068925
:10F17000921B11029B1B91FBF3F3B3F5DC7FA8BF3D
:10F180004FF4DC730362D5F80D504FF0020E29895D
:10F19000002603FB01F31912FF29A8BFFF2101225A
:10F1A0004FF4C5781E4FDFF884C0698100EB0E0371
:10F1B000CDF800E0CDE903C71146CDF81480CDE9C4
:10F1C00001666420F3F79CF901254FF0040840F232
:10F1D0008B12144B059229462A460393049707ABDA
:10F1E00002960195CDF800806420F3F789F94FF479
:10F1F000C67C63680C4804970390CDE90156CDF8AE
:10F20000008020332A462946CDF814C06420F3F745
:10F2100077F908B0BDE8F0814FF480730362B2E77C
:10F2200040A6010068A6010070A601004CA60100DE
:10F2300000232DE9F041DCF80C5088B00793D5F895
:10F2400009200028644617680EDDDCF80820D26823
:10F250001618013E013A12F8011F795C96420B44E0
:10F260000793F8D193FBF0F360680793C288002AF4
:10F2700053D08688921B11029B1B91FBF3F3B3F5CD
:10F28000DC7FA8BF4FF4DC730362D5F80D504FF05C
:10F29000020E2989002603FB01F31912FF29A8BFDA
:10F2A000FF21012240F2D3181E4FDFF884C069818C
:10F2B000831DCDF800E0CDE903C71146CDF81480D9
:10F2C000CDE901666420F3F71BF901254FF004082E
:10F2D0004FF4EA72144B059229462A460393049789
:10F2E00007AB02960195CDF800806420F3F708F98A
:10F2F00040F2D51C63680D4804970390CDE9015690
:10F30000CDF8008020332A462946CDF814C0642069
:10F31000F3F7F6F808B0BDE8F0814FF480730362AC
:10F32000B3E700BF40A6010068A6010070A6010077
:10F330007CA6010000232DE9F0411C46DCF80C20DE
:10F3400088B0D2F809206646D76801F5F06501F566
:10F35000006C0793043F57F8041FA5F5F062890974
:10F3600052F8803B5B1A95421C44F9D10435AC45F8
:10F370000794F0D194FBF0F4B36807945A88002AFC
:10F3800054D09988521A1202641A92FBF4F4B4F51C
:10F39000DC7FA8BF4FF4DC741C62726840F23A2E26
:10F3A000D2F80D204FF0020C10680025C188012210
:10F3B00004FB01F42112FF29A8BFFF211D4F1E4CA1
:10F3C00001816344CDF814E0CDF800C01146CDE9C9
:10F3D0000347CDE901556420F3F792F801244FF07B
:10F3E000040840F23B22154B059221462246039326
:10F3F000049707AB02950194CDF800806420F3F7E1
:10F400007FF84FF40F7CB3680D4804970390CDE963
:10F410000145CDF80080203322462146CDF814C0A6
:10F420006420F3F76DF808B0BDE8F0814FF4807404
:10F430001C62B2E740A6010098A60100BCA601002C
:10F44000C8A6010030B595B0202200210CA809F013
:10F4500000FB294C29492A4D2A48CDE90854CDE919
:10F460000A01294A294B0E9293F8812002AC8DF8AB
:10F470003C2093F881308DF83D30F6F7CBFF8DF8C6
:10F480003E00F6F7CDFF8DF83F00F6F7CFFF8DF881
:10F490004000F6F7D1FF8DF84100F6F7D3FF8DF865
:10F4A0004200F6F7D5FF1190F6F7D8FF1290F6F765
:10F4B000DBFFADF84C0008A8F9F7B2FDF6F7D4FF72
:10F4C000FAF718FA0023022202930120A382C4E96A
:10F4D0000133C4E903338DF81D20FBF7FBFD06ABB8
:10F4E000ADF81E0093E803008DE8030094E80F00D8
:10F4F000F9F740FD15B030BD39ED000029EC0000F2
:10F5000025ED00004DED00006E0016780000105053
:10F5100070B5002301223F2148260825022484B02B
:10F5200001A8CDE9013303938DF807608DF80850E9
:10F530008DF809208DF80F208DF80A408DF80D10F8
:10F54000FFF758F804B070BD02FB01F21212FF2A57
:10F55000A8BFFF22028070472DE9F042224E92B0F0
:10F56000224D0DAC05AF99460691089296E80F0022
:10F5700084E80F0018ABC4E90275204611A9119365
:10F58000F0F77EFE96E80F00194E09AD85E80F00F2
:10F59000C5E9027621462846F0F772FE089B069AD6
:10F5A00044F001041169D3F8012005910792D3F8C2
:10F5B0000D2010491089189E5081CDE9021445F0A4
:10F5C000010501960495D3F8093080225B6900217A
:10F5D000184609F03EFA2022034601A94846F6F7EC
:10F5E00049FF12B0BDE8F082BC8C010029EF000099
:10F5F00061ED0000295800002DE9F042224E92B042
:10F60000224D0DAC05AF99460691089296E80F0081
:10F6100084E80F0018ABC4E90275204611A91193C4
:10F62000F0F72EFE96E80F00194E09AD85E80F00A1
:10F63000C5E9027621462846F0F722FE089B069A85
:10F6400044F001041169D3F8012005910792D3F821
:10F650000D2010491089189E5081CDE9021445F003
:10F66000010501960495D3F809303C225B6900211D
:10F67000184609F0EEF90F22034601A94846F6F7AD
:10F68000F9FE12B0BDE8F082BC8C01002DF0000044
:10F69000ADED00008D5800002DE9F042224E92B0F1
:10F6A000224D0DAC05AF99460691089296E80F00E1
:10F6B00084E80F0018ABC4E90275204611A9119324
:10F6C000F0F7DEFD96E80F00194E09AD85E80F0052
:10F6D000C5E9027621462846F0F7D2FD089B069A36
:10F6E00044F001041169D3F8012005910792D3F881
:10F6F0000D2010491089189E5081CDE9021445F063
:10F70000010501960495D3F8093080225B69002138
:10F71000184609F09EF92022034601A94846F6F74B
:10F72000A9FE12B0BDE8F082BC8C01002DF10000F2
:10F73000F9ED0000415800002DE9F042224E92B050
:10F74000224D0DAC05AF99460691089296E80F0040
:10F7500084E80F0018ABC4E90275204611A9119383
:10F76000F0F78EFD96E80F00194E09AD85E80F0001
:10F77000C5E9027621462846F0F782FD089B069AE5
:10F7800044F001041169D3F8012005910792D3F8E0
:10F790000D2010491089189E5081CDE9021445F0C2
:10F7A000010501960495D3F809303C225B690021DC
:10F7B000184609F04EF90F22034601A94846F6F70C
:10F7C00059FE12B0BDE8F082BC8C010031F200009D
:10F7D00045EE0000E95800000269054B0548013A72
:10F7E00012F8011F013303F8011C8342F8D170475E
:10F7F00000008360E00183602DE9F041234E92B068
:10F80000234D0DAC05AF9846CDE90610089296E859
:10F810000F0084E80F0018ABC4E90275204611A957
:10F820001193F0F72DFD96E80F001A4E09AD85E80B
:10F830000F00C5E9027621462846F0F721FD069B18
:10F840004FF4F062D3F8093000211B69124F1846BB
:10F8500009F0FFF8DDE906210969104E0591D2F89B
:10F860000D200346126844F00104D18845F00105DB
:10F87000118140464FF4F07201A9CDE90345CDE96D
:10F880000176F6F7F7FD12B0BDE8F081BC8C0100FF
:10F8900035F3000091EE0000E5400000913A0000D1
:10F8A00030B4D0F80D30D0F809001B68C068DC888F
:10F8B00001F1800504FB02F21212FF2AA8BFFF2209
:10F8C0001A8192B251F8043B03FB02F393FBF4F369
:10F8D0008D4240F8043BF5D130BC7047F0B50F467F
:10F8E000D0F80D30D0F809201B68D468DA8885B0CC
:10F8F0001A81F4F7F7FBF4F7C1F8204680220021C3
:10F9000009F0A7F8074A0849084E094D00920191ED
:10F910002346384620226946CDE90265F6F7AAFD5E
:10F9200005B0F0BDE54000007D3A000005EF0000A5
:10F9300009EF0000002825DD2DE9F0039046043989
:10F9400082B04FEAE27901EB800051F8042FD3171F
:10F95000CDE90023DDE9002302FB09FCA2FB0867D7
:10F9600008FB03C3B40B1F4444EA8744BD13CDE92D
:10F970000045DDE9002388420A60E6D102B0BDE817
:10F98000F0037047704700BF70B5214E84B0FFF799
:10F9900059FDFFF7BDFDFEF72BFBF4F7B5F8FEF7B9
:10F9A00003FDFEF73BFB002234461A4B1A4DA3F829
:10F9B00068200FCD0FC40FCD0FC40FCD0FC4336817
:10F9C0002A680133226006D0082304A800F8043D09
:10F9D0000121F9F7D3FD01250E4B104CA3F8685017
:10F9E000F9F798FDF6F7CCF900230D482946009366
:10F9F0001A4605680220A84700F06CFB2568FEF750
:10FA0000D9FDA8702468FEF7EFFDE07004B070BD6A
:10FA1000402000200000105000FE0100340A0020A9
:10FA20008CC701000246034B51680068926807C307
:10FA3000704700BF502700202DE9F04F964683B055
:10FA4000544E9DF834709DF830C098460097634638
:10FA50000D46B6F90620B6F90410044670469DF826
:10FA60003870FBF7B9F83378800290FBF8F0002B80
:10FA70004BD0A91C96F801904B002A4604EB030ECC
:10FA800003F10208B9F1000F50D13EF8069C05F1D0
:10FA9000FF3C24F80890A3F108053EF8043C2544F7
:10FAA00024F811306189238961802380531ED2B3E9
:10FAB0001A4602F1010B4FEA4B0104EB010A063131
:10FAC00034F801903AF8028C34F81B30C84407FB34
:10FAD00008F9BAF8048096F903B043440BFB039885
:10FAE000BAF8023096F90290624509FB03834FEAA7
:10FAF000A31300FB03F34FEA2343635246D0012ACA
:10FB0000D4D1E38800226380D3E765B1A91C04EB5C
:10FB10004101043431F8022D00FB02F28C424FEA1D
:10FB200022428A80F6D103B0BDE8F08F00236380C3
:10FB3000238024F8113024F80830002DF3D07F0002
:10FB400004EB450131F802E996F90350B1F808C019
:10FB50000B88CA889C4538BF9C46964538BF964658
:10FB60000CFB07F36A000EFB02338D8896F9022026
:10FB70008C4205FB02324FEAA21200FB02F24FEA6E
:10FB800022420A81DED103B0BDE8F08F2B88AEF8A7
:10FB900000308BE750270020F0B505462C4C426919
:10FBA00094F9033094F90270C3F12003E07AC7EBB3
:10FBB0004307A37A85B0C7F34707CDE90107009350
:10FBC00005F12C0020230E460F21FFF735FF617A47
:10FBD000237A05F152046A692046CDE901170093A2
:10FBE00020210F23FFF728FFFEF7AAFA20462E2335
:10FBF0004FF0804403F1600230F8021D013B1F2BDF
:10FC000044F82210F6D14FF0804405F19A0232F800
:10FC1000020D03F16001013B44F82100591CF6D1AB
:10FC20000120FEF74FFA2846FEF792FAB4F84C305E
:10FC30001BB2336094F85030337294F851307372C1
:10FC400094F85230B37294F85330F37205B0F0BDAB
:10FC50005027002038B504220125144B144C1D7187
:10FC60002260FEF7F5FFFEF78FFFF9F753FC837E66
:10FC700043B9104B1B682BB10F4A126812B90F4AD7
:10FC8000157098470E4BD3F80021120708D50022B3
:10FC900008250C480C49C3F880510270C1F8402176
:10FCA00001211023094AD160236038BD202700209C
:10FCB000A40C002098170020801C0020971700201B
:10FCC00000E100E0A00C00200000025000000850FD
:10FCD0000122052138B50D4B0D4C5A712160FEF7FC
:10FCE000BBFF0C4BD3F80021120708D500220825D2
:10FCF00009480A49C3F880510270C1F84021012126
:10FD00001023074AD160236038BD00BF20270020A0
:10FD1000A40C002000E100E0A00C00200000025034
:10FD2000000009500121032238B50B4B0B4DD9704F
:10FD30000B4C2B7822601BB1FEF78AFE094B186032
:10FD400001232B70FEF776FE00211023064AC2F82D
:10FD50004011236038BD00BF20270020A00C0020E8
:10FD6000A40C0020482700200000025001234FF07F
:10FD70006050102110B4034A034CE372836210BC3C
:10FD800011607047A40C0020202700200F21124A88
:10FD9000124B11605B6F84B00193019B23F4FF63EE
:10FDA00023F007030293019B23F07F030393029B3D
:10FDB000B3F5800F0AD0039A094B9A4206D0019AF4
:10FDC000084B9A4202D20122074B1A700122034BC0
:10FDD000A3F86C2004B07047A40C00200000105061
:10FDE00080FF010000FC01005C27002008B5FFF740
:10FDF000CBFD00F0D5FD002008BD00BF704700BF5F
:10FE000008B54FF0CD3203490348FCF73BFC002016
:10FE100008BD00BF3046002030320020704700BFD0
:10FE200008B5F1F747FFD0F80930986808BD00BF62
:10FE300040F215132DE9F0431C4A1D4D1D4C83B0B3
:10FE400012682146009363202B46F2F7A1FBF1F7DD
:10FE50002DFF8146F1F72EFF80460027D0F809607C
:10FE6000F3F7D8FF4846F3F727FF4046F3F724FFA0
:10FE700008F08EFDF760F1F74DFF3760F1F71EFFD8
:10FE8000064601460120F3F707FF31460220F3F74B
:10FE900003FF4FF49770084A2B46126821460090E2
:10FEA0006320F2F775FB03B0BDE8F0834C07002038
:10FEB00008A70100E8A601005007002051222DE903
:10FEC000F041304B82B000921A682F492F4B6320CB
:10FED000F2F75EFBFEF78CF80546F1F7EFFE0446FD
:10FEE00001462A460120F3F789FE2A4621460220D0
:10FEF000F3F784FEF1F7DAFE0746F1F7DBFE04467E
:10FF000008F030FD804608F031FDC7F80D0008F01C
:10FF100031FD2946C4F80D003846D4F80960F3F7DE
:10FF2000F3FEF3F71BFF29462046F3F7EDFEF3F748
:10FF300015FFF36803B33368DBB120460221FFF7F6
:10FF4000CDFC3946022322464046FFF755FCD8F83F
:10FF50002020F1682046FFF7A3FC7A220C4B009288
:10FF60001A680949094B6320F2F712FB02B0BDE899
:10FF7000F081F1F7C5FEE0E708F000FD08F010FDA4
:10FF8000F060D8E74C070020F8A6010008A70100A0
:10FF9000500700202DE9F047A8B0F1F78BFE064688
:10FFA00007A8D6F80940FEF727F8D6F80D30079ACB
:10FFB0005968A36809780492276818ADCDE90257FB
:10FFC00008AA0192E268C5B2009208461A222946A0
:10FFD000FDF7A2FB65B1236803EB45010239023B43
:10FFE00033F9022F002AB8BF52428B421A80F7D150
:10FFF00001274FF0040AAB200621DFF880901C4A4D
:020000021000EC
:10000000E3680590CDE90171CDE9032939462A4617
:10001000CDF800A06220F2F773FA4FF00008AD208F
:10002000D6F80D20A3685168124A0978CDE90490EA
:100030000392CDF800A02A46CDE901887220F2F79C
:100040005FFA02264FF0AF0C0B4823682A46039054
:10005000CDF81090CDE901783946CDF814C000965E
:100060006920F2F74DFA206828B0BDE8F08700BF9C
:10007000E8B0010000B1010018B1010008A70100BB
:1000800008B50220F3F7F0FFBDE80840F4F77CB8AC
:1000900030B5044687B0FEF781FA832101220023A0
:1000A0000334094D0444059108480949CDE9013359
:1000B0000490039100922B46114664202C70F2F7B5
:1000C0001FFA07B030BD00BF8407002008A7010059
:1000D000EC9901000148F7F737BB00BF400800204A
:1000E0002DE9F04F8FB006AFFEF758FA01244FF01C
:1000F0000009D2220426DFF8B0C29E4D07F120038A
:1001000043F8140D21460592CDE903C5CDE9014917
:10011000224600966420F2F7F3F903224FF0D40C44
:10012000954807F12003DFF8848243F8102D21461B
:1001300003900495CDE9014900962246CDF814C0FC
:100140006420F2F7DDF9D8F80410FB68CA1D22F02C
:1001500007023869ADEB020D034406AA49457A60EF
:10016000FB600DDD01EBD170A3EB60031046DBB249
:10017000084402F8013B824203F10103DBB2F8D1EB
:1001800089000A3121F00701ADEB010D0DF11809CD
:100190004846F7F7EBFADF22764B009277490022C8
:1001A0006420F2F7F5F9494607F11802D8F804007F
:1001B0000124F7F763FB00264FF0040BE422704B99
:1001C00007F1200A049521464AF8040D0592CDE96D
:1001D000026322466B4B6420CDE900B4F2F790F93C
:1001E000E523D8F804200593674B21460393642048
:1001F0007B680495CDE901660094F2F781F9E62366
:100200006249D8F804206420059303914B462146A7
:100210000495CDE90146CDF800B0F2F771F9E82375
:1002200005935B4B22460393214607F11803642094
:100230000495CDE90146CDF800B0F2F761F9E92364
:10024000544A21460593039253462246642004955E
:10025000CDE90146CDF800B0F2F752F94846F7F77C
:10026000EBFAEE23324600934B49424B6420F2F7FF
:100270008FF9D8F804304946023B184607F11402BA
:10028000C7E90563F7F7FAFA00B10138012400263F
:100290004FF0040BF822F861404807F1180305926B
:1002A0002146224603900495CDE90146CDF800B0E1
:1002B0006420F2F725F9F920334BD8F804202146C1
:1002C000039305907B68CDE9016600940495642052
:1002D000F2F716F9FA202D4BD8F8042021460393A3
:1002E00005904B46CDE90146CDF800B00495642059
:1002F000F2F706F9FC20264B22460393214607F12C
:1003000014030590CDE90146CDF800B004956420B2
:10031000F2F7F6F8FD2040F201181E4B2246039337
:10032000214653460590CDE90146CDF800B004952D
:100330006420F2F7E5F8F969FB68194ADFF870E024
:1003400012680B4417485FFA83FC82F802C07346B8
:100350000390CDE9016600940495CDF814802246FF
:10036000214664208EF800C0F2F7CAF82437BD4653
:10037000BDE8F08F08A7010024A7010034A7010001
:1003800060A70100440800206CA7010078A70100C5
:1003900074A7010084A7010094A70100CCA7010065
:1003A000340A0020EC99010018A701004008002041
:1003B0008407002040F2091330B50D4A0D4D0E4C54
:1003C00083B012682146009363202B46F2F7E0F8D1
:1003D000FFF786FE40F20D10084A2B4612682146B0
:1003E00000906320F2F7D4F8002003B030BD00BFC6
:1003F0004C07002008A70100D8A6010050070020E4
:1004000040F257132DE9F041174A184D184C82B0AD
:1004100012682146009363202B46F2F7B9F8F1F7F2
:1004200045FC8046F1F794FC0746F1F72FFD0646A0
:10043000F3F7F0FC4046F3F73FFC3846F3F73CFC9B
:100440003046F3F739FCF1F7ADFCF1F749FD4FF415
:10045000B670084A2B461268214600906320F2F7D6
:1004600097F802B0BDE8F0814C07002010A8010009
:10047000FCA7010050070020CF222DE9F04FD44BFC
:10048000ADF66C0D00921A68D249D34B6320F2F797
:100490007FF8F1F70BFCD0F80940F1F759FCD0F8E0
:1004A00009300425079308F08DFAF1F7EFFCD0F836
:1004B000098008F09BFA4FF4707200213AA808F006
:1004C000C8FA402200211AA808F0C3FA1E2200210F
:1004D0000AA808F0BEFA4FF4707200210DF595607D
:1004E00008F0B7FA402200212AA808F0B2FA1E222A
:1004F00012A8002108F0ADFAE268DDF81CA009920C
:10050000043A08920DF6A60919AF0DF1E606F3F7C5
:10051000E9FDF3F739FEDDF820C00DF2E644604650
:10052000A4F1400131F8022F50F8043FA1421344D6
:100530000B80F7D140344C450CF1800CEFD1D8F84A
:1005400010000DF14601043831F8022F50F8043F35
:10055000B94213440B80F7D1DAF810300DF1A6023E
:10056000A3F1040C32F8020F5CF8043FB2420344DA
:100570001380F7D1013DCAD10DF2A6400DF66606F3
:1005800000F1400530F9023F002BB8BF03339B1048
:10059000A8420380F6D1B042F2D10DF1460636F9F9
:1005A000023F002BB8BF03339B108E423380F6D13D
:1005B0000DF1A60535F9023F002BB8BF03339B10A0
:1005C00095422B80F6D1F8F793FF0B28824F40F02D
:1005D000F880F3F787FDF3F7D7FD4FF491723B46B0
:1005E00000927E4900226020F1F7D2FF2AAB0DF580
:1005F0009562DDF820A00DF2E649A3EB020B504610
:10060000A646A9F140020BEB090132F9023F50F86E
:10061000044F31F902CF1B1B9C45B8BF0B8091459D
:10062000F3D109F14009F14574460AF1800AE6D197
:10063000D8F810000DF146020DF12601043832F908
:10064000023F50F8044F31F902CF1B1B9C45B8BF45
:100650000B80B242F3D1079B0DF1A60218690DF190
:100660006601043832F9023F50F8044F31F902CFE5
:100670001B1B9C45B8BF0B80AA42F3D14FF0000A68
:100680004FF0040B40F23713554A05930392CDF80F
:1006900000B0099B20220F2172200497CDE901AA06
:1006A0004FF001097446F1F72BFF4FF49C714D4A4E
:1006B000D8F810307220CDF800B0CDE90471039263
:1006C00049460F22CDF808A0CDF80490F1F718FFA5
:1006D00040F23910079B444A1B694946CDF800B0E7
:1006E0000590039272202022CDE9019A0497F1F738
:1006F00007FF4FF0020B40F23B123C4BCDE9047276
:10070000039320220DF595630F216220CDE9019A14
:10071000CDF800B0F1F7F4FE4FF49E72344B494629
:10072000059203930F2212AB6220CDE9019ACDF816
:1007300000B00497F1F7E4FE40F23D122D4B49461C
:100740000592039320222AAB6220CDE9019ACDF8CD
:1007500000B00497F1F7D4FE40F23F12264BCDE9EA
:100760000472039320223AAB0F216920CDE9019A4C
:10077000CDF800B0F1F7C4FE4FF4A0721F4B49460C
:10078000059203930F220AAB6920CDE9019ACDF8B7
:1007900000B00497F1F7B4FE40F24112184B4946FD
:1007A000CDE90472039320221AAB6920CDE9019AA6
:1007B000CDF800B0F1F7A4FEF8F79AFE0B283FF44D
:1007C00008AF40F24F120F4B00921A681CE000BFB6
:1007D0004C070020E8A7010010A8010004A00100B8
:1007E00024A8010038A801004CA8010060A801005D
:1007F00070A8010078A8010080A8010090A801005D
:100800009CA80100500700200449054B6320F1F724
:10081000BFFE00200DF66C0DBDE8F08FE8A70100CB
:1008200010A80100A6222DE9F041554B82B000929C
:100830001A685449544B6320F1F7AAFEFDF7D8FB20
:100840000446F1F733FA0746F1F782FA0546F1F765
:100850001DFB064608F0B2F8C5F80D0008F0C2F816
:10086000C6F80D002046F1F777FA2046F1F712FBA3
:1008700021463046F3F748FAF3F770FA2146284646
:10088000F3F742FAF3F76AFA21463846F3F73CFAEF
:10089000F3F764FAF1F70AFA0446F1F759FA064653
:1008A000F1F7F4FA054608F08DF808F09FF8FDF727
:1008B0009FFB074600212078F3F7ACFB2146384622
:1008C000F2F700FFD4F80130DB7A1BB120782F4912
:1008D000F3F7A0FBF3F706FCF3F756FC00213078A2
:1008E000F3F798FBFDF784FB294A3146F4F7A0FAA9
:1008F00030782849F3F78EFB00212878F3F78AFB3C
:10090000FDF776FB224A2946F4F7D8FD22492878DC
:10091000F3F780FBF1F7CAF90446F1F719FA074635
:10092000F1F7B4FA054608F01DF8804608F04AF8D9
:10093000064608F05BF8D4F80D30046A1868D8F859
:100940002020C1880830366AFEF7FEFDD7F80D007A
:10095000324601890A30FEF7F7FDD5F80D00224630
:1009600001890A30FEF7F0FDC9220C4B00921A688B
:100970000449054B6320F1F70BFE02B0BDE8F0819E
:100980004C070020D4A7010010A80100CD340000BE
:10099000E540000059500000A1560000500700201B
:1009A0002DE9F04784B0F8F7A3FD3522254B264901
:1009B0000092054600226420F1F7EAFDFDF7EEFD06
:1009C000224A234B10701C68FDF7E8FD214EA070F1
:1009D000DFF88CA00024DFF86C90DFF888801E4FD1
:1009E000FEB1102C1DD833689847AC4201D0F8F7FF
:1009F00075FD0125CDB94FF0CD3239461748FBF7CB
:100A00009BFEF8F775FD8442F4D0B36803909847D5
:100A1000FAF7B2FA0398254604465AF82460002EE5
:100A2000DFD1F8F765FD0446F7E74B224B4600920D
:100A3000414600226020F1F7ABFD736898470546F8
:100A4000D9E700BF08A9010010A901008407002010
:100A5000340A0020400700203046002030320020B9
:100A6000C4A8010004A0010084B02DE9F0438FB0B8
:100A7000BDF8DEC1809DDFF8D0E005FB0CF58EFBF4
:100A80000564EF17B5F5C84FC7EB64174FF00006C4
:100A9000B4BFB8464FF0FF08819C054604FB0CF03C
:100AA0000DF15C0CB0F5C84FCDE90866CDE90A66DA
:100AB0008DF82080CDE90C668CE80E003DDA8EFBC7
:100AC000003EC417C4EB6E14E4B201264FF00008D8
:100AD0007022DFF878901A4B059231463246CDE904
:100AE0000339CDE9018808AB009664208DF82A40CF
:100AF000F1F706FD04244FF0750C12480EAB43F8D5
:100B00001C7D3246314600940390CDF81090CDE91B
:100B10000168CDF814C0642008ACF1F7F1FC0FCCEB
:100B20002860696003CC28612846AA60EB6069618F
:100B30000FB0BDE8F04304B07047FF24C5E700BF25
:100B4000A8A8010084B001001F85EB5108A901008D
:100B5000472370B50E4A0F4D0F4C82B012682146E4
:100B6000009363202B46F1F713FDF1F79FF806463B
:100B7000F3F750F93046F3F79FF84F20074A2B461A
:100B80001268214600906320F1F702FD02B070BDAB
:100B90004C07002054A9010038A90100500700208B
:100BA000382370B50F4A104D104C82B012682146A0
:100BB000009363202B46F1F7EBFCFDF719FA06468C
:100BC000F1F774F801463046F1F724FE3F20084A59
:100BD0002B461268214600906320F1F7D9FC0020D3
:100BE00002B070BD4C07002054A901001CA90100EF
:100BF00050070020262370B5144A154D154C82B0BD
:100C000012682146009363202B46F1F7C1FCFDF7E3
:100C1000EFF90646F1F74AF83146F3F775F8F3F7BE
:100C20009DF807F09FFE0646807BFDF745FA3046AB
:100C3000FEF7D2FD3220084A2B461268214600906A
:100C40006320F1F7A5FC02B070BD00BF4C07002087
:100C500054A90100A8990100500700204B23F0B5CA
:100C6000114A124D124C83B0126821460093632042
:100C70002B46F1F78DFCF1F719F80746F1F71AF852
:100C80000646F3F7C7F83846F3F716F83046F3F799
:100C900013F85520074A2B4612682146009063201E
:100CA000F1F776FC03B0F0BD4C07002098A90100D5
:100CB00084A90100500700203A23F0B5114A124DD3
:100CC000124C83B012682146009363202B46F1F743
:100CD0005FFCFDF78DF90646F0F7E8FF0746F0F7F1
:100CE000E9FF39463046F2F7E5FD4320084A2B4636
:100CF0001268214600906320F1F74AFC002003B0FF
:100D0000F0BD00BF4C07002098A9010070A90100A8
:100D10005007002026232DE9F0411A4A1A4D1B4C9A
:100D200082B012682146009363202B46F1F730FC15
:100D3000F0F7BCFF8046F0F7BDFF0746FDF758F916
:100D4000064601464046F2F7DFFFF3F707F8314663
:100D50003846F2F7D9FFF3F701F807F003FE06462D
:100D6000807BFDF7A9F93046FEF736FD3420084AAE
:100D70002B461268214600906320F1F709FC02B06F
:100D8000BDE8F0814C07002098A90100C49901003A
:100D9000500700202DE9F04383B000F031FB81467D
:100DA00000F032FB804600F089FD074600F08AFD26
:100DB00073230646134D144C144A214612686320CF
:100DC00000932B46F1F7E4FBF3F7F4F9F3F722F87D
:100DD0004846F2F771FF4046F2F76EFF3846F2F7E9
:100DE0006BFF3046F2F768FF00F0CAFD8020084A2A
:100DF0002B461268214600906320F1F7C9FB03B02F
:100E0000BDE8F083C4A90100B8A901004C07002087
:100E1000500700202B232DE9F0471F4A1F4D204C7F
:100E200082B012682146009363202B46F1F7B0FB95
:100E3000FDF7DEF80646F8F785FD00F0E1FA824698
:100E400000F0E2FA814600F039FD804600F03AFDFC
:100E5000074600F001FBCAF80D0000F0F9FAC9F8E6
:100E60000D0000F01BFDC8F80D0000F01BFDC7F8D9
:100E70000D00304600F048FD304600F063FD3C2098
:100E8000084A2B461268214600906320F1F780FB48
:100E900002B0BDE8F08700BF4C070020C4A90100E4
:100EA000ACA901005007002008B5F8F74BFD431E20
:100EB0001D2B1BD8DFE803F02020201A0F241A1A5C
:100EC0001A1A1A1A1A1A1A1A20201A311A1A313131
:100ED0001A1A3131201C0021124A0846D2F88030FB
:100EE00023F00103C2F88030F8F732FD012008BD7D
:100EF00000F0BEFA012008BD00F05AFA012008BD3A
:100F00000021084A0846D2F8803043F00103C2F8B5
:100F10008030F8F71DFD012008BD00F061FD0120C3
:100F200008BD00BF0000025070B5FDF761F804462F
:100F300000F06EFA0546014622460120F2F75EFEF9
:100F4000224629460220F2F759FE00F059FA0546DA
:100F500000F05AFA064600F07FFAC5F80D0000F0DE
:100F600077FA2146C6F80D002846F2F7CDFEF2F7D3
:100F7000F5FE21463046F2F7C7FEF2F7EFFE2946AE
:100F80002046F2F79FFB07F0EDFCD5F80D301B680B
:100F9000DA881A8170BD00BF2DE9F04FADF6044D1F
:100FA0000546099000F02CFA0A9000F02DFA0B90FB
:100FB0000120F3F721F8002800F057814FF47072F8
:100FC0000021044630A807F044FD4FF4F0620021F0
:100FD0000DF5906007F03DFD4FF4F062FF21A7484A
:100FE00007F037FD0023032D0F9300F05381D4F851
:100FF00001301B790D93099B1D2B00F03A811D27B1
:10100000099BDFF8788203F1FF39F3F76BF80026CC
:10101000F3F7BAF84FF0040A83220A9B9848D3F8F2
:1010200009100B9BCD68D3F8093096499C682B4674
:101030000491039005920F2120227220CDE90166D0
:10104000CDF800A0F1F75CFA8422B3468D498E4BAF
:1010500004910393059223462022CDE90166CDF841
:1010600000A001217220F1F74BFA0F9B2A1F0C936D
:101070009C465FFA89F306920DF5906508934FF050
:10108000000A30AB03EB8B13069807934FEA4B161D
:1010900050F8043F1A46B9F11C0F1CD8DFE809F0DC
:1010A0000F146F1B1B1B1B1B1B1B1B1B1B1B1B1B4F
:1010B0000F0F1B1B1B1B1B1B1B1B1B1B580054F860
:1010C0002A209A1A22EAE27255F82A100A4445F8B0
:1010D0002A20002F6BD00AF1010ABAF1200FD7D1D4
:1010E000069B0BF1010B8033BBF10F0F05F180055F
:1010F0000CF1200C0693C2D117F1FF3785D211A84D
:101100003A220021CDF818B007F0A3FC099B033B5D
:101110001A2B00F2EB80DFE813F05700E900E9003A
:10112000E900E900E900E900E900E900E900E90077
:10113000E900E900E900EE00EE00E900E900E9005D
:10114000E900E900E900E900E900E900E900E00060
:1011500054F82A1055F82A205B1A002BA8BFD21881
:1011600045F82A20002FB6D1484BA3FB02321209C2
:10117000312A45F82A20AED8ADF8C070ABE755F853
:101180002A2006EB0A0E9A4238BF1A4645F82A2052
:1011900058F82E108B4228BF0B46D21AD2087F2A4D
:1011A00028BF7F2248F82E300CF80A2093E7374BEF
:1011B000A3FB0232089B1209012B96BF079B45F83F
:1011C0002A2023F81A2086E7202501230C9E20AC34
:1011D000002243F0800363719DF81830657011AFF1
:1011E000237084F802A0E27022710DF186050DF1E2
:1011F000740EBC46BCE80F00F44528606960AA6024
:10120000EB6007F1100705F11005F2D13B4603CB67
:10121000286069601B8820462B813146F8F798FBCF
:10122000F2F7C8FFF2F7F6FD0FA81949F9F730FEFB
:101230000A9D9DF83410D5F8013028461971F2F74F
:101240003BFD0B9C2046F2F737FD00F009F900F05A
:10125000EFF800F0F5F8D5F801100120F2F71CFDC9
:10126000D4F801100220F2F717FD0DF6044DBDE889
:10127000F08F0123ADF8C030C1E600BF00008560EB
:10128000F8A90100ECA90100E8BF0100898888885D
:10129000E4A901000FA8454A4FF4F071F9F76CFD7D
:1012A0004FF4F0727F210F9807F0D3FBD4F8013090
:1012B0001B790D93FCF79CFE0123D4F801100B71F0
:1012C000D4F80D30D4F805501A68D4F80930527BA0
:1012D00000955B68F1F7BCF991E64FF0010A30AE7A
:1012E0005546CDF818A0022320AC71E730AE20257A
:1012F000022320AC6CE7099B112B4DD04FF00E0C54
:1013000010AEB346202501210023CDF818C020AC33
:101310000E221746114403EB41110DF5906303EBC8
:10132000810132600DF538680DF5886E1F20079534
:10133000206017E051F8203058F820904FF47A756B
:1013400003EB09025210012AB8BF0122A3EB0903E3
:1013500005FB03F393FBF2F32EF810300138421C27
:1013600020600BD0DBF800306345E3DB4FF0000377
:101370002EF810300138421C2060F3D1013F7B1C55
:10138000079D3760A1F18001A8F18008AEF1400E01
:10139000CCD130AE02231BE74FF01F0C20AC6546CA
:1013A000A3460021012310AEB2E700BFE4A901006B
:1013B00040F22F1370B506460D4D0E4C0E4A82B00A
:1013C00012682146009363202B46F1F7E1F8FFF7FE
:1013D000ABFD3046FFF7E0FD40F23510074A2B46E3
:1013E0001268214600906320F1F7D2F802B070BD78
:1013F000ECA90100D0A901004C07002050070020F3
:1014000000487047C800002000487047FC040020D6
:1014100010B5064C04F11000FCF7EEFD207504F148
:101420001800FCF7EFFD2077204610BD6C0D002062
:1014300001490248F9F72CBD04AE01003C0D002023
:1014400001490248F9F724BD30AE0100980D002093
:1014500000487047B40D002000487047900D0020F0
:1014600001490248F9F714BD1CAE010060270020B5
:1014700009222DE9F04F0026ADF69C0D574B009246
:101480001A685749574B63200DF1740BF1F780F838
:101490003146A222584607F0DCFAADF83060FFF77B
:1014A000AFFF81460790FFF7B3FF0746FFF7ACFF9A
:1014B00080460890FCF79CFD054631464FF4F062EB
:1014C00046A807F0C6FA2A4639460120F2F796FBED
:1014D0002A4639460220F2F791FB29464846F2F7A0
:1014E00013FCF2F73BFC29464046F2F70DFCF2F7FD
:1014F00035FC01233446B2461D26DFF8F480ABF8F4
:101500000030F2F7EFFDF2F73FFE3F22079B002786
:10151000D3F80910089BCD68D3F809303149D3F8C6
:1015200008900592042230482B46049103900092C3
:101530000F2120227220CDE90177F0F7E1FF04238B
:10154000402200932749294B0491039305924B466F
:10155000CDE90177202201217220F0F7D1FF7C35FF
:10156000A9F1040E0DF58C79A5F18000F4464946E9
:10157000234603E0A84226D051F8043F50F8044F18
:101580005CF8042FA41A002CACBF1C191C1C0C60A6
:10159000002EEFD1A8FB04342409312C0C60E9D8CB
:1015A000BAF10E0FABF8006005D80AF1010A5FFA34
:1015B0008AFA2BF81A7001370F2F05F1800519D020
:1015C00059F8804FD0E701370F2F00F18005F7D190
:1015D00016F1FF360ED3469C93E700BF4C07002060
:1015E00048AE01005CAE0100F8A90100E8BF0100AF
:1015F00089888888F2F70EFC0798F2F75DFB089857
:10160000F2F75AFBFCF7F4FCBC220021064646A880
:1016100007F01FFA00F052F9054600F053F90446AE
:1016200000F044F9C5F80D0000F044F9C4F80D00CD
:1016300000F04CF9C5F8010000F056F94FF04053A6
:1016400093F88C20C4F801006FF3000283F88C201B
:1016500093F88C20D5F801106FF3410283F88C20A9
:1016600005203246F2F7CAFA3246D4F801100620B5
:10167000F2F7C4FA31462046F2F746FBF2F76EFB6A
:1016800031462846F2F740FBF2F768FB2946304620
:101690007A4AF3F7CDFB21463046784AF3F70EFF3E
:1016A00020210F224FF00309D5F80900744B089050
:1016B000D4F80900CDE90E120D930AF10103099047
:1016C000079300212878F2F7A5FC6C4A294630469A
:1016D000F3F7AEFB6B492878F2F79CFC00212078E9
:1016E000F2F798FC654A21463046F3F7E7FE20788A
:1016F0006549F2F78FFC4FF0010200274FF0200CF4
:10170000089B5868079B2BF81320002245AB03EB7E
:10171000C7115E4B043803EB471E0B944C6850F81E
:10172000043F234441F8043FB9F1000F7CD001325B
:101730006245F3DB0B9C002F70D019F1FF39C0D24A
:10174000F2F768FB2846F2F7B7FA2046F2F7B4FA48
:101750004FF0405393F88C103A2241F0010183F886
:101760008C1093F88C00002140F0020083F88C006C
:101770000EA807F06EF9002307220A254FF4024E47
:101780004FF0050C09260B200C21ADF818318DF80F
:101790001A318DF81B31ADF83A209DF831309DF8A3
:1017A0003020ADF83C70ADF84470ADF842500EAC4E
:1017B000ADF840A0ADF81CE18DF838C0ADF83E6042
:1017C000ADF84600ADF84A10ADF84820ADF84C3001
:1017D0000DF58F751AAF26460FCEBE4228606960A0
:1017E000AA60EB6004F1100405F11005F3D1234663
:1017F00003CB286069601B88594646A82B81F8F7FF
:10180000A7F8E022224B00921A682249224B63205B
:10181000F0F7BEFE0DF69C0DBDE8F08F099BDDF8DC
:101820003CC00127586870E71EF802809B08B8F199
:10183000000F08BF4FF07F0803FB08F30DAC34F82E
:101840001780DB0943450B60FFF471AF4FF00008D0
:101850000CABDB5D079C0A930A9B2BF814800133C9
:101860000DF1300808F807309DF830309DF83180D0
:10187000234443442BF8132059E700BF19410000CB
:1018800020CB80BB59500000A1560000DCAE010007
:101890005007002048AE01005CAE010000487047D0
:1018A0009C0800200048704714050020004870473D
:1018B000240D002000487047040E002000487047A7
:1018C000D40D002000487047EC0D002010B5054CE9
:1018D00004F10C00FCF790FBE368207523612046BF
:1018E00010BD00BF280F002010B5064C04F10C00FD
:1018F000FCF788FB207504F11000FCF789FB2046FB
:1019000010BD00BFA00F002038B50A4C41780A4A2C
:101910008D002046F9F730FA2946201D074AF9F7CD
:101920002BFA294604F10800054ABDE83840F9F7CA
:1019300023BA00BF340E00201CAF010038AF0100F5
:1019400054AF010038B50A4C01780A4A8D00204690
:10195000F9F712FA2946201D074AF9F70DFA294628
:1019600004F10800054ABDE83840F9F705BA00BFA0
:10197000900E00207CAF010098AF0100B4AF0100D1
:1019800038B50F4D0F492846F9F782FA0E4C281D3D
:101990000E49F9F77DFA05F108000D49F9F778FAD3
:1019A00020460C49F9F774FA201D0B49F9F770FA33
:1019B00004F108000949BDE83840F9F769BA00BFE9
:1019C000340E00201CAF0100900E002038AF010043
:1019D00054AF01007CAF010098AF0100B4AF01002B
:1019E00040F2BB222DE9F04FCC4BADF5377D009294
:1019F0001A68CB49CB4B044606906320F0F7C8FD2C
:101A0000FCF7F6FABC220C90002158A807F021F848
:101A10005E22FF2140A807F01CF887A8BC22002105
:101A200007F017F81B2C00F04082069B1C2B00F0DF
:101A30009C82069B142B15AB0E9300F0FD8118467B
:101A40002F22002107F005F8B74CB84EB84FB94A1D
:101A5000B94B04F10C00C6F80D200996C7F80D30FB
:101A60000A97FCF7C9FAB54DE368207505F10C003B
:101A70002361C6F80140FCF7C5FA3446287505F124
:101A80001000FCF7C5FAD6F801100C9E052032466E
:101A9000C7F80150F2F7B2F83246D7F80110062025
:101AA000F2F7ACF831463846F2F72EF9F2F756F96C
:101AB00031462046F2F728F9F2F750F9D4F8093008
:101AC0000F93D7F809301093069B172B00F0CD81A8
:101AD00004230B930F232022DDF82CA0CDE9132340
:101AE000D146974B0D9309F1FF39B9F1FF3F069BA2
:101AF00000F09180143B082BF5D801A252F823F096
:101B0000051E0100E71A0100E71A0100551D01003A
:101B1000051E0100E71A0100E71A0100251B01005C
:101B2000051E0100099B00211878F2F773FA0A9B41
:101B300000211878F2F76EFA824B0D930D9D0C9CE4
:101B40002A467A492046F3F773F92A46784920460F
:101B5000F3F7B4FC4D46099B7B491878F2F75AFA23
:101B60000A9B7A491878F2F755FA13980F9B00F1FF
:101B7000804101395C6889000B1D58AA11441C443E
:101B800010F1FF3017D354F8043D0A68134441F8AC
:101B90000439002DF4D10E9A0B9E125CB3FBF6F3C0
:101BA000002A08BF7F2203FB02F310F1FF304FEA47
:101BB000D3134B60E7D2149C109B04F11F015868AB
:101BC0008900A1F17C0358AA1144184414F1FF3490
:101BD00019D30B6850F8042D134441F80439002D33
:101BE000F4D10E9A0B9E224492F82020B3FBF6F318
:101BF000002A08BF7F2203FB02F314F1FF344FEAEF
:101C0000D3134B60E5D2A94609F1FF39B9F1FF3F83
